:020000040800F2
:108000004890002051830008A1DB0008A1CE0008A1
:1080100055D1000801AF000875E400080000000019
:10802000000000000000000000000000B98200080D
:1080300017B0000800000000FD820008A5DB000862
:108040006B8300086B8300086B8300086B83000858
:108050006B8300086B8300086B8300086B83000848
:108060006B8300086B8300086B8300086B83000838
:108070006B830008D5AF00086B8300086B83000892
:108080006B8300086B8300086B8300086B83000818
:108090006B8300086B8300086B8300086B83000808
:1080A0006B8300086B8300086B8300086B830008F8
:1080B00079DC00086B8300086B8300086B83000881
:1080C0006B8300086B8300086B8300086B830008D8
:1080D0006B830008F5E1000875E20008D9E20008AA
:1080E0006B8300086B8300086B8300086B830008B8
:1080F0006B8300086B8300086B8300086B830008A8
:108100006B8300086B8300086B8300086B83000897
:1081100011DD0008ADDE00086B8300086B830008EA
:108120006B8300086B830008E1AF00086B830008D5
:1081300000F002F800F0B0F80AA090E8000C8244C9
:108140008344AAF10107DA4501D100F0A5F8AFF2A6
:10815000090EBAE80F0013F0010F18BFFB1A43F025
:1081600001031847A0390100C03901000A444FF04B
:10817000000C10F8013B13F0070408BF10F8014B86
:108180001D1108BF10F8015B641E05D010F8016BCB
:10819000641E01F8016BF9D113F0080F1EBF10F82F
:1081A000014BAD1C0C1B09D16D1E58BF01F801CB52
:1081B000FAD505E014F8016B01F8016B6D1EF9D5D5
:1081C0009142D6D3704700000023002400250026EA
:1081D000103A28BF78C1FBD8520728BF30C148BF2A
:1081E0000B6070476E2900F00F86702900F05F82E7
:1081F000662912F04786652912F04486672912F035
:108200004186612912F0408603681B0A28BF41F0AD
:108210008001692900F0D081642900F0CD817529A1
:1082200000F0CA816F2901F00B81782900F02B82C0
:10823000E92901F0A580E42901F0A280F52901F0E7
:108240009F80EF2901F00881F82900F02A82036855
:10825000DB0928BF41F08001632901F026807329E2
:1082600001F02B80E32901F0E583F32901F0EA8393
:10827000002070471FB501F0C3F904000020002161
:1082800011F062FC401C60600020002111F072FCC3
:10829000E0601FBD10B510BD01F0D6FC1146FFF720
:1082A000E9FF0CF0FBFB01F055FF03B4FFF7F2FF11
:1082B00003BC01F055FF0000224B19680868B0E8C4
:1082C000F00F80F30988BFF36F8F4FF0000080F349
:1082D00011884EF00D0E704700000000064800683F
:1082E000006880F3088862B661B6BFF34F8FBFF3B2
:1082F0006F8F00DF00BF00BF08ED00E0EFF30980E3
:10830000BFF36F8F0F4B1A6820E9F00F106008B5AC
:108310004FF0500080F31188BFF34F8FBFF36F8F82
:1083200010F064FB4FF0000080F31188BDE80840B6
:1083300019680868B0E8F00F80F30988BFF36F8F01
:10834000704700BF00000020EFF305807047000079
:108350000948804709480047FEE7FEE7FEE7FEE7D9
:10836000FEE7FEE7FEE7FEE7FEE7FEE70448054915
:10837000054A064B7047000031DC000831810008D7
:10838000488A002048900020488C0020488C00201B
:1083900053EA020C00F069802DE9F04B4FF0000623
:1083A000002B1FBFB3FA83F503FA05F424FA05F690
:1083B0005E4012BF1643B2FA82F502FA05F4C5F127
:1083C00020051EBF22FA05FC44EA0C04203556EABB
:1083D000044C4FEA144418BF641C4FF000084FF0DF
:1083E0000009904271EB030C39D3002919BFB1FA8F
:1083F00081F701FA07F6B0FA80F700FA07F6C7F13D
:1084000020071EBF20FA07FC46EA0C062037B6FB01
:10841000F4FCA7EB0507103F07F01F0BCBF120067C
:108420000CFA0BFB2CFA06F644BFB3460026202FAD
:10843000A4BF5E464FF0000B5BEA060C08BF4FF08E
:10844000010B19EB0B09ABFB027C48EB0608C01BC8
:1084500006FB02CC0BFB03CC71EB0C01C1E70B4616
:10846000024641464846BDE8F08B13B54FF0000088
:108470004FF00001AFF30080BDE81C4070470000E2
:108480007CB51D4616460C00009001D02044401ECD
:10849000074B7B442A4669460190304600F0DBFEDC
:1084A00005461CB10020694600F0E8FE28467CBD68
:1084B000F10D00000FB41CB5084B06AA7B446946B9
:1084C0000090059800F0C7FE04460020694600F0C1
:1084D000D5FE20461CBC5DF814FB0000BD0D00005D
:1084E0000FB47CB50C0009AA009001D02044401EB6
:1084F000084B7B4469460190089800F0ACFE0546A5
:108500001CB10020694600F0B9FE28467CBC5DF82D
:1085100014FB0000910D000070B5044685690068E9
:10852000C10601D5302600E02026C00707D070BD67
:10853000D4E9012130469047206A401C20626D1E1C
:10854000F6D570BD70B5044685690078C00707D1BF
:1085500070BDD4E9012120209047206A401C206290
:108560006D1EF6D570BD70B50C460546012A05D0C6
:108570002878800600D5EA69002302E0012305E09F
:108580005B1C934202D2E05C0028F9D1A869E6188E
:10859000C01AA861286A184428622846FFF7BCFF61
:1085A00004E0D5E9012114F8010B9047B442F8D357
:1085B0002846FFF7C7FF70BD2DE9F04106460024AD
:1085C00010687529314616A510D000F0B2FB0028BE
:1085D00002DA404213A507E031688A0701D512A5E7
:1085E00002E0490704D511A5012401E000F0AAFB2F
:1085F00000210A2206F1240709E0B0FBF2FCB0FBDF
:10860000F2F302FB1C00303078541846491C002855
:10861000F3D123462A463046BDE8F04100F09BBB2B
:10862000000000002D0000002B00000020000000D2
:10863000F0B40D460188090502D5214C7C4402E0C6
:108640001F4C7C440E34002100F1240608E002F0A7
:108650000F071209E75D42EA03721B097754491CB0
:1086600052EA0307F3D102780023120704D5702DD4
:1086700006D009B1022311342246F0BC00F06BBBD6
:1086800001231034F8E770B504460D462146106802
:1086900000F058FB024629462046BDE87040002302
:1086A000C6E7D21D22F00703D3E90023C0E7036821
:1086B000126843F0200303600823C3610023B7E777
:1086C000382A01002DE9F05F894604464FF0000A80
:1086D000DFF874B1FB44C0F820A02046E168884769
:1086E000002874D0252806D0D4E901219047206ABB
:1086F000401C2062F1E700265F462046E16888477B
:108700002028054607DB312D05D2781910F8200CFA
:1087100008B10643F1E7B00701D526F00406C4F816
:108720001CA00027C4F818A02A2D09D0284606F05E
:10873000E4FD38B304EB8708303DC8F8185019E061
:1087400059F8041B204604EB87029161E1688847D1
:10875000012F054618D1E069002820DA26F020060E
:108760001DE0D8F8180000EB800005EB4000303821
:10877000C8F818002046E1688847054606F0BDFDA8
:108780000028EED1012F0AD02E2D08D12046E16815
:1087900088477F1C0546022F46F02006C4DBA069EF
:1087A000002803DA404246F00106A061F00701D03C
:1087B00026F010066C2D0BD0682D09D04C2D39D029
:1087C0006A2D35D0742D35D07A2D33D016E038E0AF
:1087D000E1682F4620468847B842054609D16C2FEC
:1087E00026D04FF48060E16806432046884705465E
:1087F00004E06C2F1AD04FF4807006430DB3A5F13E
:108800004100192802D8203546F400664A46294618
:10881000204626604E46FFF7E5FC80B101280BD0CC
:10882000F61D26F0070000F1080956E74020E4E7AE
:108830008020D8E70020D6E706F104094DE7284656
:1088400052E7206ABDE8F09FC829010070B50646CE
:1088500000F060FA0468054630460A22002100F064
:1088600055FE2C6070BD401ECAB210F8011F8A422E
:1088700002D00029F9D10020704730B505460B46DB
:108880002A4613F8014B12F8010B08B1A042F8D0A8
:108890001CB1002802D06D1CF1E7284630BD40EA2B
:1088A000010310B59B070FD1042A0DD310C808C9C6
:1088B000121F9C42F8D020BA19BA884201D901206F
:1088C00010BD4FF0FF3010BD1AB1D30703D0521CBA
:1088D00007E0002010BD10F8013B11F8014B1B1BF5
:1088E00007D110F8013B11F8014B1B1B01D1921E5F
:1088F000F1D1184610BD40EA0103024630B59B078E
:1089000010D14FF0013400E008C208C91D1B9D437F
:1089100015EAC41FF8D013F0FF0102F8011B0DD0B7
:108920001B0AF8E711F8013B002B02F8013B05D0C8
:1089300011F8013B002B02F8013BF3D130BD10B51B
:10894000431C02E010F8011B71B18107FAD14FF00E
:10895000013202C88C1A8C4314EAC211F9D0C01A31
:108960000A0603D0C01E10BDC01A10BD0A0401D0F3
:10897000801E10BD0902FCD0401E10BD40EA01035C
:1089800070B59B072ED14FF00136042A2AD308C8B0
:1089900010C99D1B9D43121F15EAC61517D0D8B2EA
:1089A000E1B2401A50EA056110D198B2A1B2401A62
:1089B00050EA05410AD123F07F4024F07F41401A5C
:1089C00050EA052102D1180EA0EB146070BDA3423D
:1089D000DBD018BA21BA884201D9012070BD4FF00E
:1089E000FF3070BD0AB9002070BD10F8013B11F8CE
:1089F000014B63B1A3420AD1521E08D010F8013BCB
:108A000011F8014B1BB1A34201D1521EEDD1181B2D
:108A100070BD032A40F2308010F0030C00F0158086
:108A200011F8013BBCF1020F624498BF11F801CB71
:108A300000F8013B38BF11F8013BA2F1040298BFD6
:108A400000F801CB38BF00F8013B11F0030300F040
:108A50006780083AC0F0088051F8043B083A51F8A2
:108A600004CBA0E80810F5E7121D5CBF51F8043BE9
:108A700040F8043BAFF30080D20724BF11F8013B5C
:108A800011F801CB48BF11F8012B24BF00F8013BBE
:108A900000F801CB48BF00F8012B7047431A28BFEC
:108AA0009A427FF6B6AF032A1044114440F2268062
:108AB00010F0030F1EBF11F8013D521E00F8013DDA
:108AC00010F0030F7FF4F6AF11F0030300F0698597
:108AD000083AC0F00B8051F8043D083A51F804CD33
:108AE00040F8043D40F804CDFFF7F3BF121D5CBF12
:108AF00051F8043D40F8043DAFF30080D20724BF95
:108B000011F8013D11F801CD48BF11F8012C24BF27
:108B100000F8013D00F801CD48BF00F8012C704776
:108B200010B5203AC0F00B80B1E81850203AA0E808
:108B30001850B1E81850A0E81850BFF4F5AF5FEA3C
:108B4000027C24BFB1E81850A0E8185044BF18C9EF
:108B500018C0BDE810405FEA827C24BF51F8043B96
:108B600040F8043B08BF7047D20728BF31F8023BEA
:108B700048BF11F8012B28BF20F8023B48BF00F87E
:108B8000012B704702F0FF0343EA032242EA02424C
:108B900000F002B84FF000020429C0F0128010F07B
:108BA000030C00F01B80CCF1040CBCF1020F18BFC9
:108BB00000F8012BA8BF20F8022BA1EB0C0100F05C
:108BC0000DB85FEAC17C24BF00F8012B00F8012B2F
:108BD00048BF00F8012B70474FF0000200B5134664
:108BE00094469646203922BFA0E80C50A0E80C50CD
:108BF000B1F12001BFF4F7AF090728BFA0E80C507E
:108C000048BF0CC05DF804EB890028BF40F8042B76
:108C100008BF704748BF20F8022B11F0804F18BFE3
:108C200000F8012B704710B5044610F0030F08BF81
:108C300011F0030F40F015804FF0013E121FC0F2FB
:108C40000E8051F8043BA3EB0E0C2CEA030C1CEA3B
:108C5000CE1C08BF40F8043BF0D0A1F1040102F1A2
:108C60000402521E08DB11F8013B002B00F8013B07
:108C7000F7D11146FFF78EFF204610BD4FF0013CA3
:108C800050F8042B51F8043B9A4221D1A2EB0C037B
:108C9000934313EACC1317D150F8042B51F8043B3B
:108CA0009A4215D1A2EB0C03934313EACC130BD1D8
:108CB00050F8042B51F8043B9A4209D1A2EB0C0363
:108CC000934313EACC13DBD04FF00000704700BF92
:108CD000D01A01BAB1FA81F101F0180122FA01F0BB
:108CE000CB40C1F12001DBB2C0B2C01A2CFA01F3B3
:108CF000D11A914311EAC311E6D17047704770470A
:108D00007047000010B500F07BFC001D10BD00BFD7
:108D1000390E010000487047E889002010B5FFF7C0
:108D2000F9FF006810BD10B50446FFF7F3FF0460BB
:108D300010BD09684A0501D540B27047C905FCD588
:108D400000B2704709684A0501D5C0B27047C9052D
:108D5000FCD580B270472DE9F0470D469946924602
:108D6000044600F124080168880604D5E06921F072
:108D70001001216000E00120A84201DD471B00E056
:108D80000027A1697A1902EB0900081AA06120786E
:108D9000C00602D42046FFF7BFFB002608E0D4E956
:108DA00001211AF806009047206A401C761C2062B8
:108DB0004E45F4DB2078C0060AD52046FFF7ACFB11
:108DC00006E0D4E9012130209047206A401C20624F
:108DD000381EA7F10107F4DC07E0D4E9012118F8F7
:108DE00005009047206A401C2062281EA5F101055D
:108DF000F3DC2046FFF7A6FB2078000602D5022010
:108E0000BDE8F0870120FBE711680268006A53059E
:108E100001D508700AE0D30501D5088006E01306E5
:108E200003D5C217C1E9000200E0086001207047C5
:108E300070472DE9FF4F0C461E464FF0FF378BB0B1
:108E4000D2E90001DDF860800A908A46C1F30A5534
:108E500005B93D46002108464FF00000BAF1000F69
:108E600000F4400005DA00EB80004FF4400101EA15
:108E700050004FEA9059B9F1010F00DDB9460A9848
:108E800050EA4A000ED044F61050A5F2FF35454393
:108E90002F14B8F1000F1ED07542291E1EDDC9F136
:108EA00000021CE0B8F1010F4FF0000001D03021AA
:108EB00003E0F24305E02154401CB042FBDB3046A6
:108EC0000022002121540B99C1F80880C1E900203B
:108ED0000FB0BDE8F08FBD1B6D1CDEE74A4600DA1F
:108EE000694206A800F022FE06AB93E8070003AB38
:108EF00083E8070050460A9901F072FB8DE80700ED
:108F0000A0F500501F3800900398002D09DD42F2B3
:108F10001F014A46084403A90390684601F0FBFD7F
:108F200008E0A0F500504A461F3803A903906846A0
:108F300001F019FE8DE807000004000C03D04FF08B
:108F4000FF30410800E01046B8F1000F03D00022C6
:108F5000009215461EE0751E05D400F055FB303218
:108F600062556D1EF9D5B3460122084302D0002296
:108F70007F1C04E02078302801D100227F1E002AC7
:108F8000099786D01DE0112D07DA00F03DFB303245
:108F900062556D1C50EA0102F5D1084302D00098D9
:108FA000C8B10EE00021681E05E0235C625C6354DA
:108FB0002254401E491C8142F7DBAB46A81B401ED1
:108FC0000990002004F80B000B98099AC0F808805B
:108FD000C0E9002B7CE711264FF0000859E72DE986
:108FE000F04F88460446D21D22F0070191B0D1E926
:108FF0000001CDE90A0105F0A9FD02460B98C00F5A
:1090000001D02D2007E02068810701D52B2002E048
:10901000202101EAC000032A099001D0072A05DBBC
:1090200003464146204600F0BBFC0BE12078800659
:1090300001D5E06900E00620B8F1650F814606D051
:10904000B8F1660F18D0B8F1670F70D131E0002089
:10905000B9F1110F009001DB112301E009F10103C7
:109060000AAA01A90CA8FFF7E4FEDDE90C700026AE
:1090700009F10105834647E001204B4600904FF07F
:1090800000470AAA01A90CA8FFF7D3FEDDE90DB03D
:109090000C995D46002610B909F101000D18B9EBD5
:1090A000050003D4C0F1FF3609F10105A5EB090065
:1090B0002BE0B9F1010F01DA4FF001090020B9F1FD
:1090C000110F0090484601DD112300E003460AAA73
:1090D00001A90CA8FFF7ADFEDDE90C704D46002696
:1090E0008346207800070AD4AB4500DA5D4601A824
:1090F000012D04DD411911F8011C302907D04F451D
:1091000002DA17F1040F04DA012082460FE06D1E27
:10911000EEE7002F02DCED1B3E4403E0781CA84282
:1091200000DD7D1CB81B00F1010A4FF000472078DC
:10913000000703D4AA4501DB4FF0FF3A0021B7F145
:10914000004F0DF143088DF8431024D002202B234B
:10915000002F01DA7F422D230A21021EA0F1010017
:1091600000DC5FB197FBF1FC97FBF1F201FB1C7C8B
:1091700017460CF1300C08F801CDEEE7A8F101001C
:1091800003702188090501D5452100E06521A0F182
:10919000010800F8011C09980FA9A1EB0807FF1DA1
:1091A00000B10120411901EBEA70A1693844081AA5
:1091B000401EA0612078C00602D42046FFF7ACF91B
:1091C000099828B1D4E901219047206A401C206207
:1091D0002078C00622D52046FFF79EF91EE0002E1B
:1091E00004DBB34502DD01A8805D00E03020D4E956
:1091F00001219047206A401C2062761CAAF10100E0
:109200005FEA000A0AD100F0FBF9C0680168405C1F
:10921000D4E901219047206A401C2062281EA5F154
:109220000105DCDC07E0D4E9012118F8010B9047C7
:10923000206A401C2062381EA7F10107F3DC20469B
:10924000FFF780F9032011B043E6000001694A1CD2
:1092500002610878704700B58FB0CDE90131002177
:10926000059105497944CDE9031011466846FFF799
:1092700029FA0FB000BD0000E5FFFFFF0A6802F801
:10928000010B0A607047D1E900239A4202D2531CB5
:109290000B601070704710B5436913B1AFF30080D5
:1092A00001E0FFF760F9012010BD127800F1240100
:1092B0000A7000224A700122EDE711684FF0FF3278
:1092C000E9E700002DE9FF5F15468A460446DFF80E
:1092D000AC80F8440027D8E900103E46CDE90010E4
:1092E00010E03AF816106A4602A800F08DFC411C06
:1092F00007D02178890603D5E269391891420DD843
:109300000744761C2078800602D5E069B84205DD66
:10931000AE42E6DB3AF816000028E2D1A069C01B95
:10932000A0612046FFF7F8F8D8E90010CDE9001059
:10933000002017E03AF818106A4602A800F064FC12
:10934000B0F1FF3F81460BD000250DF1080B05E081
:10935000D4E901211BF8050090476D1C4D45F7D35A
:1093600008F10100B0428046E4DB206A3844206204
:109370002046FFF7E7F8BDE8FF9F0000DE1D010073
:109380002DE9F0418046D21D22F007020025D2E9E6
:109390000002F52915A614D0011E72F1000106DAAB
:1093A0000023D0EB030063EB020211A608E0D8F81B
:1093B00000108B0701D50FA602E0490701D50EA6C4
:1093C00001251146002408F1240704E000F01CF9EF
:1093D00030323A55641C50EA0102F7D12B4632462E
:1093E00021464046BDE8F041FFF7B5BC0000000053
:1093F0002D0000002B0000002000000030B40021F0
:1094000000F1240408E002F00705D208303542EAF2
:109410004372DB086554491C52EA0305F3D1046822
:10942000002310A2250708D504F020040C4304D023
:10943000C46901230CA2641EC46130BCFFF78BBC5D
:1094400010B5044621461068FFF77CFC0246204612
:10945000BDE810400023D1E7D21D22F00701D1E979
:109460000023CBE700000000300000000FB4002311
:1094700000B589B00CA900910B99CB60204B7B44BF
:109480000693204B7B44079304236FF00042CDE901
:1094900001321D4A7A446B4608920246002011F0C0
:1094A0007BFD09B05DF814FB70B506464FF0FF3048
:1094B00015460C46324686B00091CDE90101694659
:1094C0000020049004A8FFF7D1FF03460498211858
:1094D00025B108B10A4600E022462A6000280DD0D6
:1094E000002B02DD0098884208D03246081B6946EE
:1094F0000094CDE9010404A8FFF7B8FF06B070BDE1
:10950000CB050000E3050000FB0100002DE9F0475A
:1095100091460F4680460446002614F8015B2DB1A3
:10952000FFF7F0FB0068405DC007F6D12B2D02D09D
:109530002D2D18D0641E4A463946204600F0A6FA62
:1095400027B13968A14201D1C7F800804FF0020469
:1095500071050BD54042002803DDFFF7DBFB0460FB
:10956000A007BDE8F08746F48066E4E70028F8DA53
:10957000FFF7D0FB04606FF00040F2E7431A28BF0A
:109580009A427FF6CDAA104410F0030F11441EBF7B
:1095900011F8013D521E00F8013D10F0030F7FF459
:1095A000F6AF103AC0F00A8010B531E91850103A01
:1095B00020E91850BFF4F9AFBDE81040530724BFAD
:1095C00031E9081020E9081044BF51F8043D40F883
:1095D000043D12F0030F08BF7047D20728BF31F8CF
:1095E000023D48BF11F8012C28BF20F8023D48BFBA
:1095F00000F8012C7047000000487047E8890020FF
:1096000000487047088A002030B5B0F10A024FEADE
:10961000900E71F100034EEA817EB0EB0E0061EB1B
:1096200091014FEA101E4EEA017E10EB0E0041EB55
:1096300011114FEA102E4EEA016E10EB0E0041EBB5
:1096400011214FEA104E4EEA014E10EB0E0041EB95
:109650001141401841F100014FEAD00040EA417049
:109660004FEAD10110EB80054FEA810444EA90747F
:1096700044EB01046D1944EB0404521BA3414FF069
:10968000000348BF0A3200D530BD401C41F1000143
:1096900030BD10B50446FFF735FB0068005D00F0F3
:1096A000010010BD2DE9F04F04460D46D21D22F0F9
:1096B000070089B0D0E9009248461746394605F0C0
:1096C00045FA0246F80F01D02D2307E020688107F4
:1096D00001D52B2302E0202101EAC0038DF82030C0
:1096E0000BB1012000E00020032A824601D0072AA6
:1096F00004DB2946204600F053F93DE1207880063E
:1097000001D40D2500E0E569C7F30A560D2D49DAAD
:1097100000214FEA175B08464FF00000002F00F4CD
:10972000400007DA00EB80004FF4400100EBD070FE
:1097300001EA60008115012901DD4FF0FF310022AF
:109740004FEA850CBCF1180F06D31346ACF1180094
:109750004FF08052C24003E04FF4801323FA0CF321
:109760000CF10C0CBCF1200F04D3ACF1200C09FA65
:109770000CF001E007FA0CF000294FF0004801DD81
:1097800018B90FE00ED140450CD319EB02095F4127
:1097900021B9404502D19F4329EA0209BBEB175F7B
:1097A00000D0761C2088000502D57B48784402E072
:1097B00079487844193808AA302302F80A30037C23
:1097C0000AF10101002E0AF1020A53546A4602DC32
:1097D0004FF0300101E04FF031014FF001088DF8FA
:1097E000001002D0A6F2FF3603E059EA470100D08C
:1097F0006A4E002D02DC2178090704D54FF00208DB
:109800002E218DF80110C44600210BE0C7F303435D
:109810003F01C35C491C6D1E02F80830052908F1A0
:10982000010801DA002DF1DC00210CE000EB1973D6
:10983000491C1B786D1E082902F808304FEA0919E7
:1098400008F1010801DA002DF0DC2178890602D543
:1098500014E0A8F10108E04505DD02EB080111F86C
:10986000011C3029F5D0B8F1000F07DD02EB08012B
:1098700011F8011C2E2901D1A8F10108002D05DDE8
:109880003E2102F808106D1E08F10108407C002EF0
:1098900002F8080008F1010804DA2D20764202F8E7
:1098A000080002E02B2002F808000A214FF47A7029
:1098B000864208F101080BDB96FBF0F3303302F827
:1098C000083096FBF0F308F1010800FB136601E095
:1098D000642E0CDB642096FBF0F3303302F8083082
:1098E00096FBF0F308F1010800FB136601E00A2E75
:1098F00006DB96FBF1F0303002F8080008F10108B1
:1099000096FBF1F001FB1060303002F80800A1690D
:1099100008F1010808EB050202EB0A00081AA06131
:109920002078C00602D42046FEF7F6FD216A08AE74
:1099300001EB0A00206204E0D4E9012116F8010BD2
:109940009047BAF1010AF7D22078C00602D5204626
:10995000FEF7E2FD6E4609E016F8010B3E280FD037
:10996000D4E901219047206A401C2062B8F1010827
:10997000F2D22046FEF7E6FD09B00320BDE8F08FE5
:10998000206A2844206203E0D4E901213020904776
:109990006D1EEBD3F8E70000431A010002FCFFFF45
:1099A0002DE9F0411F46044603260168072A01F409
:1099B000006004DB08B116A505E016A503E008B1B8
:1099C00015A500E015A521F010002060A069C01EBB
:1099D000A0610FB1401EA0612046FEF79DFD4FB172
:1099E000D4E9012138469047206A401C2062C01CFF
:1099F000206206E0206AFAE7D4E9012115F8010B9C
:109A00009047761EF8D22046FEF79CFDBDE8F08117
:109A10004E414E006E616E00494E4600696E660012
:109A200010B5436913B1AFF3008001E0FFF74AFCC2
:109A3000012010BD128800F1240182840022C2841A
:109A40000122EDE711684FF0FF32E9E7426842B1C9
:109A5000016811F8013B23B1521EC0E900121846FB
:109A600070470121C160881E704742685AB1C368BF
:109A7000016843B983688B4205D0491E521CC0E976
:109A80000012002070474FF0FF3070472DE9F05F63
:109A9000824615468B4600270AF10104B946007834
:109AA000302801D09DB113E014F8010B012778286C
:109AB00003D0582801D045B10AE00DB1102D07D1CF
:109AC000002714F8010B102502E0082500E00A2504
:109AD0000026B0460EE005FB080005FB06F1012755
:109AE0001FFA80F801EB1046B6F5803F00D3B94667
:109AF00014F8010B294600F0CCF80028EBDABBF192
:109B0000000F05D00FB1641E00E05446CBF80040B2
:109B1000B9F1000F06D0FFF7FDF802210160C81E61
:109B2000BDE8F09F48EA0640FAE700002DE9F0475B
:109B3000814616468AB0334878440DC88DE80D003A
:109B400030487844801C03AC0DC884E80D0041F611
:109B50009B300844372190FBF1F290FBF1F5A5F121
:109B6000800501FB12041B3C02D56442012000E089
:109B70000020DFF890A080460027FA44AAF1BE0A30
:109B80000DE0E00709D03246684607EB47010AEBD3
:109B9000810100F0E8FF8DE8070064107F1C002CB5
:109BA000EFD1184F7F44AC3F18E0E80714D007EB23
:109BB00004100DF1180A90E80E008AE80E00C06843
:109BC000F04201D198190890324606A903A800F086
:109BD000CAFF03AB83E807006D10641C002DE4D1BD
:109BE00032466946B8F1000F03A802D000F093FF97
:109BF00001E000F0B8FFC9E90001C9F808200AB087
:109C0000BDE8F0874817010070B516460C460546BA
:109C1000FFF778F8036893F80101012806D0FF2CBC
:109C20000FD8185D68B101202C7070BDD3F8070102
:109C30003246214603F2071303442846BDE870402C
:109C400018474FF0FF3070BD7546FFF7D5FCAE46A4
:109C500005006946534620F00700854618B020B538
:109C6000FEF784FBBDE820404FF000064FF00007F0
:109C70004FF000084FF0000B21F00701AC46ACE8B4
:109C8000C009ACE8C009ACE8C009ACE8C0098D4621
:109C900070473A2800D2303820F02002412A01D300
:109CA000A2F13700884201D34FF0FF307047000027
:109CB0002DE9FF4F064689B00878FF2806D0491CD9
:109CC0002D2805D000244FF0000908E000200CE00A
:109CD0000124F8E709EB8903491C00EB43090878E4
:109CE000FF28F7D114B1C9F1000081461078002592
:109CF0002C46AA4629462D2801D02B2804D1521CD7
:109D00002D2813D0002082468B461078FF280FD0D4
:109D10004FF0000C0A21521CA5FB017804FB0181C5
:109D200005FB0C11C5194BEB0104EEE70120EAE736
:109D3000002108464FF00000BAF1000F02D000EBFE
:109D400080004008C0F38158B8F1010F01DD4FF0E9
:109D5000FF380C9809EB000755EA040009D04FF0D2
:109D6000020917F5FA7F0BDA4FEACA70C6E900B0AC
:109D700012E04FEACA70C6E900B00DB0BDE8F08F3E
:109D8000B7F5FA7F0DDDF0487844D0E90010C6E958
:109D9000001040EACA707060FEF7BCFFC0F8009087
:109DA000EBE7391E02DAC8F1000200E0424600DAB1
:109DB000794206A8FFF7BAFE06AB93E8070003ABAB
:109DC00083E8070044F23E005BEA04010090584635
:109DD00004D144F21E012C465D460091210C090479
:109DE000014306D10099240444EA15442D04103996
:109DF000009104F07F41014306D10099240244EA16
:109E000015642D020839009104F07041014306D118
:109E10000099240144EA15742D01091F009104F0F2
:109E20004041014306D10099A40044EA9574AD0075
:109E3000891E009104F00041084304D100986D1977
:109E40006441401E009042466846002FCDE901451E
:109E500003A902DD00F09BFE01E000F070FEBAF104
:109E6000000F04460D4601D084F0004440F2FF7715
:109E700024F00040284303D0C4F30A50B84212D162
:109E8000FEF748FFC0F80090C4F30A50B8420AD168
:109E9000AE487844D0E90010C6E9001004F0004153
:109EA0000843706069E7C6E9005466E72DE9FF4F93
:109EB0001F464FF0000A4FF0FF38454691B0D7E9F2
:109EC0000146CDF83CA0FFF79BFBC0680168405CF1
:109ED0001090B96912986D1C8847396A8146884785
:109EE0000028F6D1B9F1FF3F0AD0002E24F4D06447
:109EF00011DDB9F12B0F08D0B9F12D0F0BD102E014
:109F0000404615B03AE744F48064B96912986D1C74
:109F10008847761E8146600504A901D52D2000E002
:109F20002B20002E01F1010B0DF130088DF81000EF
:109F30003FDDB9F1690F08D0B9F1490F05D0B9F18A
:109F40006E0F02D0B9F14E0F1CD13B4601A800950F
:109F500080E85002DDE912126FF0020011F020F8E3
:109F6000C11CCED10EE0B96912986D1C884781469C
:109F70001398761E44F4007405600F98401C002E60
:109F80000F9016DDB9F1300FEDD0B9F1780F02D096
:109F9000B9F1580F0DD10F9801280AD13B46CDE9F0
:109FA0000054DDE91212001F029610F0F7FFC11CE9
:109FB000A7D1109989453ED144F0800406E0139959
:109FC000681CAAF1010A44F400740860B9696D1CA8
:109FD0001298761E884730288146F0D02BE01099E1
:109FE000894505D1200603D4761E44F0800418E08C
:109FF000484605F082F908B3761E0DF123018B4522
:10A0000044F4007408D2A9F130000BF8010B2006CB
:10A0100007D5AAF1010003E0200602D40AF10100ED
:10A020008246A00502D51399681C0860B969129888
:10A030006D1C88478146002ED1DC53E0002E51DD97
:10A04000B9F1650F02D0B9F1450F4BD1A00549D543
:10A05000B9696D1C1298761E24F440748847002E4E
:10A0600081460CDD2B2804D0B9F12D0F07D144F423
:10A070008074B96912986D1C8847761E8146E00588
:10A0800001D52D2100E02B2108F8011BCDF800801F
:10A0900021E0761E0DF13901884544F400740CD29C
:10A0A000A9F1300010F0FF0088F8000002D10099FB
:10A0B000884509D908F1010806E0E00501D52448E2
:10A0C00001E042F20F708246B96912986D1C884710
:10A0D000814613980560002E04DD484605F00DF911
:10A0E0000028D6D1F96912988847FF2053468BF88B
:10A0F000000088F8000000200A900B9004AA0CA928
:10A100000AA8FFF7D5FDA00502D46FF00100F8E61C
:10A1100014F0240F0AD0E00714D13868DDE90A12E0
:10A12000031D3B600068C0E900120BE00AA9684605
:10A1300005F08CF8E00705D13868009A011D3960F8
:10A14000006802602846DCE6981D01008E1C0100B4
:10A15000F1D8FFFF0446AFF300802046FEF7A5F8D4
:10A1600001491820ABBEFEE7260002002DE9FF4F93
:10A170001F464FF03C0987B04FF00042DDE9141054
:10A1800001F10108DDF858A002EA405003900020D8
:10A1900004908346054604460590B969461E089812
:10A1A0008847AAF1010A0290BAF1000F37DD029840
:10A1B0002E2815D01021FFF76CFD00282ADB4FF068
:10A1C000010B0499014316D0B9F1000F0BDB4A468D
:10A1D000C11700F0F2F905430C43A9F1040905E0A9
:10A1E0000120059007E008B145F001050120049029
:10A1F000059800B9361DB969089808F10108884723
:10A20000BBF1000FAAF1010A0290CDD00999C1F863
:10A210000080C9E70298702808D0502806D0F96954
:10A2200008988847BBF1000F14D04FE0002002903F
:10A230000120BBF1000F049009D0B969089808F11A
:10A2400001088847AAF10109B9F1000F07DCF96993
:10A25000089888476FF001000BB0BDE8F08F2B28FD
:10A2600004D02D280CD14FF0FF300490B969089824
:10A2700008F101088847A9F10109B9F1000FE6DDED
:10A28000411CE4D00A21FFF704FD0028DFDB02991E
:10A2900008F1010801EB810100EB41000290B9696E
:10A2A000089888470A21FFF7F4FC099AA9F10109E7
:10A2B000B9F1000FC2F8008001DD0028E7DAF96982
:10A2C000089888470499029800FB016655EA040043
:10A2D00004D004F04041090002D006E0039898E061
:10A2E000A40044EA9574AD00B61E04F000410800D5
:10A2F00002D16D196441761E159810F0240F03D019
:10A300004FF00B095C4803E04FF028096FF07D0027
:10A310008246564507DAAAEB06018944B9F1410F96
:10A3200001DD4FF0410901200021A9F1010200F0F7
:10A3300044F9024628400B462140084301D0012140
:10A3400000E00021501E029143F1FF3128402140DE
:10A35000084301D0012000E000200299834651EA21
:10A360000B014FD0002108464FF00000039900F484
:10A37000400039B100EB80004FF4400100EBD07099
:10A3800001EA60008015012802DD4FF0FF3000E097
:10A3900013D0401C36D0029860B3BBF1000F0CD133
:10A3A0004A460120002100F008F9284021400843D6
:10A3B00001D0012000E00020E0B101204A46002148
:10A3C00000F0FBF8034640190A4661412D1A8C4102
:10A3D00011D3B9F1400F09DD159810F0240F02D008
:10A3E000AAF1340603E0AAF1170600E0761C002566
:10A3F0004FF0004406E05B1E42F1FF3220EA030505
:10A4000021EA0204CAF10100B04206DA1B490398AE
:10A4100008430190002000900EE0039AC4F3D3217A
:10A42000E80A0A43164940EA44500A433146CDE956
:10A430000002684604F056FF159810F0240F0BD068
:10A440001598C00715D13868DDE90012031D3B607F
:10A450000068C0E900120CE002A8694604F0F6FEAC
:10A460001598C00705D13868029A011D3960006847
:10A4700002604046F0E6000002FCFFFF0000F07FB3
:10A480000000F03F2DE9FF4F92461D4685B04FF08A
:10A490000041DDE9124BDDE914727F1E01EA4B50E9
:10A4A000414940F0FF4940EA0108002122F0200024
:10A4B0004928049102D04E2828D04CE03BA0012628
:10A4C00007C88DE80700A9690698641C88477F1EA5
:10A4D000014606D41DF8060018B121F02001814282
:10A4E0000BD0E96906988847032E34D0082E32D065
:10A4F0006FF0010009B0BDE8F08F761C032E01D08B
:10A50000082EE0D1601CCAF80000DCE7A9690698B3
:10A51000641C88477F1E2AD420F02000412826D1C1
:10A52000A9690698641C88477F1E20D420F020006B
:10A530004E281CD1A9690698641C88477F1E48F4E0
:10A54000002849F48009CAF8004001D4282806D020
:10A55000E969069888475FEACB7012D022E0A969C2
:10A560000698641C88477F1E01D4002803DAE96935
:10A5700006988847BCE72928F1D1641CCAF8004036
:10A58000E9E71BF0240F07D028680499031D2B600E
:10A590000068C0E9001805E02868021D2A6000680C
:10A5A000C0F800902046A5E70000F07F494E4649DC
:10A5B0004E495459000000007047B2F120030AD5FB
:10A5C000C2F1200301FA02F120FA03F300FA02F0CB
:10A5D00041EA0301704700FA03F14FF000007047B1
:10A5E0005FEA400C08BF91F0000F4FEA8C234FEA5E
:10A5F000C12243EA51514FEA1C5018BF00F5F04008
:10A600004FEA300018BF41F000415FEA6C5C00F097
:10A610002980BCF1FF3F08BF40F080407047130C19
:10A6200006BF12044FF0100C4FF0000C130E04BFC5
:10A6300012020CF1080C130F04BF12010CF1040CF0
:10A64000930F04BF92000CF1020CD30F04BF520011
:10A650000CF1010C11464FF00002A0F11F00A0EB1D
:10A660000C00704711F0004F08BF704731F00041F7
:10A670003FF4D5AF0B0C06BF09044FF0100C4FF0A0
:10A68000000C0B0E04BF09020CF1080C0B0F04BFE9
:10A6900009010CF1040C8B0F04BF89000CF1020CB2
:10A6A000CB0F04BF49000CF1010CCCF12003A0EB4F
:10A6B0000C0022FA03F302FA0CF241EA030100F162
:10A6C0000100704720F07F4C80EA030023F07F47B1
:10A6D000ACEB070303F57C5300F0004003F1FF03EC
:10A6E0002DE980494FEA154B09B44FEA144325EA96
:10A6F0000B4E24EA03480FF2042606EB1327490801
:10A700003E785FEA320203FB0667C7F5000707FBE6
:10A7100006F64FEA54374FEAD64606F1020607FB23
:10A72000066CCCF1005C4FEA1C472CEA074C07FB97
:10A7300006F40CFB06F504EB15464FEA961634BFFB
:10A7400000204FF000404FEAD13706FB07FC4FEAEC
:10A750001C4C0CFB0BF7D21B03FB0CF761EB070146
:10A760000CFB0EF7B0EB074072EB17420CFB08F73F
:10A7700034BFA2EB0742B2EB074261EB17414FEA4D
:10A780000C444FEA910706FB07FC4FEA1C4C0CFBFC
:10A790000BF7B0EBC74072EB573203FB0CF734BF3B
:10A7A000A2EBC742B2EBC74261EB57310CFB0EF78D
:10A7B000B0EBC70072EB57720CFB08F734BFA2EB8B
:10A7C000C702B2EBC70261EB5771039F4FEA816189
:10A7D00041EA921104EBCC044FEAD1374FEA82628E
:10A7E00006FB07FC42EA90124FEA80604FEA1C4CDD
:10A7F0000CFB0BF7D21B03FB0CF761EB07010CFB07
:10A800000EF7B0EB074072EB17420CFB08F734BFB2
:10A81000A2EB0742B2EB074261EB17414FEA8C55BE
:10A820004FEA910704EB9C2406FB07FC4FEA1C4C03
:10A830000CFB0BF7B0EBC74072EB573203FB0CF786
:10A8400034BFA2EBC742B2EBC74261EB57310CFBFE
:10A850000EF7B0EBC70072EB57720CFB08F734BF72
:10A86000A2EBC702B2EBC70261EB577115EB4C25A7
:10A870004FEA816141EA92114FEA82624FEAD13791
:10A8800042EA901206FB07FC44F100044FEA8060A4
:10A890004FEA1C4C0CFB0BF7D21B03FB0CF761EBD4
:10A8A00007010CFB0EF7B0EB074072EB17420CFBF5
:10A8B00008F734BFA2EB0742B2EB074261EB174146
:10A8C00015EB1C154FEA813141EA92414FEA823281
:10A8D00042EA90424FEA80304FEA0C7644F100049D
:10A8E00048EA03434EEA0B484FF0000EB2EB080C67
:10A8F00071EB030724BF624639464EEB0E0E4FF054
:10A90000000B0018524149414BEB0B0BB2EB080C0A
:10A9100071EB03077BF1000B24BF624639464EEB17
:10A920000E0E4FF0000B0018524149414BEB0B0B40
:10A93000B2EB080C71EB03077BF1000B24BF6246FE
:10A9400039464EEB0E0E51EA020718BF46F00106DB
:10A9500016EB0E7655F1000254F1000103D5BDE867
:10A960008901BDE80088BDE88901BDE80048B61945
:10A97000524141EB0101A3F10103704780807F7ECA
:10A980007D7C7B7A79787776767574737271717065
:10A990006F6E6E6D6C6C6B6A6A6968686766666517
:10A9A0006464636362616160605F5F5E5E5D5D5CA5
:10A9B0005C5B5B5A5A595958585757565655555516
:10A9C0005454535352525251515050504F4F4F4E76
:10A9D0004E4D4D4D4C4C4C4B4B4B4A4A4A494949C4
:10A9E0004848484747474746464645454544444406
:10A9F00044434343434242424241414146EA0646C0
:10AA0000A3F570534FEA164646EA42564FEAD22261
:10AA100042EA415210B54FEAD121A3F1010300F0FF
:10AA200017F820F0004000F1010C00F0004701EBA6
:10AA300000501146BCF5006F40EA070000D210BD7F
:10AA400002484FF0000140EA070010BD0000F07F0F
:10AA5000002B26D4770021D01CB54FEA370703B46A
:10AA60004FF010004FF010014FF000000FBCBDE898
:10AA700010400BF1010BBBF1010F08BF5FEA170794
:10AA800022BF12F1010211F101014FF0004143F127
:10AA9000000300F0004043EA00007047F9D3570874
:10AAA000DAE746EA064613F1400F4FEA16461FDD85
:10AAB00013F1200FDFBF16430A46002120335B420B
:10AAC000C8D0C3F1200746EA064602FA07F74FEA64
:10AAD000164646EA0706C3F1200722FA03F201FAF6
:10AAE00007F721FA03F14FF0000342EA0702B1E74A
:10AAF00046EA020646EA06464FEA164646EA0106D6
:10AB0000BCBF46EA0646360C4FF000034FF0000289
:10AB10004FF000019EE72DE9C048934630B491E81C
:10AB2000380007C831EA400C48BF34EA430C03D56B
:10AB3000FFF7C8FDFFF78CFFF0BCBDE800882DE9EA
:10AB4000C048934630B491E8380007C831EA400C59
:10AB500048BF34EA430C03D5FFF7B4FDFFF74EFFBF
:10AB6000F0BCBDE800882DE9C048934630B491E8B8
:10AB7000380007C810F0804F08BF13F0804F03D192
:10AB800000F019F8FFF764FFF0BCBDE800882DE97C
:10AB9000C048934630B491E8380007C810F0804FA1
:10ABA00008BF13F0804F03D100F005F8FFF726FF30
:10ABB000F0BCBDE8008820F07F4780EA030023F066
:10ABC0007F4C07EB0C03A3F57C5300F00040A3F18E
:10ABD000FE0392F0000F00F0B38095F0000F00F03C
:10ABE00077802DE901494FEA11404FEA144621EAE6
:10ABF000004800FB06FC24EA064708FB06F607FBB4
:10AC000008F800FB07F718EB06484CEB164C4FEA28
:10AC1000124B18EB07484FEA15464CEB174022EA57
:10AC20000B4E0BFB06FC25EA06470EFB06F607FB60
:10AC30000EFE0BFB07F71EEB064E4CEB164C4FF0CF
:10AC400000061EEB074E4CEB174B18EB0B0840F1C0
:10AC5000000018EB0E0B58EB000840F100008F1AB3
:10AC60004FF000013CBFC943661B14BFB5EB040C99
:10AC700000213CBFC943F61B4FEA17444EEA8E0E33
:10AC800027EA04454FEA1C4704FB07622CEA074CFD
:10AC900005FB07F70CFB05F604FB0CFC16EB07465F
:10ACA00042EB174216EB0C4642EB1C421BEB06062E
:10ACB00058EB0202414146EA9E0601D5BDE80189F2
:10ACC000B619524141EB0101A3F10103BDE801892D
:10ACD0004FEA14454FEA114724EA054621EA074C9A
:10ACE00005FB07F406FB07F70CFB06F105FB0CFC64
:10ACF00011EB074144EB17444FEA124711EB0C41AB
:10AD000044EB1C4422EA074C05FB07F206FB07F75D
:10AD10000CFB06F605FB0CFC16EB074642EB174254
:10AD200016EB0C4642EB1C456A1854F1000148BF73
:10AD30007047B619524141EB0101A3F1010370477D
:10AD400095F0000F37D04FEA11424FEA144721EA3D
:10AD5000024624EA074C02FB07F106FB07F70CFB4F
:10AD600006F402FB0CFC14EB074441EB17414FEADD
:10AD7000154714EB0C4441EB1C4125EA074C02FB40
:10AD800007F506FB07F70CFB06F602FB0CFC16EBBF
:10AD9000074645EB174516EB0C4645EB1C421219CE
:10ADA00051F1000148BF7047B619524141EB010112
:10ADB000A3F1010370474FEA14454FEA114724EA13
:10ADC000054621EA074C05FB07F106FB07F70CFBDC
:10ADD00006F24FF0000605FB0CFC12EB074241EBBC
:10ADE000174112EB0C4251EB1C4148BF70479218BF
:10ADF00041EB0101A3F101037047000070B5044667
:10AE000000688168C943C9071CD1816821F001012C
:10AE1000816000F0FDFE05460FE000BF00F0F8FE87
:10AE2000401B022809D9A06A40F01000A062E06A25
:10AE300040F00100E062012070BD20688068C043DE
:10AE4000C007EBD0002070BDF8B500260446009680
:10AE500000688168C943C90728D0816841F00101B1
:10AE60008160134813490068B0FBF1F000E0401E18
:10AE700000900028FBD100F0CBFE054611E000BF9A
:10AE800000F0C6FE401B02280BD9A06A40F010005B
:10AE9000A062E06A40F00100E06284F824600120D2
:10AEA000F8BD20688068C043C007E9D10020F8BD24
:10AEB0006800002040420F0010B500F0E7FE02F0ED
:10AEC00087FE02F02BF802F003F802F0EFF802F030
:10AED00009F902F023F902F0ADF8084806490160CB
:10AEE0000621416040F6FF71816000F097FE002866
:10AEF00001D072B6FEE710BD00300040C4890020CA
:10AF0000FEE700000FB4F0B5E1B0214C02E00120F3
:10AF100000F05EFD00F07CFEE168401A1E28F6D3CA
:10AF20004FF4C07667AB31466846669AFDF7A8FADB
:10AF300005466846FDF703FD82B24FF4FA773B46BB
:10AF40006946144801F04DFF3B46022212A1114808
:10AF500001F047FF00F05CFEE060B54203DB2946EC
:10AF60000EA009F0A5FC607800280DD0A07800287C
:10AF70000AD111A16846FDF780FC002804D0012009
:10AF8000A0700FA009F050FC61B0F0BC5DF814FB9C
:10AF90006C0000207C8800200D0A00003E20434108
:10AFA00054313A20B7A2CBCDBDD8B6CF21D0E820BE
:10AFB000256420D7D6BDDA0041542B4D50554200B0
:10AFC0003E2034473A20CAD7B4CEB7A2B2BCB3C9E8
:10AFD000B9A60000014800F061BB00003C890020D8
:10AFE000014800F05BBB00008089002030B590F87C
:10AFF00040500124AC40C56B6C60046863604368DA
:10B00000102B036803D099600068C26030BD9A605D
:10B010000068C16030BD70470FB430B5C1B0154C89
:10B0200002E0012000F0D4FC00F0F2FD2168401A9B
:10B030001E28F6D345AB4FF480716846449AFDF75D
:10B040001FFA6846FDF77BFC82B24FF4FA752B4677
:10B050006946094801F0C5FE2B46022207A10648B1
:10B0600001F0BFFE00F0D4FD206041B030BC5DF8BF
:10B0700014FB0000A0000020BC8800200D0A000086
:10B0800072B6FEE7F8B50024009490F82420254617
:10B09000012A12D0012280F824204A681F23072A9F
:10B0A0000DD20668776B521E02EB820293409F43DB
:10B0B0000B6893401F43776319E00220F8BD0668D0
:10B0C0000D2A0AD2376BD21F02EB820293409F43B4
:10B0D0000B6893401F43376309E0F76A0D3A02EBB0
:10B0E000820293409F430B6893401F43F7620A68B4
:10B0F000072306680A2A0AD3F7680A3A02EB4202D3
:10B1000093409F438B6893401F43F76008E0376983
:10B1100002EB420293409F438B6893401F43376189
:10B120000A68102A01D0112A20D1124B02689A42D3
:10B1300017D193681B0219D4936843F400039360FA
:10B140000968102912D10C490C4A0968B1FBF2F1C7
:10B1500001EB8101490000E0491E00910029FBD16B
:10B1600004E0816A41F020018162012480F82450CA
:10B170002046F8BD002401406800002040420F0036
:10B180000068C06C704700002DE9F04104004FF0EA
:10B19000000514D0A06A002628B9E66284F824606D
:10B1A000204600F083F82046FFF728FEA16A01F050
:10B1B0001001014304D0A06A40F01000A0626BE0CF
:10B1C000A16A21F4885141F00201A1623349236848
:10B1D0008B42E16904D1B1F5402F01D14FF4002138
:10B1E000277B4FF4807C41EA470261680A43A168EB
:10B1F000614509D0012907D05FF0000194F814E0FF
:10B20000BEF1010F02D00AE06146F7E7C7B1A76AB5
:10B2100047F02007A762E76A47F00107E7625F6827
:10B2200027F469470F435F60236899681C4F3940D2
:10B2300011439960A16861450BD0012909D00CE048
:10B24000DFF860E0A7690EEB47370F4347F4006172
:10B25000E5E7218A0D05A5F580152168CB6A23F461
:10B2600070032B43CB62216889680F4B19409142D0
:10B2700008D1E662A16A21F0020141F00101A16258
:10B28000BDE8F081A06A20F0020040F01000A0624A
:10B29000E06A40F00100E0620120F1E7003C01407B
:10B2A000FDF7E1FF00E0FFFFFE0E1FFF00B50068A5
:10B2B000104985B088421BD10F48816941F4007163
:10B2C0008161816901F400710491816941F0040197
:10B2D00081618069694600F00400049000200290BA
:10B2E00003900120009003200190044800F082FBAD
:10B2F00005B000BD002401400010024000080140DC
:10B300002DE9F84300260D460446009600F080FC27
:10B31000804620688168C90508D5A06A40F02000F1
:10B32000A06284F824600120BDE8F8834168C90563
:10B3300003D4C06A10F4700F26D0022000F060FD24
:10B3400038490968B1FBF0F72068036936490B42B8
:10B350004FEA61014FEAA1121BD1C3684FEA611C99
:10B3600013EA0C0F15D103690B4221D1C0681042BA
:10B370001ED114201FE0681C06D045B300F048FC25
:10B38000A0EB0800A84222D8206800688007F2D508
:10B390002AE003690B4202D1C168114206D002695A
:10B3A00022490A4206D1C068084203D1542002E073
:10B3B000292000E0FC204743009813E0681C0ED0D1
:10B3C0002DB100F025FCA0EB0800A84207D9A06A27
:10B3D00040F00400A06284F824600320A4E70098F1
:10B3E000401C0090B842E9D321686FF01200086059
:10B3F000A06A40F40070A06220688068C0F34240F8
:10B4000007280CD1207B50B9A06A20F48070A0627C
:10B41000A06AC00403D4A06A40F00100A06200202A
:10B4200082E7000068000020244992244992240009
:10B4300070B5044690F8240001280DD0012084F84E
:10B4400024002046FFF700FD02004FF0000005D069
:10B4500084F82400104670BD022070BDA16A40F23D
:10B460000123994341F48071A1621F4D23681F4954
:10B47000AB4218D10E6816F4702F14D0A66A46F4A9
:10B480008016A6620E68760505D5A66A26F40056D3
:10B4900046F48056A662A66AF6040AD5E66A26F045
:10B4A0000606E66206E0A66A26F48016A6625E68D4
:10B4B000E9E7E06284F824006FF002001860206879
:10B4C0008368C3F34243072B05D1A84208D109681A
:10B4D00011F4702F04D0816841F480118160B9E7C4
:10B4E000816841F4A001F9E70028014004240140EB
:10B4F00010B5044690F82400012807D0012084F8F4
:10B5000024002046FFF77AFC10B107E0022010BDAE
:10B51000A16A21F4885141F00101A162002184F85F
:10B52000241010BD10B590F821100022022905D07A
:10B530000421816380F82020012010BD01680B6880
:10B5400023F00E030B6001680B6823F001030B600E
:10B5500090F84030C46B012101FA03F3636080F876
:10B56000211080F82020104610BD00002DE9F05F6A
:10B5700090F821100024022903D0042181630124C2
:10B5800085E001680A6822F00E020A6001680A6814
:10B5900022F001020A603F4E3E4FB215DFF8F4C0C0
:10B5A000DFF8F090DFF8ECA0DFF8E8B0DFF8E4E0D7
:10B5B0000168783F13011502ACF1640CA9F1500940
:10B5C000AAF13C0AABF1280BAEF1140E4FF480182F
:10B5D000B14227D9B9420ED0614512D049451DD09C
:10B5E000514518D0594518D0714501D1424615E052
:10B5F000294EB14201D1012210E0274E1436B1424A
:10B6000001D110220AE0244E2836B14206D0224A47
:10B610003C32914201D11A4600E02A461E49091FD8
:10B620000A602BE0B94213D0614517D0494522D0BA
:10B6300051451DD059451DD0714501D142461AE0F2
:10B64000B14202D14FF0807215E0134EB14201D1E8
:10B65000012210E0104E1436B14201D110220AE04E
:10B660000D4E2836B14206D00B4A3C32914201D1F0
:10B670001A4600E02A46074980394A60012180F8CD
:10B680002110002180F82010416B01B1884720462D
:10B69000BDE8F09F80000240080402402DE9F05F01
:10B6A000C16B0A6801680B68046C4FF0040808FA63
:10B6B00004F8844D844E854FDFF814C2DFF81492ED
:10B6C000DFF814A2DFF814B2DFF814E218EA020F70
:10B6D00065D05FEA437862D50A68920603D40A68A7
:10B6E00022F004020A60DFF8F0814FF48062016802
:10B6F00008F1140813011402414524D9A9420DD0C0
:10B70000B1420FD0B9421AD0614515D0494515D084
:10B71000514501D1120312E0594501D104220EE036
:10B72000714501D140220AE06D4D1435A94206D081
:10B730006B4A2832914201D11A4600E022466749FD
:10B74000091F0A6029E0A94213D0B14215D0B942BD
:10B7500020D061451BD049451BD0514502D14FF443
:10B76000800217E0414502D14FF0806212E0594556
:10B7700001D104220EE0714501D140220AE0584D6A
:10B780001435A94206D0564A2832914201D11A46B0
:10B7900000E022464B4908394A60C16A71E04FF027
:10B7A000020808FA04F818EA020F70D05FEA8378FA
:10B7B0006DD50A68920606D40A6822F00A020A6069
:10B7C000012180F82110DFF810814FF40072016828
:10B7D00008F1140813011402414524D9A9420DD0DF
:10B7E000B1420FD0B9421AD0614515D0494515D0A4
:10B7F000514501D1120312E0594501D102220EE058
:10B80000714501D120220AE0354D1435A94206D0F8
:10B81000334A2832914201D11A4600E022462F498C
:10B82000091F0A6029E0A94213D0B14215D0B942DC
:10B8300020D061451BD049451BD0514502D14FF462
:10B84000001217E0414502D14FF0007212E0594555
:10B8500001D102220EE0714501D120220AE0204DE3
:10B860001435A94206D01E4A2832914201D11A4607
:10B8700000E02246134908394A60002180F8201070
:10B88000816A00291CD0BDE8F05F0847FFE7082562
:10B89000A540154214D01A0712D50A6822F00E02EC
:10B8A0000A6090F84020C36B012101FA02F25A604D
:10B8B000816380F82110002180F82010016BE0E7FF
:10B8C000BDE8F09F080002401C000240300002402A
:10B8D00044000240580002406C000240080402404C
:10B8E0001C04024030B560B11A4B026814219A4220
:10B8F00009D2194B1344B3FBF1F1890001641749D4
:10B900000AE0012030BD134B5B421344B3FBF1F15D
:10B91000890001640F490839C163022180F82110B0
:10B92000136843F6F0718B43F0E901142143D0E929
:10B9300002452C432143046921434469214384691E
:10B9400021431943116000214163012242770177AD
:10B95000084630BD08040240F8FFFDBF0000024069
:10B9600070B5044690F82000002501280CD0012075
:10B9700084F8200094F821600020012E06D084F87D
:10B9800020000225284670BD022070BD022684F8E2
:10B990002160A0632068066826F001060660204644
:10B9A000FFF724FBE06A00282068016802D041F01C
:10B9B0000E0106E021F0040101602068016841F0F9
:10B9C0000A0101602068016841F001010160D9E7C6
:10B9D00070B5044600F01CF90546601C02D004480E
:10B9E0000078044400F014F9401BA042FAD370BD63
:10B9F0005C0000202DE9F84FDFF8C891002409F120
:10BA0000040A0AF1040B23460F270BF1040ED1E0C0
:10BA10000125A54006EA0502AA4276D1DFF8A8C1B1
:10BA20004E68A6EB0C0866452BD00DDC032E34D0F7
:10BA300005DC36B3012E19D0022E2FD11BE0112EBA
:10BA400016D0122E2AD119E0B8F5881F19D006DCBD
:10BA5000B8F5803F15D0B8F5801F1FD111E0B8F5BB
:10BA6000001F0ED0B8F5041F18D10AE0CB6815E00E
:10BA7000CB681B1D12E0CB6808330FE0CB680C339A
:10BA80000CE08B682BB1012B4FF0080303D045610C
:10BA900004E0042302E0056100E00023FF2A01D84E
:10BAA000064601E000F104064FEA840501D9A5F13C
:10BAB0002005D6F8008007FA05FC28EA0C0803FAEE
:10BAC00005F548EA0508C6F800804D68ED0070D518
:10BAD0003E4DAE6946F00106AE61AD6924F0030645
:10BAE00005F0010500953A4D06EB050CDCF8085011
:10BAF000A607360F07FA06F825EA0805DFF8D4800E
:10BB0000404503D14FF0000825E052E0DFF8C8803F
:10BB1000404502D14FF001081DE0DFF8C0804045EC
:10BB200002D14FF0020816E0DFF8B480404502D1A0
:10BB30004FF003080FE0DFF8AC80404502D14FF032
:10BB4000040808E0DFF8A080404502D14FF0050866
:10BB500001E04FF0060808FA06F848EA0508CCF8B4
:10BB600008804D68D9F80060ED034D4601D51643B5
:10BB700000E096432E604D68DAF80060AD0355464C
:10BB800001D5164300E096432E604D68DBF8006057
:10BB9000ED025D4601D5164300E096432E604D68E8
:10BBA000DEF80060AD02754601D5164300E096430D
:10BBB0002E60641C0A681646E2407FF429AFBDE897
:10BBC000F88F000000040140000011100010024036
:10BBD0000000014000080140000C0140001001403D
:10BBE0000014014000180140001C0140806808401A
:10BBF00000D001207047C2680A4201D041617047FD
:10BC0000016170470AB1016170470904FBE7000058
:10BC100001488068704700005C00002070B5040097
:10BC200011D021684CF6CC400860216845F255508F
:10BC30000860D4E9000141602168A0688860FFF7CE
:10BC4000E7FF054609E0012070BD00BFFFF7E0FFF8
:10BC5000401B302801D9032070BD2068C06800282F
:10BC6000F4D121684AF6AA200860002070BD00685F
:10BC70004AF6AA210160002070470000024881684E
:10BC800002781144816070475C000020074810B5BD
:10BC9000016841F010010160032000F09FF80020CE
:10BCA00000F006F800F03EF8002010BD0020024031
:10BCB00000B5014687B000221C2000F06FF81C2060
:10BCC00000F05FF81448C16941F00101C161C06929
:10BCD00005A900F001000690684600F091F900F017
:10BCE000AFF90E494000B0FBF1F10D484FF0804232
:10BCF000491E0260416040F2E7320021C0E90321A1
:10BD0000816000F085FB10B1012007B000BD044840
:10BD100000F09AFBF9E700000010024040420F00DB
:10BD2000040200200C4808B5816941F001018161DD
:10BD3000816901F001010091C16941F08051C16147
:10BD4000C06900F0805000900448416821F0E06133
:10BD500041F00071416008BD001002400000014048
:10BD600000280DDB00F01F020121914040098000F6
:10BD700000F1E020C0F88011BFF34F8FBFF36F8F49
:10BD80007047002809DB00F01F02012191404009A3
:10BD9000800000F1E020C0F800117047F0B40E4BB5
:10BDA0001B680C46C3F30223C3F10705042D00D919
:10BDB0000425191D072901D2002300E0DB1E0126FE
:10BDC00006FA05F1491E214099409E40761E164014
:10BDD0003143F0BC02F0CEBE0CED00E0064900F0AD
:10BDE000070208684FF6FF03184040EA0220034AA2
:10BDF00010430860704700000CED00E00000FA05F9
:10BE000010B52CA401461DCC86B08DE81D002DA0D8
:10BE10002D4C00680490002004292FD00BDC012950
:10BE20002FD0022928D100F01BF96168C1F38131BC
:10BE3000491C49001EE0082920D010291CD1616846
:10BE40002268D20118D5C1F38342C9031DF802004C
:10BE500009D5616804AAC1F34041515C1B4AB2FB99
:10BE6000F1F1484301E01A4948436168490203D4AB
:10BE700040000321B0FBF1F006B010BD00F000F966
:10BE8000FAE7226AC2F30121012903D1920701D501
:10BE9000C803F1E7022905D1626A920702D549F683
:10BEA0004040E9E70329E7D121688903E4D54FF24F
:10BEB0002440E1E702030405060708090A0B0C0DFC
:10BEC0000E0F1010010200000010024000127A0054
:10BED00000093D002DE9F0470F46050061D0434EB3
:10BEE000306800F00700B84209D2306820F007003F
:10BEF00038433060306800F00700B84251D12868FC
:10BF00003B4C810712D5400703D5606840F4E060E0
:10BF100060602878000703D5606840F46050606076
:10BF20006068A96820F0F000084360602878C007C6
:10BF300028D06868012810D02168022810D089070D
:10BF400000292EDA616821F0030101436160FFF7E7
:10BF50005FFE804641F288390DE021688903EFE7F2
:10BF60008901EDE7FFF754FEA0EB0801494502D92E
:10BF70000320BDE8F0876068696800F00C00B0EB52
:10BF8000810FEFD1306800F00700B8420BD930685C
:10BF900020F0070038433060306800F00700B842F6
:10BFA00001D00120E5E72878400705D56068E968F9
:10BFB00020F4E060084360602878000706D56068D8
:10BFC000296920F4605040EAC100606000F058F830
:10BFD0006168084AC1F30311515CC8400649086012
:10BFE00006480068FFF764FE0020C2E70020024018
:10BFF00000100240FCAF0108680000206000002033
:10C000000F2202600C4A536803F003034360536835
:10C0100003F0F0038360536803F4E063C360526885
:10C020004FF4E06303EAD20202610448006800F0C2
:10C030000700086070470000001002400020024026
:10C040000448054900684968044AC1F30221515C6B
:10C05000C840704768000020001002400CB0010882
:10C060000448054900684968044AC1F3C221515C8B
:10C07000C840704768000020001002400CB0010862
:10C0800012A185B00FC98DE80F0014A0144A0068F2
:10C0900004905168134801F00C03042B10D0082BB6
:10C0A0000ED1C1F38343C9031DF803000AD55168BB
:10C0B00004AAC1F34041515C0A4A5043B0FBF1F07D
:10C0C00005B0704708494843FAE700000203040539
:10C0D000060708090A0B0C0D0E0F101001020000D4
:10C0E0000010024000127A0000093D002DE9F84FCF
:10C0F000040070D02078C04DC00749D06868C0F3F4
:10C100008100012807D06868C0F38100022809D1A6
:10C110006868C00306D52868800339D560680028A0
:10C12000E7D035E06068B0F5803F0BD010B1B0F5D6
:10C13000A02F11D0286820F480302860286820F4CF
:10C14000802002E0286840F480302860606890B168
:10C15000FFF75EFD06460AE0286840F4802028606C
:10C16000F0E700BFFFF754FD801B642873D82868F0
:10C170008003F7D50CE0FFF74BFD064605E000BF56
:10C18000FFF746FD801B6428F0D828688003F7D4A9
:10C1900020789A4E80074FF001094FF0000839D5FA
:10C1A000686810F00C0F07D06868C0F3810002289F
:10C1B00009D16868C00306D42868800714D52069AF
:10C1C000012808D110E02069B0B1C6F80090FFF74F
:10C1D0001FFD074605E00AE1FFF71AFDC01B022814
:10C1E000C4D828688007F7D52868616920F0F8006E
:10C1F00040EAC10028600DE0C6F80080FFF708FDA6
:10C20000074604E0FFF704FDC01B022823D8286876
:10C210008007F7D4207800072CD57948A169D9B1D7
:10C22000C0F80090FFF7F4FC074604E0FFF7F0FCCD
:10C23000C01B02280FD8686A8007F7D571484FF4F1
:10C24000FA510068B0FBF1F0009000BF0098411E69
:10C250000091FAD20EE080E0C0F80080FFF7D8FC31
:10C26000074604E0FFF7D4FCC01B022875D8686AB3
:10C270008007F7D42078400760D5E8690027C00020
:10C2800008D4E86940F08050E861E869012700F0CF
:10C29000805000905C480168C90513D4016883464A
:10C2A00041F480710160FFF7B3FC824606E000BFF5
:10C2B000FFF7AEFCA0EB0A0064284ED8DBF80000C4
:10C2C000C005F5D5E06801280AD008B1052813D0CB
:10C2D000286A20F001002862286A20F0040002E0A9
:10C2E000286A40F001002862E06841F2883B98B17A
:10C2F000FFF78EFC82460BE0286A40F004002862BB
:10C30000EEE700BFFFF784FCA0EB0A0159455AD8BD
:10C31000286A8007F6D50CE0FFF77AFC824605E034
:10C32000FFF776FCA0EB0A0159454CD8286A800734
:10C33000F6D41FB1E86920F08050E861E06988B365
:10C340006968C1F38101022944D00228C6F86080DF
:10C3500004D0FFF75DFC044638E034E0FFF758FCFA
:10C36000074604E0FFF754FCC01B02282BD82868BE
:10C370008001F7D4206AB0F5803F05D16868A168D4
:10C3800020F4003008436860D4E908010843696874
:10C3900021F4741108436860C6F86090FFF738FC18
:10C3A000044606E025E000BFFFF732FC001B022830
:10C3B00009D828688001F7D51BE000BFFFF728FCEB
:10C3C000001B022802D90320BDE8F88F28688001ED
:10C3D000F4D40EE00128F7D06868226A00F48031B6
:10C3E000914204D1616A00F47010884201D00120AA
:10C3F000EAE70020E8E700000010024000004242A7
:10C40000800442426800002000700040704770477E
:10C4100010B5040003D094F83D0010B107E00120EE
:10C4200010BD002084F83C00204600F00CF80220EB
:10C4300084F83D00211D206801F024FC012084F8CF
:10C440003D00002010BD70470168CA6842F001023B
:10C45000CA600068816801F00701062903D00168FD
:10C4600041F00101016000207047704770B504463B
:10C47000006801694FF00005C943890715D4C168F8
:10C48000C943890711D4E91E016101202077206882
:10C4900080698007204602D0FFF7E7FF04E000F044
:10C4A00098F8204600F096F8257720680169C9437E
:10C4B000490717D4C168C943490713D46FF0040171
:10C4C0000161022020772068806910F4407F2046B7
:10C4D00002D0FFF7CAFF04E000F07BF8204600F02E
:10C4E00079F8257720680169C943090716D4C1681E
:10C4F000C943090712D46FF00801016104202077B5
:10C500002068C0698007204602D0FFF7AEFF04E034
:10C5100000F05FF8204600F05DF82577206801699B
:10C52000C943C90617D4C168C943C90613D46FF0FB
:10C5300010010161082020772068C06910F4407F55
:10C54000204602D0FFF791FF04E000F042F82046B9
:10C5500000F040F8257720680169C943C90708D170
:10C56000C168C943C90704D1891E0161204600F092
:10C5700032F820680169C943090609D4C168C94372
:10C58000090605D46FF0800101612046FFF73EFFE8
:10C5900020680169C943490609D4C168C9434906ED
:10C5A00005D46FF040010161204600F01BF82068BF
:10C5B0000169C94389060BD4C168C943890607D4F8
:10C5C0006FF0200101612046BDE87040FFF71FBFFA
:10C5D00070BD704770470068B0F1804F01D1FFF720
:10C5E0004DBB7047704710B504460068416994F828
:10C5F0003920C1F3C011212A0BD151B1416921F079
:10C6000080014161206B08B1FEF78CFF204601F0EC
:10C61000BBFC2068416994F83A20C1F38011222ABA
:10C620000BD151B1416921F040014161606B08B10A
:10C63000FEF778FF204601F099FC002010BD0000B5
:10C6400038B54D4A016800235414914220D14B491A
:10C65000CA68521CCA6001680A684A6800920A687F
:10C660004A6800920A684A6800920A684A6800921A
:10C670000A6849680091C36300F06EFD012879D112
:10C680003F49224601F5075000F064FA3D486CE04E
:10C690003D4A914215D10A684A6800920A684A6880
:10C6A00000920A684A6800920A684A6800920A681A
:10C6B00049680091C363314932480122891CC0385E
:10C6C00030E0324A914215D10A684A6800920A68FD
:10C6D0004A6800920A684A6800920A684A680092AA
:10C6E0000A6849680091C363244926480122091D4C
:10C6F000803817E0264A914218D10A684A680092A9
:10C700000A684A6800920A684A6800920A684A6899
:10C7100000920A6849680091C363184919480122C8
:10C72000491D4030BDE8384000F060BA194A9142D6
:10C7300020D10A684A6800920A684A6800920A682A
:10C740004A6800920A684A6800920A68496800913B
:10C75000C36300F001FD00280CD10949224601F510
:10C76000065000F0F7F9074840380068C16841F00A
:10C770001001C16038BD0000004C0040480100209D
:10C78000FC660020BC8800200038014000440040C6
:10C79000005000400048004070B502680446106830
:10C7A000D168536910F00F0F51D003F0010501F467
:10C7B000907635435DD0C20705D0CA0503D5E26B3C
:10C7C00042F00102E263420705D5DA0703D0E26BCB
:10C7D00042F00202E263820705D5DA0703D0E26B7A
:10C7E00042F00402E263020705D5DA0703D0E26BE8
:10C7F00042F00802E263E26B002A34D0800604D5DE
:10C80000880602D5204601F0C8FB20684069E16B2C
:10C81000C0F3801001F008010143204624D001F04C
:10C82000A5FB2068416949061AD5416921F04001FC
:10C830004161606BA0B11B494163606BFEF796FEDE
:10C84000002810D0606B416BBDE87040084783063C
:10C850000FD58B060DD52046BDE8704001F09DBB7D
:10C860002046FFF7EDFE70BDFFF7EAFE0020E06313
:10C8700070BD030606D50B0604D52046BDE8704002
:10C8800001F032BC4006F3D54806F1D5D168204608
:10C8900021F04001D160202184F8391000F0FEFA27
:10C8A00070BD0000CDDE000870B5040004D094F81F
:10C8B0003900002510B106E0012070BD84F8385021
:10C8C000204600F023F8242084F839002068C1684D
:10C8D00021F40051C160204601F0AAFB20680169E3
:10C8E00021F4904101612068416921F02A014161F0
:10C8F0002068C16841F40051C160E563202084F8DC
:10C90000390084F83A00002070BD00002DE9F043A2
:10C9100085B00024009401940294039405460168B4
:10C920007F48DFF8F8C1022203237E4F06156145D8
:10C9300025D1816941F480418161816901F480419F
:10C940000491816941F0040181618069694600F0C8
:10C95000040004901002CDE9000203933846FFF76B
:10C9600049F8CDE90064694638460294FFF742F879
:10C97000002202212520FFF711FA25202AE0DFF806
:10C98000A8814FF0040C414529D1C16941F400311F
:10C99000C161C16901F400310491816941F0040170
:10C9A00081618069694600F00400CDE90330CDE97A
:10C9B00000C23846FFF71EF80820CDE9000469469A
:10C9C00038460294FFF716F8002203212620FFF7CD
:10C9D000E5F92620FFF7D5F905B0BDE8F083DFF8CB
:10C9E0004C814FF400674FF08009414537D1C16950
:10C9F00041F48021C161C16901F480210491816900
:10CA000041F0080181618069CDE9006200F0080011
:10CA1000CDE90330464E69463046FEF7EBFFCDE9DF
:10CA20000074694630460294FEF7E4FF424E4148E6
:10CA3000C6E90004C6E9024934617461B461304654
:10CA4000F461FEF74FFF08B1FEF71AFB6E63002298
:10CA5000012127207562FFF7A1F92720BAE7DFF847
:10CA6000DC80414537D1C16941F40021C161C16910
:10CA700001F400210491816941F010018161806914
:10CA8000CDE9006200F01000CDE903302C4E69467C
:10CA90003046FEF7AFFFCDE9007469463046029498
:10CAA000FEF7A8FF284E2748C6E90004C6E9024958
:10CAB00034617461B4613046F461FEF713FF08B16C
:10CAC000FEF7DEFA6E630022012134207562FFF763
:10CAD00065F934207EE71D4A91427FF47DAFC1693C
:10CAE00041F48011C161C16901F48011049181692F
:10CAF00041F0200181618069CDF800C000F0200084
:10CB000004900120029069461148FEF773FF00224D
:10CB100003213520FFF742F935205BE7003801405B
:10CB2000001002400008014000440040004800405E
:10CB3000000C0140300002403C890020004C0040C5
:10CB40000010014030040240808900200050004065
:10CB500000140140F8B5044690F83A0020283CD172
:10CB6000C1B3BAB394F83800012836D0012084F854
:10CB70003800A162A2850025E563222084F83A00EE
:10CB8000636B17489862636B1648D862636B1648EC
:10CB90001863606B134645630846666B216802465E
:10CBA0003046091DFEF7DCFE2068016841680091EF
:10CBB00084F83850C16841F48071C16020684169CF
:10CBC00041F0010141612068416941F0400141614A
:10CBD0000020F8BDFFE70120FBE70220F9E7000095
:10CBE00027DF000863DF0008DDDE000890F83A3038
:10CBF000202B22D1F9B1F2B190F83830012B1CD0A2
:10CC000081628285C2850021C163222280F83A2098
:10CC100080F838100168CA6842F48072CA600168FE
:10CC20004A6942F001024A610068C16841F020018E
:10CC3000C16000207047012070470220704700004B
:10CC40002DE9F84F00685A490126DFF86881002570
:10CC5000884226D1424698F802005749D2780D28DA
:10CC600011D00A280FD03F2A07D28854521C88F8C6
:10CC70000320FEF7CDFFC8F810004E494E480122B0
:10CC8000891C803031E0002AF7D08D544A49521C6B
:10CC9000A1F18000FBF744FF88F8006088F803509A
:10CCA000EBE74649884215D198F8060098F8041039
:10CCB0003F2809D2404A40321154401C88F80600EF
:10CCC000FEF7A6FFC8F814003A493B480122091DA7
:10CCD000C0300AE03A4988420BD198F8050007F0C5
:10CCE00029FB344901223748491DBDE8F84FFFF7B9
:10CCF0007DBF3549DFF8D490DFF8D4A0354C42F23F
:10CD0000FF774FF4005B884226D1D8F80800401C1A
:10CD1000C8F8080000F020FA012813D1208800F597
:10CD20000050B8420ED220884F4648445A462A49FD
:10CD3000FBF76FFE208800F50050208020883D54CE
:10CD40008AF800601F4C403C2068016840680090F1
:10CD50005A462149204622E02049884226D100F047
:10CD6000FBF998B9208800F50050B8420ED220880F
:10CD70004F4648445A461849FBF74BFE208800F5B9
:10CD80000050208020883D548AF800600D4C803C83
:10CD900020680168406800905A460F492046FFF716
:10CDA000D9FE2068C16841F01001C160BDE8F88F6C
:10CDB00000380140480100207C87002000440040EA
:10CDC00000500040FC880020004C0040442E002011
:10CDD0006C00002072000020FC660020004800402B
:10CDE00070472DE9F843044690F839001F4616466F
:10CDF0000D46202850D1A5B19EB194F838000128E5
:10CE00004AD0012084F838004FF00008C4F83C8074
:10CE1000212084F83900FEF7FBFEA6848146E684D3
:10CE200026E00120BDE8F883E08C401EE084A06885
:10CE30004B46B0F5805F4FF000024FF08001204676
:10CE4000009703D001F081F9E8B90DE001F07DF918
:10CE5000C8B928882168C0F308004860206908B173
:10CE60006D1C05E0AD1C03E0216815F8010B48605E
:10CE7000E08C0028D8D14B46002240212046009764
:10CE800001F063F908B10320CCE7202084F83900D1
:10CE900084F838800020C5E70220C3E7704700000F
:10CEA00006490020064B0A1D0C682406FCD51C5CB4
:10CEB0001460401C2728F7D3FEE70000003801402B
:10CEC000D4AF01080148FEF7D2BE0000C48900209B
:10CED000114808B5416941F001014161416901F022
:10CEE00001010091416941F0020141614069002264
:10CEF00000F00200009011460D20FEF74FFF0D20BC
:10CF0000FEF73FFF002211463A20FEF747FFBDE83B
:10CF100008403A20FEF735BF001002402DE9F041ED
:10CF200086B000253F4800950195029503958169DB
:10CF300041F020018161816901F020010491816942
:10CF400041F004018161816901F00401049181696A
:10CF500041F008018161816901F008010491816952
:10CF600041F01001816180692F4F00F010000490A2
:10CF7000002280213846FEF745FEBE1500223146CC
:10CF80003846FEF73FFEDFF8A4800022012140462C
:10CF9000FEF738FE002204214046FEF733FE022051
:10CFA000CDE9025001248025CDE900546946384678
:10CFB000FEF720FD694638460096FEF71BFD6946E0
:10CFC00040460094FEF716FD042000906946404656
:10CFD000FEF710FD002210214046FEF713FE11203F
:10CFE00001901020009069464046FEF703FD104E68
:10CFF000002240213046FEF705FE4020CDE9000426
:10D0000069463046FEF7F6FC002280213046FEF7E6
:10D01000F9FD694630460095FEF7ECFC06B0BDE828
:10D02000F081000000100240000C0140001001409F
:10D03000000801400C4810B50A4901604FF4E13185
:10D040004160002181600C22C160C0E9041281614D
:10D05000C161FFF729FC002803D0BDE81040FEF7AE
:10D060000FB810BD004C0040BC8800200E4810B521
:10D070000C4901604FF4965141604FF4805181603A
:10D0800000214FF48062C0E903120422C0E90521A7
:10D09000C161FFF709FC002803D0BDE81040FDF78F
:10D0A000EFBF10BD00500040FC8800200C4810B5B8
:10D0B0000A4901604FF4E1314160002181600C2296
:10D0C000C160C0E904128161C161FFF7EDFB002876
:10D0D00003D0BDE81040FDF7D3BF10BD00380140BC
:10D0E000FC8700200C4810B50A4901604FF4165126
:10D0F0004160002181600C22C160C0E9041281619D
:10D10000C161FFF7D1FB002803D0BDE81040FDF757
:10D11000B7BF10BD004400403C8800200C4810B54B
:10D120000A4901604FF4E1314160002181600C2225
:10D13000C160C0E904128161C161FFF7B5FB00283D
:10D1400003D0BDE81040FDF79BBF10BD0048004074
:10D150007C880020FEE7000001484079704700000D
:10D160007C00002001488079704700007C0000208E
:10D1700010B504200CF0B2F80149C86010BD0000E1
:10D180007C00002001B50E499DF800008A7990428C
:10D1900010D002280ED8887101226946822005F03D
:10D1A00023F89DF8000030B1012806D005A109A0A0
:10D1B00007F03AFB08BD0EA1F9E70EA1F7E7000062
:10D1C0007C0000205769466928C5E4CDF8C8C8B579
:10D1D000E32900003E204E45543A20C1AACDF8B7BD
:10D1E000BDCABDD2D1B1A3B4E6202D3E2025730027
:10D1F000344700005769466928B9CCB6A8C8C8B5F5
:10D20000E329000038B5194D00242C706C70EC70C7
:10D210002C718DF8004001226946822004F09AFEAC
:10D220009DF80000022801D98DF800409DF800000B
:10D23000A87140B10EA007F0F7FA012005F070FBCD
:10D240000120687138BD6C71002005F069FB07F0A2
:10D250008FFE02F02FFA07F0B3FEE87810B10EA0AF
:10D2600007F026FB14480078287038BD7C000020A9
:10D270003E204E45543A20C9CFB4CEC1AACDF8B70E
:10D28000BDCABDCEAA2057694669A3AC5769466995
:10D2900020D3C5CFC80000003E20344720CEDE207A
:10D2A00053494D20BFA8A3ACC7EBB2E5C8EB205350
:10D2B000494D20BFA80000006D0000202DE9F0417D
:10D2C000244E8046B4B0B07815460C464FF0FF3778
:10D2D00008B121A003E007F05DFE18B127A007F018
:10D2E000A3FA21E0707988B1B8F1000F1AD0CCB15F
:10D2F0002078B8B12AA14046FBF7BFFAB0B1434647
:10D300002AA2C82102A8CDE9004519E02A462146F3
:10D31000404602F015FB044607F052FE204634B0AA
:10D32000BDE8F08107F04CFE3846F8E70DB12CA0BF
:10D3300000E02DA0CDE9004043462DA2C82102A85F
:10D34000FBF7CEF802A808F067FA07F039FE0020D4
:10D35000E5E700007C0000203E204E45543A20BD09
:10D36000F8B6C82FBDE1B9FBC9CFB1A8B1BBB6AA09
:10D37000C6FA2028B7A2CBCDC3A629003E204E4531
:10D38000543A20BDF8B6C82FBDE1B9FBC9CFB1A84A
:10D39000B1BBB6AAC6FA2028415420C3A629000072
:10D3A00070726F6772657373000000007B2268659E
:10D3B00061646572223A222573222C22626F64799D
:10D3C000223A7B226964223A22252E313673222C9E
:10D3D0002270726F6772657373223A25647D7D00D7
:10D3E000747275650000000066616C736500000072
:10D3F0007B22686561646572223A222573222C22A1
:10D40000626F6479223A7B226964223A22252E31A6
:10D410003673222C2273756363657373223A257306
:10D420007D7D000002F006BBF8B54A4C42F2107652
:10D43000204661790069002529B1474F39780029D4
:10D4400057D0256179E0454F397879B1256125813B
:10D450000020FFF797FE00BF07F08AFD02F05AFB9D
:10D4600007F0AEFD387820703D4870E0E17811B9E2
:10D47000217900293BD028B1FEF7CAFB2169401A67
:10D48000B042E9D3FEF7C4FB20612089401C83B27F
:10D490002381032000902279E17832A007F008FA76
:10D4A000E570257107F064FD02F004F907F088FDCE
:10D4B000E07808B92079A8B120890328CCD30321CA
:10D4C00038A007F0F5F942A007F0F2F9012005F0C5
:10D4D00027FA00F0C3FF2570657001206071258177
:10D4E0002561B9E740A007F09FF92581B4E72561E0
:10D4F000FBE728B1FEF78CFB2169401AB0421DD32F
:10D50000FEF786FB206120890122401C81B2218127
:10D510003FA007F0CDF907F02BFD07F021FF0646ED
:10D5200007F04EFD4EB1208940B140A007F0C0F990
:10D5300007F0E0FE2581256100E0258107F018FD58
:10D5400008F0B8F807F03CFD387820703F480078C4
:10D550006070F8BD7C000020980000206D00002065
:10D560006E0000203E204E45543A20344720B2BB86
:10D57000BFC9D3C320286E6F5F73696D3D25642CCE
:10D58000206E6F5F7369676E616C3D256429A3AC83
:10D59000D6D8CAD4B3F5CABCBBAF2025642F256446
:10D5A000000000003E204E45543A20344720D6D893
:10D5B000CAD420256420B4CEC8D4B2BBBFC9D3C35B
:10D5C000A3ACBBD8CDCBB5BD2057694669000000E0
:10D5D0003E204E45543A20C7D0BBBB203447202DB7
:10D5E0003E205769466900003E204E45543A20349B
:10D5F000472053494DBFA82FD0C5BAC5D5FDB3A309
:10D60000BBF2CDF8C2E7D2D1BBD6B8B4000000005F
:10D610003E204E45543A205769466920C1ACBDD3DF
:10D62000B3A2CAD42025642F256400003E204E45B5
:10D63000543A205769466920C1ACBDD3CAA7B0DCB3
:10D64000A3ACBBD8CDCBB5BD20344700990000209A
:10D6500030B51B4D04469BB0A87808B119A003E073
:10D6600007F098FC28B120A01BB0BDE8304007F0BF
:10D67000DBB868790028204618D00DF0FFF8CDE916
:10D68000000122A2602102A8FAF72AFF02A808F0EE
:10D69000C3F820460DF0F2F802460B4628A007F02A
:10D6A0009DF81BB0BDE8304007F08ABC0DF0E6F8ED
:10D6B00002460B4629492A48FDF724FCE9E7000009
:10D6C0007C0000203E204E45543A20656E6572670E
:10D6D0007920C9CFB1A8B1BBB6AAC6FA2028B7A293
:10D6E000CBCDC3A6290000003E204E45543A20650C
:10D6F0006E6572677920C9CFB1A8B1BBB6AAC6FA68
:10D700002028415420C3A629000000007B22686520
:10D7100061646572223A22696F742E70726F702E86
:10D72000706F7374222C22626F6479223A7B2265B7
:10D730006E65726779223A252E32667D7D00000083
:10D740003E204E45543A20656E6572677920D2D1ED
:10D75000B7A2B2BC20252E3266000000BC0000201B
:10D7600060B7010870B5164D044698B0A8784FF020
:10D77000FF3608B113A003E007F00CFC28B119A094
:10D7800007F052F8304618B070BD687910B154B146
:10D79000012309E00CB1012200E0002219491A48D6
:10D7A000FDF7B0FB08E0002318A260216846FAF7F5
:10D7B00097FE684608F030F807F002FC0020E2E728
:10D7C0007C0000203E204E45543A20B5E7C1BFC939
:10D7D000CFB1A8B1BBB6AAC6FA2028B7A2CBCDC399
:10D7E000A62900003E204E45543A20B5E7C1BFC9E6
:10D7F000CFB1A8B1BBB6AAC6FA2028415420C3A60F
:10D8000029000000BC00002038B601087B226865B2
:10D8100061646572223A22696F742E70726F702E85
:10D82000706F7374222C22626F6479223A7B2270AB
:10D830006F77223A25647D7D00000000F0B5184D19
:10D840000646B3B0A87814460F4608B115A003E009
:10D8500007F0A0FB28B11BA033B0BDE8F04006F0F4
:10D86000E3BF0CB1234603E00FB11EA300E01EA3EB
:10D87000687970B1009333461FA2C82101A8FAF756
:10D880002FFE01A807F0C8FF33B0BDE8F04007F055
:10D8900097BB324621492248FDF734FBF4E70000EC
:10D8A0007C0000203E204E45543A20D3A6B4F0C957
:10D8B000CFB1A8B1BBB6AAC6FA2028B7A2CBCDC3B8
:10D8C000A62900003E204E45543A20D3A6B4F0C904
:10D8D000CFB1A8B1BBB6AAC6FA2028415420C3A62E
:10D8E000290000004F4B0000636F6D6D616E642076
:10D8F0006661696C656400007B226964223A2225B6
:10D9000073222C22636F6465223A302C226D65737A
:10D9100073616765223A222573227D00BC000020D6
:10D92000A0B401082DE9F04FCBB0DFF848910746CD
:10D93000DDE9548A99F802001C4615460E4608B1E6
:10D940004DA003E007F026FB28B153A04BB0BDE883
:10D95000F04F06F069BF584899F80510DFF85C9160
:10D96000007819B3002860D050460CF087FF83463A
:10D97000019156980CF082FF00908A4657980CF05F
:10D980007DFFCDE90676CDE90854019BCDF82880CE
:10D99000CDE904B3009A8DE80704B9F87430484A19
:10D9A0004FF480710BA8FAF79BFD5AE010B3504674
:10D9B0000CF064FF83468A4656980CF05FFFCDE971
:10D9C000000157980CF05AFFCDE90854CDF8288093
:10D9D000CDE90676CDE904BA0246DDE90003CDE9DA
:10D9E0000021CDE90203B9F8742034493548FDF728
:10D9F00089FA39E006F0A8FA0CF040FF82468B461F
:10DA000057980CF03BFF02460B46CDF81880039662
:10DA10008DE88C00CDE90454CDE908ABB9F8742049
:10DA200026492948FDF76EFA1EE006F08DFA0CF043
:10DA300025FF82468B4657980CF020FF02460B4686
:10DA4000CDF8188003968DE88C00CDE90454CDE91B
:10DA500008ABB9F874301D4A4FF480710BA8FAF77F
:10DA60003FFD0BA807F0D8FE4BB0BDE8F04F07F024
:10DA7000A7BA00007C0000203E204E45543A20D733
:10DA8000B4CCACC9CFB1A8B1BBB6AAC6FA2028B7EE
:10DA9000A2CBCDC3A62900003E204E45543A20D744
:10DAA000B4CCACC9CFB1A8B1BBB6AAC6FA20284144
:10DAB0005420C3A62900000064010020BC000020FF
:10DAC000C4B7010860B5010898B601084CB8010850
:10DAD00030B5134C054699B0A07808B111A003E009
:10DAE00007F058FA28B117A019B0BDE8304006F089
:10DAF0009BBE607968B12B461AA260216846FAF78E
:10DB0000EFFC684607F088FE19B0BDE8304007F02A
:10DB100057BA2A4620492148FDF7F4F9F4E70000F6
:10DB20007C0000203E204E45543A20B0E6B1BEC9EC
:10DB3000CFB1A8B1BBB6AAC6FA2028B7A2CBCDC335
:10DB4000A62900003E204E45543A20B0E6B1BEC999
:10DB5000CFB1A8B1BBB6AAC6FA2028415420C3A6AB
:10DB6000290000007B22686561646572223A22699F
:10DB70006F742E70726F702E706F7374222C22620D
:10DB80006F6479223A7B226677766572223A222583
:10DB900073227D7D00000000BC000020F8B4010865
:10DBA0007047000010B5502080F31188BFF34F8FED
:10DBB000BFF36F8F0BF032FE18B104494FF0805065
:10DBC0000860002080F3118810BD000004ED00E023
:10DBD00030B58FB028216846FAF7FEFF14210AA855
:10DBE000FAF7FAFF01210804CDE90010002402949D
:10DBF00002250491CDE907504FF4E01009906846E2
:10DC0000FEF774FA08B172B6FEE70F20CDE90A05F7
:10DC10004FF48060CDE90C4002210AA80E94FEF773
:10DC200059F9002801D072B6FEE70FB030BD0000F0
:10DC30000D48016841F00101016041680B4A114043
:10DC4000416001680A4A11400160016821F48021A5
:10DC50000160416821F4FE0141604FF41F018160C1
:10DC60000449C00308607047001002400000FFF83C
:10DC7000FFFFF6FE08ED00E00148FEF7F7BB0000ED
:10DC800004020020F0B502681C4B1D4D1D4E1E4FB6
:10DC90001E4C4FF0804C984209D0A04207D06045FE
:10DCA00005D0A84203D0B04201D0B84204D122F03E
:10DCB000700E4A6842EA0E02984209D0A04207D08C
:10DCC000604505D0A84203D0B04201D0B84203D18C
:10DCD00022F44075CA682A434D6922F080022A4323
:10DCE00002608A68C2620A688262984201D0A042D9
:10DCF00001D10969016301214161F0BD002C01409E
:10DD00000004004000080040000C004000340140C6
:10DD1000F8B51E4C20680168C943C90631D40168B2
:10DD20000026406800902046FEF75DFC606B0068AE
:10DD30004068174DC0F500500004000C28801AD030
:10DD4000FFF70AFA012816D1124C20882A8842F2DD
:10DD5000FF71104488420ED20F4F20880F4938447B
:10DD6000FAF757FE208829880844208020880C492B
:10DD70003E54012008704FF4005208490348FEF752
:10DD8000E9FEBDE8F8400148FEF706BDBC8800206A
:10DD90004401002072000020442E0020FC66002078
:10DDA0006C000020F8B52A4C054694F83A0020286B
:10DDB00002D02046FEF717FC2648AA00B0FBF2F37B
:10DDC0006421B3FBF1F36FF0180673436560B0FB99
:10DDD000F2F5B0FBF2F605EB8305322303EB0515F4
:10DDE000B5FBF1F5B6FBF1F605F0F00505EB061510
:10DDF000B0FBF2F6B0FBF2F0B0FBF1F06FF01802FE
:10DE0000504306EB800003EB0010B0FBF1F0124929
:10DE100000F00F0028440860206801684168009104
:10DE2000016841680091016841680091016841689A
:10DE300000910168406800904FF40052074904487F
:10DE4000FEF788FE2068C16841F01001C160F8BD8E
:10DE5000BC88002000E9A435084C0040FC66002086
:10DE600010B50A4C94F83A00202802D02046FEF75C
:10DE7000BAFB4FF4005206490448FEF76BFE2068D7
:10DE8000C16841F01001C16010BD0000BC880020D5
:10DE9000FC66002004480068C16821F01001C160E0
:10DEA0000148FEF7A0BB0000BC8800200148FEF737
:10DEB00073BC0000FC880020012202490248FEF7E2
:10DEC00095BE00004D010020FC88002010B5406A7E
:10DED0000021C185C184FEF7B3FB10BD70B5446A53
:10DEE0002068406994F83910C0F3C010002521293A
:10DEF00004D118B1E584204600F046F82068406956
:10DF000094F83A10C0F38010222904D118B1E585A5
:10DF1000204600F02BF8E06B40F01000E063204654
:10DF2000FEF78EFB70BD10B50146406A09680968AE
:10DF3000890613D40021C1850168CA6822F4807261
:10DF4000CA6001684A6922F001024A6101684A69AF
:10DF500022F040024A61202180F83A10FEF770FE5C
:10DF600010BD10B5406AFEF73BFF10BD0168CA68DE
:10DF700022F49072CA6001684A6922F001024A6183
:10DF8000202180F83A1070470168CA6822F0C00268
:10DF9000CA60202180F83910704710B590F83A1007
:10DFA000222901D0022010BD8168B1F5805F11D017
:10DFB0000169002901681FD0496801F07F03816A67
:10DFC0004A1C82620B70C18D491E0904090CC1856F
:10DFD00018D02BE00269816A002A0268526805D0D5
:10DFE000D2B20A80816A491C8162ECE7C2F308025E
:10DFF0000A80816A891CF7E74A68816A4B1C836240
:10E000000A70E0E70168CA6822F02002CA6001686D
:10E01000CA6822F48072CA6001684A6922F001026B
:10E020004A61202180F83A10FEF70AFE002010BD58
:10E030002DE9F041044600680169E26821F440518D
:10E04000114301612169A06808436169084321689F
:10E05000CA6841F20C639A430243CA60206841696E
:10E06000A26921F44071114341611E492068642571
:10E070003226884202D1FDF7F3FF01E0FDF7E0FF11
:10E0800000EBC00101EB001160686FF01807800021
:10E09000B1FBF0F2B2FBF5F2B1FBF0F37A4303EB24
:10E0A0008202B1FBF0F306EB0212B2FBF5F2B3FB16
:10E0B000F5F302F0F00202EB0312B1FBF0F3B1FB57
:10E0C000F0F0B0FBF5F0784303EB800006EB0010B6
:10E0D000B0FBF5F0216800F00F0010448860BDE847
:10E0E000F08100000038014090F83910212901D05A
:10E0F000022070478168B1F5805F016A0BD04A1C2D
:10E100000262026809785160C18C491E0904090C39
:10E11000C1840ED017E009880268C1F3080151607C
:10E1200001690029016A02D0491C0162ECE7891CDF
:10E13000FBE70168CA6822F08002CA600068C16813
:10E1400041F04001C160002070472DE9F041984640
:10E1500017460E460446069D1DE0681C1BD02DB1D7
:10E16000FDF756FDA0EB0800A84214D92068C1684D
:10E1700021F4D071C1602068416921F00101416141
:10E18000202084F8390084F83A00002084F8380010
:10E190000320BDE8F0812068006836EA000004D062
:10E1A0000020B842D9D00020F3E70120F9E70000B1
:10E1B00070B50E4C2078002508B1257010E0E0788D
:10E1C00088B1FDF725FD2169401A64280BD908485C
:10E1D000E278014685548038521CFAF7A1FCE570BC
:10E1E0000348803870BD002070BD00004801002049
:10E1F0007C8700200148FEF7CFBA0000FC87002092
:10E200000B4810B500210170C1700161402109481F
:10E21000FAF7E2FC074840218038FAF7DDFC0449B0
:10E2200004480122891CBDE810408030FEF7DEBCA6
:10E23000480100207C8700202DE9F0410B4C074667
:10E240006078002810D000266670A079884201D23C
:10E25000014600E0491E8DB22A4605493846FAF7C4
:10E26000D8FB7E55A6712846BDE8F0814801002004
:10E27000BC8700200148FEF78FBA00003C880020D0
:10E280000B4810B50021417081714161402109485E
:10E29000FAF7A2FC074840218038FAF79DFC0449B0
:10E2A00004480122091DBDE810408030FEF79EBCE5
:10E2B00048010020BC87002010B5064CA07900283A
:10E2C00007D0FDF7A5FC6169401A142801D9012087
:10E2D000607010BD48010020F8B51E4C2068016830
:10E2E000C943C90630D40168002640680090204622
:10E2F000FEF779F9606B00684068174DC0F5005073
:10E300000004000C288019D0FEF726FFB0B9134C8A
:10E3100020882A8842F2FF71104488420ED2104FA2
:10E32000208810493844FAF774FB2088298808446B
:10E33000208020880C493E54012008704FF4005280
:10E3400008490448FEF706FCBDE8F8400148FEF71E
:10E3500023BA00007C8800204401002072000020C5
:10E36000442E0020FC6600206C000020F8B52A4CEA
:10E37000054694F83A00202802D02046FEF733F9EB
:10E380002648AA00B0FBF2F36421B3FBF1F36FF06F
:10E39000180673436560B0FBF2F5B0FBF2F605EBCF
:10E3A0008305322303EB0515B5FBF1F5B6FBF1F65A
:10E3B00005F0F00505EB0615B0FBF2F6B0FBF2F048
:10E3C000B0FBF1F06FF01802504306EB800003EB56
:10E3D0000010B0FBF1F0124900F00F002844086073
:10E3E00020680168416800910168416800910168F6
:10E3F000416800910168416800910168406800909F
:10E400004FF4005207490448FEF7A4FB2068C16896
:10E4100041F01001C160F8BD7C88002000E9A435FE
:10E4200008480040FC66002010B50A4C94F83A00F9
:10E43000202802D02046FEF7D6F84FF400520649B5
:10E440000448FEF787FB2068C16841F01001C160F5
:10E4500010BD00007C880020FC6600200448006895
:10E46000C16821F01001C1600148FEF7BCB800008E
:10E470007C880020FEE700001CB50C460822694697
:10E4800000F03AFA9DF8031000989DF8072061F318
:10E490001F60019962F31F610A4A0240B2F1005FF6
:10E4A00002D0014608A006E00C48814202D3204475
:10E4B000814204D90AA006F0B7F900201CBD012052
:10E4C0001CBD00000000FE2F3E20564620657874DB
:10E4D0003A2053503D307825580000000080000855
:10E4E0003E205646206578743A2052563D307825B5
:10E4F0005800000070B5054600F012FB00F0DBFA92
:10E500000A4C002210212046FDF77CFBD82000F0A9
:10E5100053FA284600F0D7FA012210212046FDF7D1
:10E5200071FBBDE8704000F0C6BA0000000C01406D
:10E5300000BF00BF00BF00BF704770B50D000446AC
:10E5400024D009F0D5FE25446D1E04E0204600F0DD
:10E550006BFA04F580542004000C01D0AC42F5D9CC
:10E560004FF6FF76A019A8420AD82046FFF7C2FF4F
:10E5700004F58034F6E7204600F056FA04F580549E
:10E58000AC42F8D9BDE8704009F0CEBE70BD02467D
:10E5900000200146535C491C184480B22029F9D35D
:10E5A0007047000010B5044600680649884207D14C
:10E5B0002046FFF7ECFF218C884201D1012010BDDD
:10E5C000002010BD4F5441572DE9F04186B0374827
:10E5D00000240294816941F004018161816901F0A4
:10E5E00004010591816941F008018161816901F0AF
:10E5F00008010591816941F001018161806900F0A4
:10E60000010005902A48416821F0E06141F0007165
:10E6100041600320039001251020CDE90005DFF8BB
:10E62000948069464046FDF7E5F908200090694668
:10E630004046FDF7DFF9204FEE0369463846009665
:10E64000FDF7D8F920208DE8310069464046FDF7F6
:10E65000D1F9012210214046FDF7D4FA0022082109
:10E660004046FDF7CFFA002231463846FDF7CAFA98
:10E6700004A8049400F068F99DF810009DF81110AA
:10E68000000440EA01219DF8120001430B48814239
:10E6900006D00BA006F0B2F8012006B0BDE8F0816C
:10E6A0000FA006F0C1F80020F7E7000000100240BC
:10E6B00000000140000C0140000801401740EF003D
:10E6C0003E2057323551363420B3F5CABCBBAFCAF1
:10E6D000A7B0DC212049443D307825303658000071
:10E6E0003E2057323551363420B3F5CABCBBAFB3E8
:10E6F000C9B9A62C2049443D307825303658000051
:10E7000010B58AB009F0F4FD684600F017F828B19A
:10E7100009F00AFE4FF0FF300AB010BD0198401C0E
:10E720000190BDF81200401CADF81200684600F0E0
:10E730008BF8044609F0F8FD2046EDE730B593B0BC
:10E74000054609F0D5FD222269464FF4002000F06D
:10E75000D3F8222209A94FF4012000F0CDF8684631
:10E76000FFF720FF044609A8FFF71CFF54EA000149
:10E7700008D08CB118B10A99019888420CD3222292
:10E7800069460BE022212846FAF704FA09F0CCFD8D
:10E790004FF0FF3013B030BD222209A92846FAF706
:10E7A00038F909F0C1FD0020F4E710B58AB009F08E
:10E7B0009FFD6846FFF7C2FF28B109F0B5FD4FF095
:10E7C000FF300AB010BD0198401C019001208DF867
:10E7D0001400684600F038F8044609F0A5FD20460C
:10E7E000EFE7000070B58AB014460D46064609F002
:10E7F0007FFD6846FFF7A2FF28B124216846FAF79B
:10E80000EBF9104800900198ADF80860401C0190A9
:10E81000CDF80A5001208DF810008DF8110000206D
:10E82000ADF812008DF814008DF81E00ADF80E4002
:10E83000684600F009F8044609F076FD0AB0204663
:10E8400070BD00004F54415710B58AB001462222D6
:10E850006846FAF7DEF86846FFF799FEADF8200043
:10E8600009F046FD4FF40024204600F0DDF8222296
:10E870006946204600F036F94FF40124204600F0A6
:10E88000D3F822226946204600F02CF909F04CFD0D
:10E890000AB0002010BD00002DE9F04115000E4621
:10E8A000044624D0B5F5807F21D800F039F900F076
:10E8B00002F9104F002210213846FDF7A3F902207B
:10E8C00000F07AF8204600F0FEF8002404E0305D05
:10E8D00000F072F8641CA4B2AC42F8D301221021FB
:10E8E0003846FDF78FF9BDE8F04100F0E4B8BDE827
:10E8F000F0810000000C01402DE9F04115460E4664
:10E90000044609F0F5FC0F4F002210213846FDF7B0
:10E9100079F9032000F050F8204600F0D4F80024E4
:10E9200004E000BF00F044F83055641CAC42F9D359
:10E93000012210213846FDF765F9BDE8F04109F0E4
:10E94000F3BC0000000C014070B50D4D04460022E0
:10E9500010212846FDF756F99F2000F02DF800F011
:10E9600027F8207000F024F8607000F021F8A07003
:10E970002846BDE8704001221021FDF743B9000090
:10E98000000C014070B5094D002210212846FDF70A
:10E9900039F9052000F010F800F00AF804460122C9
:10E9A00010212846FDF72EF9204670BD000C0140CD
:10E9B000FF2000F001B800002DE9F0470024DFF847
:10E9C0006090184F064625464FF40048300601D5A2
:10E9D000012200E0002241464846FDF713F9700687
:10E9E000060EFFF7A5FD012208213846FDF70AF9BA
:10E9F000FFF79EFD6006040E20213846FDF7F6F86D
:10EA0000012801D144F00104002208213846FDF715
:10EA1000F9F86D1C082DD9DB2046BDE8F087000011
:10EA200000080140000C014070B5054600F078F880
:10EA300000F041F80A4C002210212046FDF7E2F8D0
:10EA40002020FFF7B9FF284600F03DF801221021F1
:10EA50002046FDF7D7F8BDE8704000F02CB8000064
:10EA6000000C01402DE9F041C0B015460F4680462C
:10EA700009F03EFC4FF4807617E03446A54200D8FA
:10EA8000ACB2224669464046FFF736FF2246394679
:10EA90006846F9F704FF28B109F046FC002040B0B1
:10EAA000BDE8F081A04427442D1B002DE5D109F0DD
:10EAB0003BFC0120F3E710B500E000BFFFF762FF69
:10EAC000C007FAD110BD10B50446C0F30740FFF7E8
:10EAD00073FFC4F30720FFF76FFFE0B2BDE81040FB
:10EAE000FFF76ABF2DE9F04115460F46064609F0CB
:10EAF000FFFB0DE0F0B2C0F58074A54200D8ACB2C7
:10EB0000224639463046FFF7C7FE264427442D1BD0
:10EB1000002DEFD109F008FC0120BDE8F0810000D4
:10EB200010B5FFF7C8FF084C002210212046FDF762
:10EB300069F80620FFF740FF20460122BDE810409B
:10EB40001021FDF75FB80000000C0140490050EAB9
:10EB5000C12018BF04204A0D18BF40F0010040F248
:10EB6000FF72B2EB515F08BF40F00200012808BFFE
:10EB7000052070470907090E002804DB00F1E0209A
:10EB800080F80014704700F00F0000F1E02080F8DA
:10EB9000141D7047BFF34F8F05480168054A01F403
:10EBA000E06111430160BFF34F8F00BFFDE700003C
:10EBB0000CED00E00400FA05BFF34F8F0548016833
:10EBC000054A01F4E06111430160BFF34F8F00BFBC
:10EBD000FDE700000CED00E00400FA05BFF34F8FE5
:10EBE00005480168054A01F4E06111430160BFF383
:10EBF0004F8F00BFFDE700000CED00E00400FA05B8
:10EC00002DE9F74F144694B00021C4E9021115997B
:10EC1000079121F00045C9498D4206DC1599C4E9E8
:10EC2000000117B00020BDE8F08FC549DFF814A33C
:10EC3000A9423CDD0799C44E0029C44FC44A159926
:10EC4000534619DD0BF030FD554506D0C14AC24B85
:10EC50000BF02AFDC4E900010AE04FF0D352BE4B8D
:10EC60000BF022FD32463B460BF01EFDC4E90001CD
:10EC700017B00120BDE8F08F0AF0C4FF554506D05B
:10EC8000B44AB54B0AF0BEFFC4E900010AE04FF0F8
:10EC9000D352B14B0AF0B6FF32463B460AF0B2FF00
:10ECA000C4E9000117B04FF0FF30BDE8F08FAB4969
:10ECB000A942159978DB21F0004183468846A84A8D
:10ECC000A84B0BF0CBFA0022A74B0AF09BFF0BF0EE
:10ECD000E9F909900BF015FA06460F469C4A53468F
:10ECE0000BF0BCFA43465A460BF0ECFB80468A46D2
:10ECF000984A994B304639460BF0B0FA2A0D012557
:10ED00000B92424653460BF0DDFB032DC4E9000194
:10ED100039D00B98C1F30A51401A05EB451111394E
:10ED2000814230DA9148C346784400EB0510CDF8B3
:10ED30000CA00C90D0E90023304639460BF08EFA37
:10ED400002460B4604910690584603990BF0ACFC22
:10ED500080468A4602460B46584603990BF0A4FCAF
:10ED6000049B069A0BF0A0FC83460C98039139464D
:10ED7000D0E9022330460BF071FA5A46039B0BF0A0
:10ED800093FC6D1CBDE707980028A2BF099817B037
:10ED9000BDE8F08F616881F000416160099817B0AB
:10EDA0004042BDE8F08FFFE784461598C1F3130198
:10EDB000C0F30A50A0F2F5304FEA601800F01F06C9
:10EDC000C6F12000139000200690079041F4801EA9
:10EDD00005206D4676B1664A08EB00017A4452F888
:10EDE000213002EB8101B3404A68139922FA01F104
:10EDF000194305E05F4908EB0002794451F82210FD
:10EE0000A1FB0E27A1FB0C131A449A4234BF012325
:10EE1000002303EB070A05EB8003D3E901B70F4496
:10EE20008F4234BF0121002193448B4411B193459B
:10EE300002D903E0934501D2012100E00021C3E99A
:10EE400001B7514445F82010011EA0F10100C1DCBA
:10EE50000298059F00F10050800F12900298DDE9A2
:10EE6000035680000BF04DF9834628460D910BF0B8
:10EE70005FF96FF01D020CF03BF8CDE90E01304652
:10EE80000BF056F96FF03D020CF032F880468A46DE
:10EE900038460BF04DF96FF05D020CF029F807468B
:10EEA0004246534611910AF0ADFEDDE90E230AF009
:10EEB000A9FE5A460D9B0AF0A5FE00250E465A46AD
:10EEC00028460D9B0BF0F0FBDDE90E230BF0ECFB6D
:10EED000424653460BF0E8FB3A46119B0BF0F2FA20
:10EEE000DFF898A0244A53460BF0B8F90746884645
:10EEF000234A244B314628460BF0B0F93A464346A4
:10EF00000AF080FE074688464FF0A8425346314635
:10EF100028460BF0A3F93A4643460AF073FE159AC9
:10EF200012F0004F04D0129A81F000415242129226
:10EF3000C4E90001129817B0BDE8F08FFB21E93F4A
:10EF40007CD90240FB21F93F7370032E8A19A33B41
:10EF5000000040543163621A61B4D03DFB21394155
:10EF600083C8C96D305FE43F0000E03FC4C30000C8
:10EF700040C3000022C30000182D4454FB21F93D7A
:10EF80003326A611460B113C2DE9FF4D21F0004818
:10EF900007460C46B8F1795F08DA0BF083F80028D1
:10EFA00001BF0020324904B0BDE8F08D3A46234647
:10EFB000104619460BF052F9054602462D480E46FA
:10EFC0000B460621784400F05DF82A4633460BF0E4
:10EFD00045F9DDE9022382468B46384621460BF08F
:10EFE0003DF904460F4652465B46284631460BF033
:10EFF00035F922463B460BF057FB07468A464FF051
:10F00000FF32284631460BF073FF1B4A90450ADA5F
:10F010003A4653460BF048FB04B00022BDE8F04DE1
:10F02000134B0BF04FBA154A4245A8BFA8F500157F
:10F030004FF00004B8BF124D22462B460BF034FBB4
:10F040000646884622462B46002009490BF02CFB39
:10F0500004460D463A465346304641460BF024FBE3
:10F0600004B022462B46BDE8F04D0BF02BBA000051
:10F070000000F03FF8C000003333D33F0000E93F09
:10F080000000D23F2DE9F0414F1E00EBC7010446BE
:10F09000D1E9000115461E4637F006020DD02A467A
:10F0A00033460BF0DBF87F1E04EBC703D3E90023E4
:10F0B0000AF0A8FD37F00602F1D1022F25D0042F67
:10F0C00013D0062F18BFBDE8F0812A4633460BF057
:10F0D000C5F8D4E90A230AF095FD2A4633460BF019
:10F0E000BDF8D4E908230AF08DFD2A4633460BF01B
:10F0F000B5F8D4E906230AF085FD2A4633460BF01D
:10F10000ADF8D4E904230AF07DFD2A4633460BF01E
:10F11000A5F8D4E902230AF075FD2A4633460BF020
:10F120009DF8D4E90023BDE8F0410AF06BBD000072
:10F130002DE9FF4D054621F0004084B00C46B0F1AA
:10F14000795F0BDA2846FFF701FD042808BF00F0BD
:10F1500075F8284608B02146BDE8F08D2A460B46D2
:10F1600010460BF07BF806460F462A4623460BF066
:10F1700075F8804626488A4632463B460521784443
:10F18000FFF780FF83461098029160B3214A224B1B
:10F19000404651460BF062F8CDE900015A46404620
:10F1A0005146029B0BF05AF882468846DDE906017B
:10F1B0004FF0FF320BF09CFE524643460BF074FAC0
:10F1C00032463B460BF04AF8DDE906230BF06CFAB9
:10F1D000DDE900230BF068FA08B02A462346BDE8B3
:10F1E000F04D0BF06FB90B465A46304639460BF0DE
:10F1F00035F8084A084B0AF005FD424653460BF025
:10F200002DF808B02A462346BDE8F04D0AF0FABCB6
:10F2100036C00000495555555555C5BF01220BF064
:10F2200067BE00221346104611460AF0A7BD40F201
:10F23000013200204FF0E0410BF05ABE024A00209C
:10F2400011070BF055BE000001FDFFFF10B504468D
:10F25000D1E9000100F002F8206010BDF8B50446C5
:10F260000D466A4604F0D6FB00987E3000900028D8
:10F270001FDC00221346204629460AF0D7FE18D08C
:10F28000002140F608004FF00000064620462946BF
:10F290000AF086FC044640F6080006EA00014FF03A
:10F2A000000034F0004004BF0220F9F73CFD204686
:10F2B000F8BD0098FF280DDB0220F9F734FD00228D
:10F2C0001346204629460BF0C7F88CBF04484FF080
:10F2D000FF40F8BD20462946BDE8F8400AF060BC72
:10F2E000000080FF10B504460A46D4E90003194621
:10F2F00005F0F8F9C4E9000110BD30380A2801D240
:10F300000120704700207047F0B5214C0F46C1B076
:10F31000217881423AD8FE216846F9F7B1F80646CD
:10F320006068002540B10AF06BFA022804D1C11EC2
:10F3300060680AF01DF901256423012215A1164811
:10F34000FDF74FFD3846F9F7FAFA82B264233946E1
:10F350001148FDF746FD6423022210A10E48FDF777
:10F3600040FDB2B24FF4FA7369460B48FDF739FD20
:10F37000642302220AA10848FDF733FD002D05D0C1
:10F3800000231A46194660680AF022F841B0F0BD21
:10F39000B40000205B000000FC8700205D2000001E
:10F3A0000D0A000070B5FCF733FC184C6168401A78
:10F3B000C82807D3FCF72CFC60604FF400511448B8
:10F3C000FCF719FC6078134D30B1FCF721FCA16803
:10F3D000401A642810D270BD207830B12846BDE8AC
:10F3E000704000220221FCF70DBCFCF711FCA16863
:10F3F000401AB0F5FA7FEED3FCF70AFCA06028466D
:10F40000BDE870400221FCF7F6BB00003801002087
:10F4100000100140000801403EB50024104800944F
:10F42000019402940D498460016004730475012500
:10F4300005614FF460214460C161FBF7A5FE08B18E
:10F44000FBF71EFECDE90045694605480294FBF72F
:10F4500019FE002801D0FBF713FE3EBD0024014039
:10F46000CC6600202DE9F04F704C012093B021793B
:10F47000002591B1617881B1E07800280FD06C4807
:10F48000007800280BD1FCF7C3FBA16851B1627969
:10F49000411A4AB14EF6602207E0A560607113B0D0
:10F4A000BDE8F08FA060FAE7624A9142F7D3A0600E
:10F4B0006571AA46E580DFF880B18BF800502570B1
:10F4C0005EA0FBF71FFD1325A046642001F0EBFBB7
:10F4D00098F8000088B35CA15748F9F7CEF90028E6
:10F4E000DDD15BA15448F9F7C8F930B345B358A151
:10F4F0005148F9F7C2F90A300446F9F7A7F90C9018
:10F500002C212046F9F7AFF906001DD02C21701CE4
:10F51000F9F7A9F9C0B12C21401CF9F7A4F90500AD
:10F5200013D02C21681CF9F79EF904000ED02C2171
:10F53000601CF9F798F9074609E0FFE76D1EC4D192
:10F5400046A005F0B5F9AAE70025002400271EB162
:10F55000701CF9F77BF900E00020CDF824A0CDF86D
:10F5600028A08146CDF82CA0CDF808A0CDF80CA09D
:10F57000CDF810A0CDF814A0A5B19CB197B1621B35
:10F580003E1B901E521E761E0A2803D8691C09A82D
:10F59000F9F73FFA701E0B2804D83246611C02A806
:10F5A000F9F737FAA8F806A08BF800A088F800A0B1
:10F5B000B9F1010F34D19DF8240080B39DF8080003
:10F5C00068B309A801F05AFB04460D4602A801F0F1
:10F5D00055FB10AB0EAACDE9002322462B4609F0BD
:10F5E00049FADDE91001CDE9000121A20C2109A8A9
:10F5F000F8F776FFDDE90E01CDE900011CA20D212F
:10F6000002A8F8F76DFF09AA02A91BA005F00CF9E2
:10F6100009AB02AA1C491D48FBF774FC3FE7FFE752
:10F620004A461BA00C9905F0FFF838E76C00002053
:10F630007E000020E0930400442E002041542B4320
:10F64000474E53494E4600002B4D5355423A000059
:10F650002B43474E53494E463A0000003E20475048
:10F66000533A2043474E53494E4620B3ACCAB100EB
:10F67000252E3666000000003E204750533A2025D4
:10F68000732C257300000000BC000020F8B20108B4
:10F690003E204750533A20CEB4B6A8CEBB28727550
:10F6A0006E3D2564206669783D2564292CCCF8B927
:10F6B000FD000000F0B5C1B050A005F0B5F866211E
:10F6C0005248F9F767FA132251A15048F9F7ABFAFB
:10F6D0004E48132253A11430F9F7A5FA4B481322D0
:10F6E00055A12830F9F79FFA4848132257A13C301A
:10F6F000F9F799FA45494FF4EB601322A1F850004D
:10F70000424855A15230F9F78EFA032441F2883667
:10F710004FF4FA6540F6B8372CE000BF02F01CF950
:10F7200001F09AFE811C08D0C11C08D068B12146A6
:10F730004DA005F0BDF830461AE051A000E057A0FA
:10F7400041B0BDE8F04005F0B3B801F031FD00284C
:10F7500029D0214658A005F0ABF82A465CA15DA04F
:10F7600000F0E8F92A465AA15EA000F0E3F9384615
:10F77000FCF72EF9201EA4F10104CFDC5C4C2278AA
:10F780005C4D29785CA005F039F82878002832D142
:10F79000207800282FD10A2008F058FC6420FCF7BC
:10F7A00017F9FFF7F7F95D49012048705CA005F0F3
:10F7B0003BF83220FCF70CF95C4A5D496846F8F7E3
:10F7C00079FE69465BA0FBF79DFB4FF496742046DB
:10F7D000FCF7FEF85848007800280CD0564B534AE6
:10F7E00056496846F8F766FE694652A0FBF78AFB61
:10F7F0002046FCF7EDF841B0F0BD00003E20344754
:10F800003A20B3F5CABCBBAF2E2E2E0044560020C2
:10F8100034366330383063333835633336353265E8
:10F82000000000003736363939303738383139334F
:10F83000373032363737000036616539363232625A
:10F8400037303334333236620000000035382E3121
:10F85000372E31342E3935002F696F742F6461745F
:10F86000612F646F776E2F003E2034473A20CDF829
:10F87000C2E7CAA7B0DC2CD6D8CAD42025640000C1
:10F880003E2034473A20CEDE2053494D2CD6D0D6E8
:10F89000B920344720B3F5CABCBBAF003E20344783
:10F8A0003A20CEDED0C5BAC52CD6D0D6B920344742
:10F8B00020B3F5CABCBBAF003E2034473A204D51BF
:10F8C000545420CAA7B0DC2CD6D8CAD42025640052
:10F8D0004F4B000041542B4D444953434F4E4E452E
:10F8E0004354000041542B4D495053544F50000095
:10F8F000800000207F0000203E2034473A20C1AC29
:10F90000BDD3CAA7B0DC2CCEDE2053494D3D2564C3
:10F910002C20CEDED0C5BAC53D2564006C00002089
:10F920003E2034473A20526561647900BC000020D3
:10F930009CB2010825730000F82A002060B301087A
:10F940002DE9FC4115460C4606004FF0FF3714D058
:10F950009CB1207888B119A13046F8F78EFF78B1B4
:10F960003346194A19491A48CDE90045F8F7A2FD6E
:10F97000174918A0FBF7C6FA1DE03846BDE8FC8120
:10F980000DB115A000E016A0CDE9004033460E4AA7
:10F9900015490F48F8F78EFD1E23032213A10C48CA
:10F9A00001F0BCFB18B112A004F082FFE5E7294684
:10F9B00018A004F039FF0020E0E7000070726F67C4
:10F9C0007265737300000000BC000020C8B301081A
:10F9D000102B002025730000747275650000000074
:10F9E00066616C736500000034B401084F4B000081
:10F9F0003E204F544120BDE1B9FBC9CFB1A8CAA7F1
:10FA0000B0DC28D6D8CAD4203320B4CECEDE204FE6
:10FA10004B2900003E204F544120BDE1B9FBD2D11B
:10FA2000C9CFB1A83A20737563636573733D2564CC
:10FA30000000000030B599B06846FEF77FFE18B9A7
:10FA40009DF81100032802D0012019B030BD9DF8A7
:10FA50001400F8B9BDF8080008B106F085FB0024D1
:10FA60004FEA0405FEF7A1FE09A8FEF767FE20B9DC
:10FA70009DF8380008B1012402E0322001F013F9AA
:10FA80006D1C032D02DA002CECD000E01CB10CA0A0
:10FA900004F0CAFE02E010A004F0B0FE182112A883
:10FAA000F9F79AF8BDF8083013A2182112A8F8F750
:10FAB00017FD012212A911A0FDF700FCC5E7000007
:10FAC0003E204F544120C8B7C8CFB1EAD6BED2D1EC
:10FAD000D0B4C8EB000000003E204F544120C8B70E
:10FAE000C8CFD0B4C8EBCAA7B0DC28D2D1D6D8CA08
:10FAF000D4203320B4CE290025750000696F742E00
:10FB00006F74612E636F6E6669726D2E706F7374A1
:10FB10000000000070B5064C002502E0257002F0E0
:10FB200017F920780028F9D1BDE87040FFF79ABC9A
:10FB30006C0000206423633292FBF3F2D3B2012203
:10FB400001F0ECBA1CB58246DDE904561F4690462A
:10FB5000894610A004F068FE03F0FAFC00210120A1
:10FB600008F0D8F80E4C01202070CDE900563B4635
:10FB700042464946504600F025F80020207009A072
:10FB800004F096FE112008F061FA6420FBF720FFD4
:10FB9000FFF700F83E204F54413A20BDF8C8EB0073
:10FBA0007E0000203E204F54413A20CAA7B0DCD648
:10FBB000D0D6B92CB8B4CEBBBBD6B8B4C1AACDF898
:10FBC000000000002DE9FF4F83B091468A4683462E
:10FBD00001F0C2FEC3A004F027FE05244FF47A769C
:10FBE00040F6B8352A46C3A1C3A0FFF7A3FF48B12A
:10FBF0002146C2A004F018FE304601F054F8641EFD
:10FC0000002CEFDC002C76D04FF4FA7001F04BF8AA
:10FC1000BCA004F009FE41F288363246B5A1B6A078
:10FC2000FFF788FF08B1BDA028E0C1A004F0FCFDEB
:10FC30003246B0A1C4A0FFF77DFF00285BD10324AA
:10FC40003246C3A1C4A0FFF775FF30B12146C5A05D
:10FC500004F0EAFD641E002CF2DC002CD3D02A460E
:10FC6000A4A1C3A0FFF766FF0028E7D1C2A004F05B
:10FC7000DBFD1E2001F01EFF28B1C5A007B0BDE8C6
:10FC8000F04F04F015BEC6A004F0CEFD2A4699A19F
:10FC9000C6A0FFF74FFF08B1CCA064E02A4695A1AB
:10FCA000CCA0FFF747FF08B1D0A05CE042F210778C
:10FCB0003A4690A1CFA0FFF73DFF08B1D1A052E096
:10FCC0002A468CA1D1A0FFF735FF08B1D3A04AE0A6
:10FCD000D4480090A0F11403A0F12802D2A1DB487F
:10FCE000F8F7E8FB4FF4FA64224682A1D748FFF701
:10FCF00021FF20B100E0F0E3D5A004F0D9FDC94810
:10FD0000D8A1283800F13C02B0F85030CF48F8F7BD
:10FD1000D1FB3A4677A1CD48FFF70CFF10B1D6A032
:10FD200004F0C6FD3A4673A1D9A0FFF703FF10B156
:10FD3000DCA004F0BDFDE1A004F076FDC34853460D
:10FD40005A46E3A19638CDF80090F8F7B3FBBF49C7
:10FD5000E3A0963904F068FD324666A1E3A0FFF700
:10FD6000E9FE28B1E4A007B0BDE8F04F04F05CBDA7
:10FD7000B64AE3A1963AA2F1FA00F8F79BFB41F2EA
:10FD800088325CA1E448FFF7D5FE08B1E3A00AE0A1
:10FD9000E4A004F049FD42F21072E5A1E8A0FFF7EB
:10FDA000C9FE50B1EAA004F03FFD07B02246BDE80D
:10FDB000F04F50A1E8A0FFF7BDBEA44800264FF4C5
:10FDC00020517830F8F7E6FEE6480021C180017046
:10FDD0004FF4FA730E22E4A1E748FDF702F832204F
:10FDE00000F061FF994843A17830323CF8F745FDB7
:10FDF00008B9002CF3DC9548E0A17830F8F73DFD18
:10FE00006FF02F0828B99148E0A17830F8F735FD58
:10FE1000B8B13A21F8F727FD98B100BF10F8011FDB
:10FE20002029FBD00929F9D042460178A1F13003FD
:10FE3000092B06D806EB860302EB4303CE18401CC1
:10FE4000F3E73146D5A004F0EFFCD7A004F0ECFCBA
:10FE5000DFA004F0E9FC3146E6A004F0E5FCD2A006
:10FE600004F0E2FCEDA004F0DFFC4FF4802001463A
:10FE7000FEF763FBF0A004F0D7FC4FF0FF300190D9
:10FE80004FF00009000C0090CB464A46F0A00699BE
:10FE9000FFF756FDF4A004F0C7FCAA465946F6A0A9
:10FEA00004F0C2FC5A46F8A19B48F8F703FB5446FD
:10FEB000524610A19848FFF73DFE08B1F8A00CE0AB
:10FEC0000BF6FF32F9A19448F8F7F4FA224609A19B
:10FED0009148FFF72FFE18B1FBA004F0A5FC0DE33D
:10FEE000FAE100003E204F54413A20CDF8C2E72EFF
:10FEF0002E2E00004F4B0000415400003E20415484
:10FF0000202564003E204F54413A20B5DAB6FEB4B5
:10FF1000CE20415420B2E2CAD40000003E20B5DA1F
:10FF2000B6FEB4CE20415420CAA7B0DC00000000C9
:10FF30003E204F54413A20B5DAB6FEB4CE204154AB
:10FF400020B3C9B9A60000004154453000000000AC
:10FF5000524541445900000041542B4350494E3F03
:10FF6000000000003E2053494D20256400000000A1
:10FF700041542B43535100003E204F54413A20B589
:10FF8000C8B4FDCDF8C2E7B8BDD7C52E2E2E0000EF
:10FF90003E204F54413A20B8BDD7C5B3ACCAB100DA
:10FFA0003E2053415042522E2E2E000041542B53DE
:10FFB000415042523D332C312C22434F4E54595024
:10FFC00045222C2247505253220000003E2053313C
:10FFD0000000000041542B53415042523D332C311C
:10FFE0002C2241504E222C22220000003E2053326F
:10FFF0000000000041542B53415042523D312C31FE
:020000040801F1
:10000000000000003E2053330000000041542B53F9
:10001000415042523D322C31000000003E2053340A
:10002000000000006C56002041542B4D434F4E46BB
:1000300049473D222573222C222573222C22257329
:10004000222C302C302C302C30000000CC2D002005
:100050003E204F54413A204D434F4E46494720CA17
:10006000A7B0DC0041542B4D495053544152543DEC
:10007000222573222C2564003E204F54413A204D06
:100080004950535441525420CAA7B0DC000000002C
:1000900041542B4D434F4E4E4543543D312C363049
:1000A000000000003E204F54413A204D434F4E4E39
:1000B00045435420CAA7B0DC000000003E204F5446
:1000C000413A204D51545420BECDD0F700000000DD
:1000D000687474703A2F2F25733A256425730000D5
:1000E0003E20485454503A202573000041542B4878
:1000F000545450494E4954003E20494E4954000042
:1001000041542B48545450504152413D2255524C79
:10011000222C2225732200003C2C00203E20555228
:100120004C0000003E20484541442E2E2E00000089
:100130002B48545450414354494F4E3A000000005C
:1001400041542B48545450414354494F4E3D320082
:100150003E2048454144000041542B4854545054DB
:1001600045524D006C00002041542B4854545048D7
:100170004541440D0A0000007C880020436F6E74E6
:10018000656E742D4C656E6774683A00636F6E74AB
:10019000656E742D6C656E6774683A003E20B4F32A
:1001A000D0A13D25644200002A2A2A2A2A2A2A2A86
:1001B0002A2A2A2A2A2A2A2A2A2A2A2A2A2A2A2A9F
:1001C0002A2A2A2A2A2A2A2A2A2A2A2A2A2A0000E3
:1001D0002A20204F544120C9FDBCB6BFAACABC206A
:1001E000202020202020202020202020202020200F
:1001F000202A00002A2020B4F3D0A13A2025642030
:10020000D7D6BDDA2020202020202020202020202A
:1002100020202020202020202A0000003E20D5FD84
:10022000D4DAB2C1B3FD2057323551363420D0C2B2
:10023000B2DBCEBB2E2E2E003E2057323551363447
:1002400020D0C2B2DBCEBBB2C1B3FDCDEAB3C90090
:10025000696F742E6F74612E70726F67726573733D
:100260002E706F73740000005BCFC2D4D85D20BFC6
:10027000AACABC203E3E3E003E20444C20C6ABD223
:10028000C63D25640000000041542B485454505092
:100290004152413D22425245414B222C25640000EF
:1002A0003E2042524B20CAA7B0DC000041542B48EC
:1002B000545450504152413D22425245414B454ECB
:1002C00044222C25640000003E2042524B454E44FF
:1002D00020CAA7B0DC00000041F28832AFF2B011B2
:1002E000B5A0FFF727FC10B15946B7A094E0B94874
:1002F000C08802904FF4FA730E22B7A1BA48FCF7F7
:1003000070FD00256C1EFBF783FC074677E0002C90
:100310006DDAB04A029830E0B4490B5C2B2B2BD13C
:100320000B1893F801C0BCF1480F25D193F802C017
:10033000BCF1540F20D193F803C0BCF1540F1BD172
:1003400093F804C0BCF1500F16D193F805C0BCF16E
:10035000520F11D193F806C0BCF1450F0CD193F8A0
:1003600007C0BCF1410F07D193F808C0BCF1440F9E
:1003700002D15B7A3A2B05D0401CD1880B398842D8
:10038000CADB39E000230A3000E0401CB2F806C0A6
:1003900060450FDA11F800C0BCF1200FF5D0BCF1B8
:1003A000090FF2D006E000BF03EB830308EB430321
:1003B0006344401CB2F806C0604509DA11F800C079
:1003C000BCF1300F04D3BCF1390FEDD900E0401C73
:1003D000B2F806C0604504DA11F800C0BCF10A0F9B
:1003E000F5D1D188884207DA1D46441C04E07948DB
:1003F000C088001BA84209DA142000F054FCFBF767
:1004000007FCC11B42F21070814280D3002D01DD38
:10041000002C04DA594676A004F006FA6EE06D4826
:10042000C088001BA84208DA6A48C0882B46021B15
:10043000594673A004F03CFA14E06C482A460119AE
:100440000BF580200F460290FEF74CFB39462A46FA
:100450000298FEF707FB08B1002713E0594674A085
:1004600004F0CCF95246AFF27451AFF21430FFF7FA
:1004700061FB95E05D48E119415C009801F038FCB2
:100480007F1C0090AF42F5DB09EB0500AB448146D1
:10049000002E23DD642109FB01F090FBF6F4642CAF
:1004A00000DD642433464A4621466BA004F0BCF9C3
:1004B0000A2094FBF0F2019991FBF0F0824212DDE8
:1004C00022460194AFF278200699FFF739FA4FF4EB
:1004D00000516648FBF78FFB05E069E002462946BC
:1004E00063A004F0A1F9B5F5406F07DB002E01DD34
:1004F000B14503DABBF5603FFFF4D0AC5446524639
:10050000AFF21061AFF2B030FFF714FB5FEA090001
:1005100011D0002E00DC064658A0119A009904F074
:1005200083F9119848B111990098884205D05DA0CF
:1005300004F064F934E063A030E0314664A004F0D4
:1005400073F931464FF48020FDF796FF28B364A07D
:1005500004F06AF9AFF2B03004F066F966A004F076
:1005600063F96DA004F060F9AFF2C43004F05CF9F7
:10057000012273A00699FFF7E3F9204600F093FBF0
:10058000DDE910023146FEF72DF9082007F05EFD87
:10059000642000F088FBFEF7FDFA6EA004F044F939
:1005A000069907B00022BDE8F04F65A0FFF7C8B973
:1005B00007B0BDE8F08F000041542B48545450411F
:1005C0004354494F4E3D30003E2041435420402586
:1005D000640000006C00002041542B4854545052D9
:1005E0004541440D0A0000007C880020442E002074
:1005F0003E20CEDECAFDBEDD2040256400000000A6
:100600003E20444C20CAFDBEDDBFE92040256420C9
:10061000B2BBCDEAD5FB3A20D2D1CAD52025642F72
:10062000256420D7D6BDDA2CD6D8CAD42E2E2E00DB
:100630003E2057323551363420D0A3D1E9CAA7B075
:10064000DC206F66667365743D25642CD6D0D6B900
:10065000204F5441000000003E205B2533642525D7
:100660005D2025642F256442000000000010014039
:100670003E202B2564423D25644200003E20573237
:10068000355136342043524331363D3078253034AD
:10069000582028B7FECEF1C6F73D307825303458C3
:1006A000290000003E205732355136342043524352
:1006B000313620B2BBC6A5C5E421D6D0D6B9204F6D
:1006C000544100003E20CEDECAFDBEDD0000000029
:1006D0003E3E3E20D0A3D1E9202564422E2E2E009E
:1006E0005B204F4B205D20B9CCBCFED0A3D1E9CD1F
:1006F000A8B9FD21000000002A20204F544120CF3E
:10070000C2D4D8CDEAB3C921202020202020202027
:10071000202020202A0000002A2020D5FDD4DAD66F
:10072000D8C6F4BDF8C8EB20426F6F744C6F61649B
:1007300065722E2E2E20202020202020202A00002E
:10074000696F742E6F74612E726573756C742E7080
:100750006F7374005BCAA7B0DC5D000010B533A0F6
:1007600004F062F832A004F05FF83AA13BA004F074
:100770005BF843A004F058F803F05EFE01F0FAFBCA
:1007800004F062F8474C474947A034F8642F3C31E5
:1007900004F04AF8434948A004F046F841494AA009
:1007A000143104F041F8218A4BA004F03DF8FDF724
:1007B0000BFF07F055FB07F02DF902F027FF03F0C0
:1007C0006FFB02F0CFFB03F0C7FFFEF725FE07F03B
:1007D00085FE03F0FDFB05F0D5FA43484FF001011B
:1007E00000780028084603D005F05CFB3FA002E03B
:1007F00005F058FB41A005F05DFB0221084605F01D
:1008000051FB42A005F056FB43A004F00DF8FCF7A5
:10081000F9FCFDF735FDFDF707FEFDF7F1FC00F0F3
:10082000D7FABDE8104000F01FBB00000000000038
:100830002A202A202A202A202A202A202A202A2068
:100840002A202A202A202A202A202A202A202A2058
:100850002A202A00312E352E360000002A202020A2
:1008600020202020B0E6B1BE3A2025732028525423
:100870004F532920202020202020202A0000000083
:100880002A202A202A202A202A202A202A20202022
:1008900042792048656C65692020202A202A202A78
:1008A000202A0000BC0000203E20B7FECEF1C6F793
:1008B0003A2025733A2564003E20BFCDBBA7B6CBB6
:1008C00049443A20257300003E20D3C3BBA7C3FB95
:1008D0003A202573000000003E20B0E6B1BED0F201
:1008E000BAC53A202575000064010020D6C7C4DCD3
:1008F000CBAEB2FACDB6C1CFBBFA0000BCCCB5E7E7
:10090000C6F7BFD8D6C6D6D5B6CB000056312E35E1
:100910002E362052544F53003E204F4C45443A202F
:10092000B3F5CABCBBAFCDEAB3C9000010B5FBF745
:100930006FF9074CA169401AB0F5FA7F07D3FBF7AE
:1009400067F9A061BDE81040002005F023B810BD94
:10095000940100201CB503F093FF07F0DBFCFCF7CB
:1009600007FC00240320CDE90004020223460EA167
:100970000E4808F013FF0220CDE900040502002311
:100980002A460BA10B4808F009FF0120CDE900041D
:1009900000232A4608A1094808F000FF07F0EAFFF3
:1009A00007A003F02BFFFEE76E65740055530108A6
:1009B00061707000D9090108737973004D830108D3
:1009C0003E2052544F533A20B5F7B6C8C6F7C6F486
:1009D000B6AFCAA7B0DC00004D4D4E4C4E4E0127BD
:1009E0004FF00008207928B9287818B12771FBF753
:1009F0000FF96061287878B1607968B9677107F09C
:100A0000D5F807F0BFF945A0FDF762F845A003F05F
:100A10000BFFFBF7FDF8E0602078002826D128784E
:100A2000002823D04848007800281FD0FBF7F0F8B2
:100A3000E168401A42F22831884217D9607828B11B
:100A4000A078002812D1A77040A00DE02770FCF715
:100A5000E9FC002807DAE770FBF7DAF8206146A026
:100A600003F026FF02E04CA003F0DEFEE078A8B120
:100A7000287898B1FBF7CCF82169401A47F2305139
:100A800088420BD9FBF7C4F82061FCF7CBFC0028A7
:100A900004DB84F803804DA003F0C6FE207808BB79
:100AA0002079F8B1FBF7B4F86169401A4EF660217D
:100AB000884217D94BA003F0FBFE092007F0C6FAC5
:100AC000FDF71EFE6420FAF783FFBFF34F8F5248F5
:100AD0000168524A01F4E06111430160BFF34F8F96
:100AE00000BFFDE706F00EFF307850B1FBF790F83D
:100AF0004B490968401A642803D986F8008007F03A
:100B000041F902F0CFFA0A2007F094FE6AE70000EC
:100B10007C00002094010020A8000020312E352EFA
:100B2000360000003E204D61696E3A204D5154540C
:100B300020526561647920BAF3CAD7B4CED7B4CC59
:100B4000ACC9CFB1A80000007D0000203E204F546A
:100B50004120C8B7C8CFCCF8B9FDA3A8C4A3C4E24C
:100B6000CAA7B0DCA3ACD3C3D3DABBD8CDCBB2E237
:100B7000CAD4A3A9000000003E204F544120C8B7AA
:100B8000C8CFCDA8D6AACEB4CBCDB4EFA3ACC9D430
:100B9000BAF3D6D8CAD400003E204F544120D2D157
:100BA000C8B7C8CFA3A84D51545420526561647989
:100BB000202B20CAD7B4CEB7A2B2BCB3C9B9A620E5
:100BC0002B20D1D3B3D93973A3A900003E204F54B1
:100BD0004120C8B7C8CFCDA8D6AAD6D8CAD4B3C9E1
:100BE000B9A600003E204F544120BDA1BFB5B3AC13
:100BF000CAB13A204D51545420526561647920B5F0
:100C0000AB203120B7D6D6D3C4DACEDE204D505536
:100C100042A3ACB8B4CEBB000CED00E00400FA0572
:100C2000AC00002070B58AB00646002009900D4641
:100C300009A802F0CFFE002801DA002405E00A210D
:100C4000401C90FBF1F201FB1204FF2224216846B4
:100C5000F7F798FF0848009009988DF80860401C45
:100C60000190FF208DF80900E0B26946039506F077
:100C700081FB0AB070BD00004C54535230B583B0B4
:100C80000446F8F74BF805460020CDE9000002467F
:100C900021466846F8F708FC2846F8F744F8DDE9ED
:100CA000000103B030BD10B5044608F0A9FD0228CC
:100CB00004D014E0142007F0BDFD143C142CF9D22C
:100CC000002C15D02046BDE8104007F0B3BD14201D
:100CD000FAF77EFEFCF7F6F8FFF728FE143C142C1A
:100CE000F5D2002C04D02046BDE81040FAF770BEC3
:100CF00010BD00002DE9F04190B01546884606462B
:100D000003461FA240216846F7F7EAFB4FEA0004BA
:100D1000FDF74EFA0028FBD1A2B24FF4FA736946F0
:100D20001948FCF75EF8322095FBF0F44FF0FF37DE
:100D30001EE0322000F078F8FDF73AFA050017D0EF
:100D40004146F7F79AFD38B1294610A003F06CFD33
:100D5000002010B0BDE8F08110A12846F7F78DFD06
:100D600030B129460FA000BF03F0A2FD3846F0E7DE
:100D7000201EA4F10104DCDC314610A0F4E70000E1
:100D800025730D0A00000000FC8700203E20424C25
:100D9000452041543A202573000000004552524F2F
:100DA000520000003E20424C4520415420D3A6B4BE
:100DB000F0B4EDCEF33A2025730000003E20424C03
:100DC0004520415420B3ACCAB13A2025730000003D
:100DD00030B585B000241248009401940294039425
:100DE000816941F00801816180690E4D00F00800C1
:100DF0000122049011462846FAF704FF01200090D2
:100E00001120CDE901040220039069462846FAF733
:100E1000F1FD012211462846FAF7F4FE05B030BD77
:100E200000100240000C014010B5044605E06420AB
:100E3000FAF7CEFDFCF746F8643C642CF7D2002CA0
:100E400004D02046BDE81040FAF7C2BD10BD000036
:100E500010B5012203A1842001F0C6F9BDE81040BD
:100E600000F002B80000000030B593B01C210CA8BF
:100E7000F7F7B2FE1A220CA9842001F06BF80020CB
:100E80008DF8490049A10CA8F7F7F8FE60B3484C6B
:100E9000002201212046FAF7B5FE40F24C40FFF750
:100EA000C3FF012211462046FAF7ACFE4FF416703C
:100EB000FFF7BAFFFDF77CF90028FBD14FF4FA7376
:100EC0000C223CA13E48FBF78CFF1D2440F2DC5570
:100ED0003220FFF7A9FFFDF76BF9211EA4F10104F1
:100EE00008DD0028F4D006E030A136A003F09CFC19
:100EF00013B030BD40B12DA1F7F7BFFC20B12BA13D
:100F000038A003F091FC15E0002428A33DA2302175
:100F10006846F7F7E5FA2A463DA16846FFF7EAFE7C
:100F2000641C032C02DA0028EFD109E040B139A09B
:100F300003F0BEFC2A4636A141A0FFF7DBFED7E74F
:100F400041A34AA230216846F7F7CAFA2C462A463E
:100F50002FA16846FFF7CEFE47A350A23021684676
:100F6000F7F7BEFA22462AA16846FFF7C3FE42A35E
:100F70004DA230216846F7F7B3FA224624A168460D
:100F8000FFF7B8FE4BA003F04FFC0025224620A13E
:100F900050A0FFF7AFFE10B16D1C022DF6DB04224E
:100FA00002A1842001F020F9A2E700004274310080
:100FB000000C014041542B4E414D453D3F0D0A0070
:100FC000FC8700203E20424C453A20C5E4D6C3D2DF
:100FD000D1BBBAB4E628257329A3ACCCF8B9FDC9B6
:100FE000E8D6C3003E20424C453A20C3FBB3C6D2EC
:100FF000D1CAC7202573A3ACCEDED0E8C9E8D6C3DA
:101000000000000041542B4E414D453D257300002A
:101010004F4B00003E20424C453A20C9E8D6C3C39E
:10102000FBB3C6CAA7B0DCA3A8C4A3BFE9CEB4BDB6
:10103000D3BBF2D3A6B4F0D2ECB3A3A3A9000000B3
:1010400041542B54533D31003030303066666530AA
:10105000303030303130303038303030303038307F
:1010600035663962333466620000000041542B5506
:10107000554944533D257300303030306666653144
:10108000303030303130303038303030303038304F
:1010900035663962333466620000000041542B55D6
:1010A000554944523D25730041542B5555494457E9
:1010B0003D2573003E20424C453A20C3FBB3C6D3C6
:1010C000EB205555494420D2D1C9E8D6C3CDEAB367
:1010D000C900000041542B5245424F4F543D31004E
:1010E0000168426811448268C0681044084470472F
:1010F000084810B50168084A914208D1FFF7F0FF8F
:10110000044910310968884201D1012010BD002036
:1011100010BD000000BF0020524853522DE9F05F7F
:101120000127994616468B4682460025DFF86080E7
:1011300027E000BFA8F8065016490D7088F8005047
:10114000514615A0F9F7DEFE4C460FE06420FFF78C
:10115000AAFD98F80010404641B1057059460D4867
:10116000F7F78BFB10B1002724B108E0641E14F0E0
:10117000FF04EBD15246314608A003F099FB761EDE
:10118000F6B20EB1002FD5D13846BDE8F09F000071
:101190006C000020442E0020257300003E204154A6
:1011A00020B3ACCAB1205B7225755D3A202573006F
:1011B0002DE9F0415449A0B00520087053A003F078
:1011C00033FB56480090A0F11403A0F1280254A16B
:1011D00001A8F7F76FF90F2301225AA101A8FFF721
:1011E0009DFF4FF0FF3800283AD14C4856A12838CF
:1011F00000F13C02B0F8503001A8F7F75BF93C234E
:10120000012250A101A8FFF789FF002828D153A18E
:101210005548F7F732FB1D25544C0026C8B92670F7
:101220002F466420FFF73FFD207800281CD0267051
:101230004AA14D48F7F721FB20B94DA14A48F7F7DD
:101240001CFB88B1002F04DA474AE1884CA003F068
:101250002FFB3C2301223BA152A0FFF75FFF30B1DF
:10126000404620B0BDE8F0817F1EDAD5ECE752A100
:101270003D48F7F702FB002823D138A13A48F7F799
:10128000FCFAF0B926706420FFF70DFD2078A8B1B4
:10129000267049A13448F7F7F0FA48B92FA132482F
:1012A000F7F7EBFA20B947A12F48F7F7E6FA28B18C
:1012B000002D06DA2C4AE18845A021E06D1EE2D51A
:1012C000F8E7164B4BA1283B03F1520201A8F7F7B0
:1012D000F1F8322301224CA101A8FFF71FFF38B11A
:1012E00018A12148F7F7C9FA38B149A003F09CFAD0
:1012F0004DA003F099FA0020B3E71B4AE1884EA005
:1013000003F0D6FAACE70000900000203E203447FE
:101310003A204D5154542E2E2E0000006C560020C1
:1013200041542B4D434F4E4649473D222573222CB5
:10133000222573222C222573222C302C302C302C89
:10134000300000004F4B000041542B4D4950535486
:101350004152543D222573222C256400434F4E4EAA
:10136000454354204F4B0000442E00206C000020C9
:101370002B4D495043414C4C4241434B000000002F
:101380003E2034473A2054435020C1ACBDD3B3ACC7
:10139000CAB12C6C6173745B25645D3A20252E38CC
:1013A0003073000041542B4D434F4E4E4543543D46
:1013B000312C363000000000434F4E4E41434B204D
:1013C0004F4B00002B4D434F4E4E45435445440078
:1013D0003E2034473A204D51545420C1ACBDD3B3C4
:1013E000ACCAB12C6C6173745B25645D3A20252E08
:1013F0003830730041542B4D5355423D22257325FF
:1014000073222C300000000053554241434B000032
:101410003E2034473A204D53554220D2D1BDD3CA45
:10142000DC284F4B290000003E2034473A204D5124
:101430005454204F4B0000003E2034473A204D5377
:10144000554220CAA7B0DC2C627566665B25645DD8
:101450003A20252E383073002DE9F05FA8A003F064
:10146000E3F9AB4C022020704FF4E130FCF77EFF33
:1014700005230122A7A1A8A0FFF750FE4FF0FF3BD4
:101480004FF4612558B12846FCF770FF142303225E
:10149000A0A1A1A0FFF742FE00286FD11EE01E23ED
:1014A00001229CA19DA0FFF739FE0028F5D1284616
:1014B000FCF75CFF6420FFF7F6FB1423012295A1E3
:1014C0009AA0FFF72BFE1423032292A192A0FFF70C
:1014D00025FE0028E1D197A003F0A6F914230322EA
:1014E0008CA18DA0FFF71AFE0028D6D10A23012275
:1014F00088A196A0FFF712FE0028CED10320A146B6
:1015000020700227DFF84CA2934C4FF00108002511
:10151000E5808AF80050257090A0F9F7F3FC1E26AC
:101520002DE06420FFF7BFFB2078002827D025702E
:101530008DA18848F7F7A1F928BB8DA18548F7F759
:101540009CF970B98CA18348F7F797F948B98CA139
:101550008048F7F792F920B98EA17E48F7F78DF908
:1015600068B190A003F0A4F9062189F8001093490E
:1015700081F800806FF00100BDE8F09F9CE0761ECE
:1015800016F0FF06CDD178A17248F7F776F938B991
:101590004FF47A70FAF71CFA381EA7F10107B7DC8E
:1015A00071A16C48F7F769F948B1854F0A23012208
:1015B0003D7084A185A0FFF7B1FD20B11CE086A09D
:1015C00003F076F978E07FA16248F7F756F998B111
:1015D000C11D00E0491C08782028FBD0002600E04F
:1015E000761C885D3038092801D8132EF8DB324686
:1015F0007348F7F70EFABD55387820B170497BA0D3
:1016000003F012F902E07DA003F052F91E2000F071
:1016100051FA002850D1DFF8FC9189F800500F23CF
:1016200001227DA17EA0FFF779FD58B17EA003F0D5
:101630003FF91423012237A182A0FFF76FFD002894
:101640003AD12BE087A14348F7F717F958B1801D2D
:10165000F7F7FCF806461F2806D8642070431F21C0
:1016600090FBF1F701E063260027324639467FA060
:1016700003F0DAF8632E01D0022E08DA394682A090
:1016800003F0BCF889F800806FF0020074E7142FB3
:10169000CFDA394681A003F00BF9CAE714230122FF
:1016A0001CA183A0FFF73AFD30B99623032219A1AC
:1016B00085A0FFF733FD08B158465DE7E570207956
:1016C000C0B11E23012213A183A0FFF727FD08B19B
:1016D00085A007E01E2301220EA18CA0FFF71EFDAE
:1016E00018B18FA003F0E4F804E084F8038091A01F
:1016F00003F09AF894A003F097F800203CE700006C
:101700003E2034473A20CDF8C2E72E2E2E000000AE
:10171000900000204F4B00004154000041542B49E1
:1017200050523D3932313630300000004154265796
:10173000000000003E2034473A20B2A8CCD8C2CAEC
:10174000202D3E20393231363030000041544530B2
:1017500000000000442E00206C00002041542B4368
:1017600050494E3F000000005245414459000000DE
:101770004E4F2053494D00004E4F53494D0000003D
:1017800053494D204E4F5420494E534552544544E1
:10179000000000002B434D45204552524F523A2045
:1017A000313000003E2034473A20CEB4BCECB2E2E7
:1017B000B5BD2053494D20BFA80000007F00002088
:1017C000F82A00202B49434349443A0041542B490D
:1017D00043434944000000003E2034473A20534927
:1017E0004D20CEB4BECDD0F7000000003E203447DF
:1017F0003A20494343494420257300003E203447A2
:101800003A20494343494420B6C1C8A1CAA7B0DC25
:1018100000000000800000202B4353513A000000DC
:1018200041542B43535100003E2034473A20435348
:101830005120B2E9D1AFCAA7B0DC2CBCCCD0F8D6CD
:10184000B4D0D00041542B53415042523D332C313F
:101850002C22434F4E54595045222C22475052536C
:10186000220000002B4353513A2000003E20344711
:101870003A20D0C5BAC52025642525202872737367
:10188000693D2564290000003E2034473A20CEDE21
:10189000D0C5BAC520282564252529003E20344717
:1018A0003A20D0C5BAC5C8F52028256425252900C9
:1018B00041542B53415042523D332C312C22415044
:1018C0004E222C222200000041542B534150425200
:1018D0003D312C310000000041542B43474E535002
:1018E00057523D31000000003E2034473A20474E19
:1018F000535320C9CFB5E7CAA7B0DC28C4A3BFE9BA
:10190000CEDE20474E53533F2900000041542B4365
:10191000474E534149443D33312C312C312C310059
:101920003E2034473A20474E535320B8A8D6FACA2F
:10193000A7B0DC003E2034473A20474E535320D214
:10194000D1BFAAC6F40000003E2034473A20CDF8AB
:10195000C2E7204F4B0000002DE9F041454886B01A
:101960000126067044A002F05FFF2720FAF7F8F97D
:101970000D20FAF7F5F94448FAF735FE4348016BB4
:1019800021F001010163016BC907FCD14FF48071A3
:1019900041603D4D00242868016841680491016858
:1019A00041680491016841680491016841680491AB
:1019B00001684068364F0490FC80DFF8D88088F8D2
:1019C00000403C7034480294816941F00401816117
:1019D0008069694600F0040004901020CDE90006FB
:1019E00002202E4E03903046FAF704F8012210210F
:1019F0003046FAF707F94FF47A70F9F7E9FF002259
:101A000010213046FAF7FEF85FF00006FBF75AFAAD
:101A10006420F9F7DDFF761C282EF7DBFC8088F8C0
:101A200000403C7028680168416804910168416881
:101A3000049101684168049101684168049101685A
:101A4000406804904FF4005215490F48FBF782F8A4
:101A50002868C16841F01001C1600D20FAF791F9C2
:101A60002720FAF78EF90FA002F0DEFE06B0BDE8DF
:101A7000F0810000900000203E2034473A20B8B4A6
:101A8000CEBB2E2E2E0000007C88002000000240DD
:101A90006C000020442E002000100240000801408D
:101AA000FC6600203E2034473A20B8B4CEBBCDEAD5
:101AB000B3C900002DE9F04782460025A946DFF8AA
:101AC000888000EB8A0736E04C46A8F806901F494C
:101AD00081F8009088F800901D49042008701DA02E
:101AE000F9F710FAA1461E26444618E06420FFF7D5
:101AF000DAF8207898B184F8009019A11348F6F725
:101B0000BCFE08B119A005E01DA11048F6F7B5FE0E
:101B100028B120A002F088FE0020BDE8F087761EE4
:101B200016F0FF06E2D10A201E3595FBF0F1524671
:101B30001DA002F079FEB5EB470FC5DB22A002F035
:101B4000B7FE4FF0FF30E8E76C000020442E002085
:101B50009000002041542B43474154543F00000063
:101B60002B43474154543A20310000003E20344773
:101B70003A20434741545420D2D1B8BDD7C50000C4
:101B80002B434745563A204D452050444E20414373
:101B9000542031003E2034473A2050444E20D2D1C8
:101BA000BCA4BBEE000000003E2034473A2043476F
:101BB00041545420CEB4B8BDD7C52CD6D8CAD420F1
:101BC00025642F25640000003E2034473A20434717
:101BD00041545420B8BDD7C5B3ACCAB10000000011
:101BE00010B50FE0A3F14104192C01D82033DBB26A
:101BF000A2F14104192C01D82032D2B2934209D16A
:101C0000401C491C03781BB10A78002AEAD101E084
:101C1000087808B1002010BD012010BD2DE9F04169
:101C20000A4C054620880026094F854201D32680AC
:101C300008E020887919421B0548F6F72FFF208815
:101C4000401B208020883E54BDE8F08172000020B7
:101C5000442E002000B5244B21F0004287B09A4268
:101C6000DCBF0022134629DD204B9A4208D140B93F
:101C70004FF00100F7F757F8FDF7D3FA07B000BDB2
:101C800003DBFDF7CBFA07B000BD02AAFCF7B8FFF3
:101C900010F0030104BF0DF1080C9CE80F000DD0FB
:101CA000012001290ED0022914D00DF1080C00905A
:101CB0009CE80F00FDF73CFA07B000BDFDF764F9A2
:101CC00007B000BD0DF1080C00909CE80F00FDF777
:101CD0002FFA05E00DF1080C9CE80F00FDF754F910
:101CE00007B081F0004100BDFB21E93F0000F07F1B
:101CF000484000214AF20102C30702D082EA5000A4
:101D000000E04008491C0829F6DB704710B54FF089
:101D1000E0218A690C4B0D4C1B68B3FBF4F3434381
:101D20009A4209D288699042FCD8981A4A698B690C
:101D3000121A9A42FAD810BDD01A8B699342FAD27D
:101D40008B698342F9D210BD6800002040420F0029
:101D50002DE9F05F3F4840A18246F6F78EFD002452
:101D6000DFF8F080DFF8F8902746254638B13AA131
:101D7000801DF6F782FD040026D0012709E039A175
:101D80005046F6F77AFD20B938A15046F6F775FDB2
:101D9000A8B100260CB126782570514636A002F075
:101DA00043FD32A15046F6F768FD4FF47A7B80B1CF
:101DB00004B1267034A002F021FD062020E038A1F5
:101DC0005046F6F75AFD08B10026E6E7A9F8065096
:101DD0003CE024A15046F6F750FD30B104B1267026
:101DE00032A002F00BFD04200AE02DA15046F6F7C8
:101DF00044FD60B104B1267034A002F0FFFC0F2056
:101E000006F024F95846F9F7E3FDFCF7C3FE504607
:101E100003F0E8F804B12670002FD7D0002CD5D0FD
:101E2000B9F80610A4EB0A004E460F1A002F0CDD7D
:101E30003A4621460748F6F731FEF780F18801203F
:101E400008F801503070BDE8F09FF58088F8005028
:101E5000F9E70000442E00202B4D5355423A000074
:101E60006C000020434C4F53454400002B4E4F2044
:101E700053657276696365003E204D5154543A2093
:101E8000252E3230307300003E20344720D2ECB390
:101E9000A33A20CEDEB7FECEF12CB8B4CEBB000004
:101EA000626F6F742E726F6D000000003E20344729
:101EB00020D2ECB3A33A204D5154542F5443502018
:101EC000D2D1B6CFBFAA2CB8B4CEBB003E20344787
:101ED00020D2ECB3A33A20C4A3BFE9D6D8C6F428D5
:101EE000626F6F742E726F6D292CB8B4CEBB000078
:101EF0002DE9F047DFF85480174689460646002250
:101F000080214046F9F77EFE0122D1031048F9F7FF
:101F100079FE02253146484602F0D0FB5FF000040E
:101F200017F8011B012004F073F8641CE4B2102CB4
:101F3000F6D3761C6D1EF6B215F0FF05EAD14046C9
:101F4000BDE8F04701228021F9F75CBE0010014096
:101F5000000C014070B5154606460C4606F0C8F95F
:101F60002A462146304602F0EBFC044606F0DCF936
:101F7000204670BD2DE9F04FA5249FB02146FA20E0
:101F800002F00EFDFA2002F0A3FC0246214649A011
:101F900002F04AFC78215048F6F71EFE78224E499E
:101FA0000020FFF7D7FF4C4C01464CA0B4F874302A
:101FB000226F02F039FC2046534D226F00F11401CC
:101FC00000F1280B00F13C0A00F150094FF4EB68D6
:101FD0001E91AA4220D14DA1F6F750FE00281BD138
:101FE0004FA11E98F6F74AFEB0B952A15846F6F72F
:101FF00045FE88B954A15046F6F740FE60B955A198
:102000004846F6F73BFE38B9B4F86400404503D1C2
:10201000B4F8741053A048E0206FB4F87470A8426C
:1020200001D1012600E0002678212B48F6F7D4FDE7
:1020300036A12948F6F75FFC39A11E98F6F75BFC3C
:102040003CA15846F6F757FC3FA15046F6F753FC23
:1020500040A14846F6F74FFCA4F8648006B9002773
:10206000A4F874700020C4F86600A4F86A0084F82C
:102070006C00256778221849683400F0B5F83FA055
:10208000A16802F0D1FB78216846F6F7A5FD782219
:1020900069460020FFF75EFF0146BDF874303FA09F
:1020A0001C9A02F0C1FBA18948A002F0BDFB1FB041
:1020B000BDE8F08F3E20454550524F4D20CCBDB27B
:1020C000E23A20D0B43D3078253032582C20B6C1C9
:1020D0003D30782530325800BC0000203E20454578
:1020E00050524F4D20B6C1C8A1206572723D256483
:1020F0002C204D616769633D3078253038582C209D
:102100005665723D25750000EFBEADDE3436633096
:1021100038306333383563333635326500000000BC
:102120003736363939303738383139333730323657
:102130003737000036616539363232623730333432
:10214000333236620000000035382E31372E3134FC
:102150002E3935002F696F742F646174612F646F9D
:10216000776E2F00454550524F4D20C5E4D6C3D35E
:10217000D0D0A72C205665723D2575003E204545E0
:1021800050524F4D20D0B4C8EBCDEAB3C92C204DEE
:10219000616769633D307825303858003E204545F9
:1021A00050524F4D20BBD8B6C1D0A3D1E9206572A3
:1021B000723D25642C204D616769633D3078253080
:1021C00038582C205665723D257500004545505203
:1021D0004F4D20C5E4D6C3D2D1D0DEB8B42C2056A2
:1021E00065723D25750000002DE9F04715468146D2
:1021F0008846002606F07CF81BE000BF09F00700C7
:10220000C0F10804AC4200D9ECB22246414648462F
:1022100002F0FEFB070004D0024649460DA002F082
:1022200047FB09EB04003E4300F0FF09281BA044D4
:1022300085B2002DE2D106F077F826B131460DA027
:1022400002F036FB02E013A002F0EEFA3046BDE8E1
:10225000F08700003E20454520D0B4C8EBCAA7B0A7
:10226000DC204025752C206572723D307825303297
:10227000580000003E20454550524F4D20D0B4C874
:10228000EBD7DC2041434B20B4EDCEF33D30782535
:10229000303258003E20454550524F4D20D0B4C8F2
:1022A000EBB3C9B9A60000000346002001F07F028D
:1022B000C909002901D042F080021A5400F101003E
:1022C000C0B2F3D17047000070B5124C92B02288B2
:1022D0006946402A02D2238800220BE040230022D4
:1022E0000D4DAD5CA5F120065E2E00D92E258D5436
:1022F000521C92B29A42F3D30022CA540BB10B463D
:1023000000E006A32288014606A002F0D1FA12B02E
:1023100070BD000072000020442E002028656D7002
:10232000747929003E205769466920BDD3CAD55B20
:1023300025735D206964783D25753A20257300007A
:102340002DE9F04388460A468146014699B045A0EA
:1023500002F06AFA002442F210764FF4FA6540F275
:10236000DC5708E0002C06DD44A002F0A1FA4FF48F
:102370007A70FEF798FC3A4645A146A000F068FC4A
:102380002A4643A146A000F063FC00285ED12A46FD
:102390003FA146A000F05CFC002857D14B4647A265
:1023A000602101A8CDF80080F6F79AF801A94AA0AB
:1023B000F8F732FE00F0D6FB314648A000F024FDCD
:1023C00030B148A002F074FA4CA0FFF77DFF3DE069
:1023D0004D494EA002F028FA29462DA000F014FD28
:1023E0004FF49670FEF75FFC51A0F8F715FE00F071
:1023F000B9FB314651A000F007FDC0B150A002F07A
:1024000057FA55A0FFF760FF55A0F8F705FE00F05A
:10241000A9FB29461EA000F0F7FC70B151A002F004
:1024200047FA00F09FFB002019B0BDE8F08300F0F0
:1024300099FB55A002F0F8F9F5E72A4658A15BA0F0
:1024400000F006FC58B15CA002F032FA641C022CC9
:1024500088DB63A002F02CFA4FF0FF30E4E766A0BF
:10246000F2E700003E20576946693A20BDF8C8EB04
:10247000CDB8B4AB2025733A257500003E205769CE
:1024800046693A20CDB8B4ABD6D8CAD40000000013
:102490004F4B000041542B434950434C4F53450090
:1024A00041542B4349504D55583D300041542B4326
:1024B00049504D4F44453D310000000041542B43ED
:1024C000495053544152543D22544350222C22250A
:1024D00073222C257500000025730000434F4E4EDB
:1024E000454354003E20576946693A2054435020E2
:1024F000C1ACBDD3CAA7B0DC0000000043495053B3
:102500005441525400000000442E00203E205769E0
:1025100046693A2054435020D2D1C1ACBDD32C20BF
:10252000BDD3CAD53A20252E3130307300000000CB
:1025300041542B43495053454E4400003E00000097
:102540003E20576946693A2043495053454E44203E
:10255000CEDE20273E27000043495053454E44001D
:10256000415400003E20576946693A20CEDE2041A2
:102570005420D3A6B4F02C20BCD9B6A8D2D1BDF833
:10258000C8EBCDB8B4AB00003E20576946693A208D
:10259000CDB8B4ABC4A3CABDB3C9B9A6000000008E
:1025A0002B4349504D4F44453A31000041542B4391
:1025B00049504D4F44453F003E20576946693A20F7
:1025C0004349504D4F444520D2D1BBB9D4ADBBF2A5
:1025D000B4D3CEB4C9E8D6C3B3C9B9A600000000CD
:1025E0003E20576946693A20BDF8C8EBCDB8B4AB78
:1025F000CAA7B0DC000000003E20576946693A20B7
:102600004349504D4F444520C8D4CEAA20312C20F8
:10261000C1ACBDD3BFC9C4DCB1BBB7FECEF1C6F7F8
:10262000B9D8B1D50000000010B540F24C442046A6
:10263000FEF739FB03210FA000F000FB2046FEF758
:1026400032FB4FF4FA6422460BA10CA000F000FB11
:1026500028B10BA002F02CF94FF0FF3010BD22463C
:1026600005A10EA000F0F4FA0FA002F0DDF80020A2
:1026700010BD00002B2B2B004F4B000041540000DD
:102680003E20576946693A20CDCBB3F6CDB8B4ABFE
:10269000CEDE20415420D3A6B4F0000041542B4399
:1026A0004950434C4F5345003E20576946693A20F4
:1026B000CDCBB3F6CDB8B4ABB3C9B9A6000000001A
:1026C00010B512A002F0B0F8FFF7AEFF00F04AFA22
:1026D00017A0F8F7A1FC40F6C410FEF7E4FA4FF497
:1026E000E130FBF75FFB4FF4FA6214A114A000F095
:1026F000AFFA28B113A002F0DBF84FF0FF3010BDA5
:1027000019A002F091F8002010BD00003E2057698A
:1027100046693A2041542B524553544F5245202884
:10272000CDFCBCC7D2D1B1A3B4E6C8C8B5E329007B
:1027300041542B524553544F524500004F4B00001B
:10274000415400003E20576946693A20B2A8CCD8CF
:10275000C2CAB8B4CEBBBAF320524553544F524507
:1027600020CEDED3A6B4F0003E20576946693A2059
:10277000524553544F524520CDEAB3C92C20D2D1F3
:10278000B1A3B4E6C8C8B5E3D2D1C7E5B3FD000034
:1027900030B585B00024124800940194029403944B
:1027A000816941F00401816180690E4D00F00400EF
:1027B0000490012220212846F9F724FA20200090D5
:1027C0000120CDE901040220039069462846F9F76B
:1027D00011F9012220212846F9F714FA05B030BD7D
:1027E000001002400008014000B5154999B00720CB
:1027F0000870282213A117A002F016F81DA000905F
:1028000010A31FA2602101A8F5F76AFE01A921A06B
:10281000F8F702FC00F0A6F928211FA000F028FB21
:1028200048B120A002F044F826A0FFF74DFD4FF07C
:10283000FF3019B000BD25A001F0F6FF0020F8E739
:10284000900000204F726179426F782D36423045FA
:10285000000000003E20576946693A20C1ACBDD354
:10286000B9CCB6A8C8C8B5E32027257327202825EA
:10287000647329006E6B7932303139323030360072
:1028800041542B43574A41503D222573222C222587
:1028900073220000257300005749464920474F54D2
:1028A000204950003E20576946693A20B9CCB6A865
:1028B000C8C8B5E3C1ACBDD3CAA7B0DCBBF2B3ACEA
:1028C000CAB1000043574A41500000003E205769FA
:1028D00046693A20B9CCB6A8C8C8B5E3D2D1C1ACD4
:1028E000BDD300002DE9F04107460E469046104644
:1028F000F6F725F885B2AE420CD30024761B07E02C
:1029000038192A464146F5F7CAFF30B1641CA4B213
:10291000A642F5DA0020BDE8F0813819FBE7000097
:1029200008B1012200E0002240210148F9F76AB90C
:1029300000080140F8B54AA001F076FF3420F9F70D
:102940000FFA3A20F9F70CFA4A48F9F74CFE4A48D0
:10295000016821F0010101600168C907FCD1464905
:102960004FF480702C390860424800680168416863
:102970000091016841680091016841680091016817
:102980004168009101684068009000F0EBF83B4C12
:10299000002220212046F9F735F94FF4FA70FEF7AE
:1029A00082F9012220212046F9F72CF940F2DC546B
:1029B0002046FEF778F900F0D5F84FF4E1352846C7
:1029C000FBF7F0F93A20F9F7DCF93420F9F7D9F9F7
:1029D00022462BA12BA000F03BF9EE0090B130462F
:1029E000FBF7E0F9224626A126A000F031F90028E5
:1029F00031D025A001F05CFF2846FBF7D3F94FF05A
:102A0000FF30F8BD40F6B8321DA127A000F020F934
:102A100018B12CA001F04CFF20E03046FBF7C2F9C2
:102A2000C820FEF740F9224615A116A000F010F9C3
:102A300078B12DA001F03CFF2846FBF7B3F96420E4
:102A4000FEF731F94FF4FA620DA131A000F000F960
:102A500004E036A000E03CA001F0E6FE0020F8BD56
:102A60003E20576946693A2045535020B8B4CEBB42
:102A70002E2E2E00BC8800203004024000080140A9
:102A80004F4B0000415400003E20576946693A20F0
:102A9000CBF9D3D0B2A8CCD8C2CABEF9CEDE204181
:102AA0005420D3A6B4F0000041542B554152545F3A
:102AB0004445463D3932313630302C382C312C30BB
:102AC0002C3000003E20576946693A205541525447
:102AD0005F44454620CAA7B0DC2C20B1A3B3D62062
:102AE00031313532303000003E20576946693A2096
:102AF00039323136303020B2BBBFC9D3C32C20BBF2
:102B0000D8CDCBB5BD20313135323030000000009A
:102B100041542B554152545F4445463D3131353285
:102B200030302C382C312C302C3000003E205769AE
:102B300046693A20B2A8CCD8C2CA202D3E203932EC
:102B400031363030000000003E20576946693A2097
:102B5000B2A8CCD8C2CAD2D1CAC720393231363095
:102B60003000000003490020088003490870034931
:102B70000870704772000020442E00206C00002076
:102B800070B5054601460FA001F04EFE00244FF43B
:102B90007A760AE015A0F8F73FFAFFF7E3FF31462F
:102BA00016A000F031F940B1641CAC42F2DB16A073
:102BB00001F07EFE4FF0FF3070BD19A001F034FE31
:102BC000002070BD3E20576946693A20BCECB2E94E
:102BD000D2D1B1A3B4E6C8C8B5E3B5C4D7D4B6AFB3
:102BE000C1ACBDD3202825647329000041542B4378
:102BF000495053544154555300000000535441541C
:102C000055533A32000000003E20576946693A2089
:102C1000CEDED2D1B1A3B4E6B5C4C8C8B5E30000D6
:102C20003E20576946693A20D2D1C1ACBDD3B1A389
:102C3000B4E6B5C4C8C8B5E3000000000A460146C2
:102C40004FF47A730148FAF7CCB80000BC88002032
:102C500070B50E460446014615460AA0F8F7DCF9A1
:102C6000FFF780FF2946304600F0CEF8002808D054
:102C7000214605A001F01CFE2046FFF725FB4FF082
:102C8000FF3070BD257300003E2057694669204122
:102C90005420B3ACCAB13A20257300002DE9F041AD
:102CA00064211FA001F0C0FD2A49082008702A4CA9
:102CB0000120207041F2883228A129A0FFF7C8FF27
:102CC0004FF0FF36002508B1257021E0FFF74AFFDD
:102CD000642127A000F0CCF84FF4FA6740B127A098
:102CE00001F0E6FD3A461DA12BA0FFF7B1FFEBE78F
:102CF0002DA001F099FD3A4618A127A0FFF7A8FFE3
:102D000025700A20FFF73CFF28B12FA001F0D0FD6D
:102D10003046BDE8F08134A001F086FD0020F8E7E0
:102D20003E20576946693A20536D617274436F6E55
:102D300066696720BFAACABC2028256473292C2095
:102D4000C7EBD3C3204553502D546F7563682041A2
:102D50005050000090000020390100204F4B00002F
:102D600041542B43575354415254534D41525400F4
:102D7000636F6E6E65637465640000003E20576982
:102D800046693A20536D617274436F6E66696720BD
:102D9000B3ACCAB10000000041542B435753544F09
:102DA00050534D41525400003E20576946693A2025
:102DB000536D617274436F6E66696720D2D1BBF147
:102DC000C8A1C8C8B5E300003E20576946693A204B
:102DD000536D617274436F6E66696720CEB4BBF148
:102DE000C8A1B5BD204950003E20576946693A2028
:102DF000536D617274436F6E66696720D2D1C1AC46
:102E0000BDD3C8C8B5E300002DE9F0418046642079
:102E100091FBF0F44FF0FF37104E114D17E0642096
:102E2000FDF741FF307890B1298842460D48FFF701
:102E300059FD10B10020BDE8F08198F80000452848
:102E400005D0298808A20748FFF74CFD18B9201EB5
:102E5000A4F10104E3DC3846EDE700006C0000203B
:102E600072000020442E00204552524F52000000B4
:102E70002DE9F041804601EB810045000C464FF002
:102E8000FF371B4E2DE06420FDF70DFF1948007839
:102E9000C0B1318842461848FFF724FD30B12146C1
:102EA00016A001F0C1FC0020BDE8F08131881AA213
:102EB0001148FFF717FDC0B9318819A20E48FFF776
:102EC00011FD90B90A2095FBF0F100FB115040B9BB
:102ED000002C06DD14480460214614A0641E01F095
:102EE000A3FC281EA5F10105CDDC3846DCE7000077
:102EF000720000206C000020442E00203E20576904
:102F000046693A20B5C8B4FDCDEAB3C92028CAA3A2
:102F100020256473290000004552524F52000000E2
:102F20004641494C00000000940000203E205769B3
:102F300046693A20B5B9BCC6CAB120256473000001
:102F40000148C088704700006001002001484089A6
:102F500070470000600100200148008A70470000AF
:102F600060010020FEB50026012202A97C20029605
:102F7000FEF7F0FF9DF808000A252E4CA52821D069
:102F8000A5208DF80800012202A97C20FFF72CF96A
:102F90002582E5808DF808508DF80960022202A98B
:102FA0007820FFF721F9E0888DF80800000A8DF8F5
:102FB0000900022202A97A20FFF716F91EA001F0EB
:102FC00033FC19E0022202A97820FEF7C3FFBDF806
:102FD0000800208241F2883608B1B04200D925822B
:102FE000022202A97A20FEF7B5FFBDF80800E080B2
:102FF00008B1B04200D9E5802079002819D0E088D6
:1030000007F0AEFD1A4E314607F0CCFC07F036FC57
:1030100005460F46208A07F0A3FD314607F0C2FCA3
:1030200007F02CFCCDE9005702460B4611A001F039
:10303000FBFBFEBD600100203E20464545443A2092
:10304000CAD7B4CEB3F5CABCBBAF2C20C9E8D6C32F
:10305000C4ACC8CF20C8A5C6A43D312E304B472CE8
:1030600020B5A5B4CECDB6C1CF3D312E304B4700F3
:10307000000020413E20464545443A20B3F5CABCF5
:10308000BBAF2C20C8A5C6A43D252E31664B472CCE
:1030900020B5A5B4CECDB6C1CF3D252E31664B4768
:1030A000000000002DE9F04F544C8FB0207900282B
:1030B0007ED0FBF701F92078012816D047F2305670
:1030C0006078012528B1F8F7A3FD6169401AB04284
:1030D00012D3F8F79DFD60616423082248494948EE
:1030E000F9F77FFE607818B106E04FF47A76E7E7EB
:1030F000657045A001F098FB06A82021FBF79CF81D
:1031000000285FDD01460EAA06A800F0B7FA0028E5
:1031100058D1BDF83800A081218A884201D9401ACF
:1031200000E000206081A07830B9A5703CA000F0DC
:10313000BBFB3FA001F078FB2078012842D138A0EA
:1031400000F0B2FB208965898346401B00D54042D0
:1031500086B2E681E08807F003FD3B4907F022FCD8
:1031600007F08CFB81468A46304607F0F9FC364969
:1031700007F018FC07F082FB07468846284607F050
:10318000EFFC314907F00EFC07F078FB05460E46D0
:10319000584607F0E5FC2C4907F004FC07F06EFBED
:1031A0008DE8E00702460B4628A001F03DFB00E059
:1031B00008E0E089E188884207D332A001F034FBBF
:1031C00000F0C6F90FB0BDE8F08F60892189884210
:1031D00007D9E078401CC0B2E070142803D331A0B6
:1031E00009E00020E070F8F713FDA169401A3049AA
:1031F0008842E7D92FA000F0E3F9E3E7600100205F
:1032000070B001083C8800203E20464545443A20E5
:10321000CAD7B4CEB2E9D1AFD2D1B7A2CBCD0000DC
:10322000696F742E70726F702E706F73740000006F
:103230003E20464545443A20CAD7B4CED6D8C1BF71
:10324000D2D1C9CFB1A80000000020413E204645A0
:1032500045443A20CDB6CEB9D6D020C6F0CABC3D42
:10326000252E316620B5B1C7B03D252E316620D25E
:10327000D1BCF53D252E316620B5A5B4CE3D252E19
:10328000316600003E20464545443A20B4EFB5BDC6
:10329000C4BFB1EACDB6CEB9C1BF2C20CDA3D6B93B
:1032A00000000000D6D8C1BFB7B4D4F600000000BB
:1032B000C0270900CDB6CEB9B3ACCAB1000000003A
:1032C00038B541F28831884218D80D4C022269463F
:1032D000E0808DF80000000A8DF801007A20FEF7EA
:1032E00083FFE08807F03CFC064907F05BFB07F032
:1032F000C5FA02460B4604A001F096FA38BD00005C
:1033000060010020000020413E20464545443A200F
:10331000C9E8D6C3B5A5B4CECDB6C1CF3D252E31B3
:10332000664B4700FEB541F2883188422CD8174CD5
:103330002082A189814201D3091A00E00021618124
:103340008DF80800000A8DF80900022202A97820F1
:10335000FEF74AFF608907F003FC0D4E314607F087
:1033600021FB07F08BFA05460F46208A07F0F8FB91
:10337000314607F017FB07F081FACDE90057024606
:103380000B4604A001F050FAFEBD000060010020D1
:10339000000020413E20464545443A20C9E8D6C3B6
:1033A000C8A5C6A43D252E31664B472C20D6D8CBC8
:1033B000E3BEBBD6D83D252E31664B47000000004A
:1033C0002DE9FC41411E41F288322A4E91420ED332
:1033D00007F0C6FB314607F0E5FA07F04FFA02B0F6
:1033E0000246BDE8F0410B4623A001F061BA2A4C29
:1033F0002178012935D0A178002934D061890029AC
:1034000033D0E08021810020E081E070F8F700FCFB
:10341000A06101202070014604F07CFC07221F49B6
:103420006620FEF7E1FE208907F09AFB314607F09F
:10343000B9FA07F023FA05460F46E08807F090FB3B
:10344000314607F0AFFA07F019FACDE90057024606
:103450000B4613A001F0E8F9BDE8FC411EA000F006
:1034600023BA21A002E029A000E030A0BDE8FC4181
:1034700001F01EBA000020413E20464545443A2056
:10348000B5A5B4CECDB6C1CFC1BFCEDED0A73D2548
:103490002E31664B47000000600100202201002011
:1034A0003E20464545443A20BFAACABCCDB6CEB957
:1034B00020B5A5B4CE3D252E31664B472C20C6F055
:1034C000CABC3D252E31664B472C20BCCCB5E7C687
:1034D000F7313DBFAA000000696F742E70726F70E3
:1034E0002E706F73740000003E20464545443A201C
:1034F000D5FDD4DACDB6CEB9D6D02C20BAF6C2D40A
:10350000B1BEB4CEC7EBC7F3000000003E20464575
:1035100045443A20B3D3CEB4BECDD0F72C20CEDE76
:10352000B7A8BFAACABCCDB6CEB900003E2046455A
:1035300045443A20CAA3D3E0D6D8C1BFCEAA203092
:103540002C20CEDEB7A8BFAACABCCDB6CEB900002B
:1035500010B5104C207800281BD00021012004F069
:10356000D9FB07220C496620FEF73EFE02202070A0
:10357000E08907F0F5FA094907F014FA07F07EF937
:1035800002460B4606A001F04FF9BDE8104004F0DA
:1035900003BB10BD6001002022010020000020417B
:1035A0003E20464545443A20CDA3D6B9CDB6CEB946
:1035B0002C20D2D1BCF5C9D93D252E31664B470010
:1035C00010B504460021012004F0A4FB072207499E
:1035D0006620FEF709FE064903200870214605A073
:1035E00001F066F9BDE8104004F0D6BA22010020CF
:1035F000600100203E20464545443A20D2ECB3A36A
:10360000CDA3D6B92C2025730000000008B5FF20FB
:103610008DF8000001226946AC20FEF79BFC9DF866
:103620000000012802D901208DF80000054910F0A2
:10363000FF00087101D004A100E007A10BA001F078
:10364000F3F808BD60010020B3C6D6D8CDB6C1CF0F
:1036500028B4F8B3D3290000CBC4C2B7BCCCB5E7BB
:10366000C6F728CEDEB3D329000000003E20B2FA10
:10367000C6B7C4A3CABD3A20257300002DE9F041A6
:1036800094B00E46044690464C216846F5F7A4FADD
:10369000182E02D91827002502E0374600250AE037
:1036A00005EB450069460844635D40A20421F4F738
:1036B00017FF6D1CADB2BD42F2D36A4631463DA044
:1036C00001F0B2F8092E08D2314642A001F0F0F81C
:1036D0004FF0FF3014B0BDE8F0812178012906D009
:1036E00001224BA001F0E4F86FF00200F2E76178EC
:1036F000832908D003290DD0032251A001F0D8F866
:103700006FF00400E6E7A2785A4801F0D1F86FF0B4
:103710000300DFE707234FF6FF7100204AF201059F
:10372000225C51400022CE0702D085EA510100E020
:103730004908521CD2B2082AF5D3401C80B29842E4
:10374000EED3B4F80720914205D04B4801F0B0F811
:103750006FF00100BEE7A179404661F3070061798F
:1037600061F30F20217961F31740E17861F31F6065
:103770004249054607F008FA07F0D6F941F28831C8
:10378000002801DA002002E0884200DD084684B209
:10379000A8F80040284607F071F802460B4638A00A
:1037A000009401F041F8002094E7000025303258E1
:1037B000200000003E20464545443A20343835205C
:1037C000CAD5B5BD20256420D7D6BDDA3A202573E9
:1037D000000000003E20464545443A20BDE2CEF6BA
:1037E000CAA7B0DC2DD6A1B3A4B6C8B9FDB6CC2803
:1037F00025643C39292CBFC9C4DCB2A8CCD8C2CAC4
:10380000B2BBB6D4BBF2CFDFC2B7B8C9C8C50000DF
:103810003E20464545443A20BDE2CEF6CAA7B0DC7C
:103820002DD5BEBAC5B2BBB7FB28CAD53078253076
:10383000325820C6DACDFB307825303258290000C6
:103840003E20464545443A20BDE2CEF6CAA7B0DC4C
:103850002DB9A6C4DCC2EBB2BBB7FB28CAD5307801
:103860002530325820C6DACDFB3078253032582941
:103870000000000024B9010874B9010800002041CB
:103880003E20464545443A2034383520D4ADCABCA4
:10389000C3ABD6D83D252E31664B472028302E317C
:1038A0006B673D25642900002DE9FF47314C608995
:1038B00007F056F9304F394607F074F80646E088AD
:1038C00007F04EF9394607F06DF80546208A07F0F3
:1038D00047F9394607F066F80146284890F86A200B
:1038E00002B1012201AB009283E8620090F86910F6
:1038F00009B1012300E0002390F8681009B101220A
:1039000000E0002290F86700002802D04FF001018B
:1039100001E04FF0000102D04FF0010001E04FF054
:103920000000F9F7FFFF208A07F01AF9B946394677
:1039300007F038F806F0A2FF07468846E08807F04F
:103940000FF9494607F02EF806F098FF05460E4697
:10395000608907F005F9494607F024F806F08EFF64
:103960008DE8E00102460B4605A000F05DFFBDE8D2
:10397000FF8700006001002000002041BC00002003
:103980003E20464545443A20BEBBD6D83D252E3183
:10399000664B4720B5A5B4CECDB6C1CF3D252E315F
:1039A000664B4720C8A5C6A43D252E31664B47006F
:1039B00001B59DF8000000B1012005498DF8000017
:1039C000012208716946AC20FEF70EFC08BD00001C
:1039D00060010020F0B5002689B007464FF0FF35A2
:1039E00034466946204603F0A1FC684603F0B0FC6B
:1039F00038B1002D03DB0198801B002801DD019EFA
:103A00002546641CE4B20A2CEBD307B13E6009B032
:103A10002846F0BD10B5144600222260114A21F05C
:103A200000439342A8BF10BD53EA000208BF10BD77
:103A3000B3F5801FA8BF226807DA362207F058FACC
:103A40006FF0350221F000432260DFF81CC06FF3F5
:103A50001E510CEB23531A4441F0FF5141F0005129
:103A6000226010BD0000F07F02FCFFFF1FB5402068
:103A700000900120019002900220039069460248C4
:103A8000F7F7B8FF1FBD0000001001402DE9F04F0F
:103A90000F468DB015461E46044621F0004104F045
:103AA00001FCDFF8A8816A4B424606F0D7FB81464D
:103AB0008A464246674B2046394606F0CFFB2A46E7
:103AC000334606F0CBFB8B4608904246604B2846B7
:103AD000314606F0C3FB2A46334606F0BFFBCDE96C
:103AE000051000225C4B2846314606F0B7FB0191D9
:103AF000049001222046394607F0FAF98046002258
:103B0000564B039106F07EF8019B049A06F07AF872
:103B1000DDE9053206F076F85B46089A06F072F8A1
:103B20004A46534606F06EF882468B4640464C4A5B
:103B30004C4B039906F092FB04F064FB00224A4BC5
:103B400006F08CFB804689460022484B20463946C9
:103B500006F084FB424A434B06F080FB04F052FB24
:103B60000022414B06F07AFB42464B4606F04AF8EB
:103B7000012207F0BDF90022374B06F0FFF852464C
:103B80005B4606F03FF881468A460022324B2846C3
:103B9000314606F0F3F8324A324B06F05FFB04F090
:103BA00031FB0022324B06F059FB074688462C4A6F
:103BB0002C4B2846314606F051FB8B46044604F058
:103BC00021FB0022284B06F049FB3A46434606F00B
:103BD00019F8012207F08CF900221F4B06F0CEF8ED
:103BE0004A46534606F00EF8074688462046594690
:103BF0000022204B06F0C2F804F004FB00221E4B0A
:103C000006F02CFB0446894600221C4B2846314610
:103C100006F0B4F8124A134B06F020FB04F0F2FA57
:103C20000022174B06F01AFB22464B4605F0EAFF2E
:103C3000012207F05DF90022074B06F09FF80DB056
:103C40003A464346BDE8F04F05F0DCBF9A99999992
:103C50009999C93F9999B93F00000840000059C09F
:103C6000182D4454FB210940000034400000184046
:103C70000000444000003E40000074400000284026
:103C8000000064402DE9FF5F0D4682B0044621F03C
:103C9000004104F007FB6B4E6B4F32463B4606F08B
:103CA000DDFA82468B4632463B462046294606F0E0
:103CB000D5FADDE904230F46064606F0CFFA804622
:103CC00089463046394622462B4606F0C7FA064654
:103CD0000F46DDE90401012207F00AF9CDE90001F0
:103CE00000225A4B2046294605F08CFFDDE90023CF
:103CF00005F088FF32463B4605F084FF42464B46BE
:103D000005F080FF52465B4605F07CFF8046894601
:103D100001222046294607F0EBF84D4A4D4B06F0AC
:103D20009DFA04F06FFADFF830A10022534606F046
:103D300095FA0F4606460022484B2046294606F0D3
:103D40008DFA434A434B06F089FA04F05BFA0022ED
:103D5000534606F083FA32463B4605F053FF0122F4
:103D600007F0C6F8DFF8F8B000225B4606F006F868
:103D700042464B4605F046FF8046894600225B4698
:103D80002046294605F0FAFF314A324B06F066FA22
:103D900004F038FA0022334B06F060FA0E4607466C
:103DA0002B4A2C4B2046294606F058FA04F02AFAF2
:103DB0000022534606F052FA3A46334605F022FFF7
:103DC000012207F095F800225B4605F0D7FF424636
:103DD0004B4605F017FF804689460022224B2046BD
:103DE000294605F0CBFF1A4A1A4B06F037FA04F0C1
:103DF00009FA0022154B06F031FA0E46074600225A
:103E00001A4B2046294605F0B9FF114A114B06F01E
:103E100025FA04F0F7F90022154B06F01FFA3A468E
:103E2000334605F0EFFE012207F062F800225B4600
:103E300005F0A4FF06B042464B46BDE8F05F05F032
:103E4000E1BE00009A9999999999B93F00C07240D2
:103E5000182D4454FB210940000034400000184054
:103E6000000008400000444000003E4000002840A0
:103E700000C0624010B500240848F7F7D9FA0A21BB
:103E80000648F7F73DFA18B90448F7F779F984B20C
:103E90000248F7F72DFB204610BD0000CC6600203D
:103EA00008B5FF208DF8000001226946AD20FEF71D
:103EB00051F89DF80000012802D901208DF800007A
:103EC000054910F0FF00087101D004A100E005A130
:103ED00007A000F0A9FC08BD6C000020BFAAC6F432
:103EE00000000000B9D8B1D5284750533029000050
:103EF0003E2047505320B6A8CEBB3A202573000081
:103F000001B59DF8000000B1012005498DF80000C1
:103F1000012208716946AD20FEF766F908BD000070
:103F20006C000020064810B5817831B10549006A5F
:103F300006F0F6FEB0F5000F00DA002010BD00001C
:103F4000B80100200AD7A33C70B5114C6068002866
:103F50001DD006F0EDF806460D46D4E90E0106F038
:103F6000FBF832462B4606F079F94FF00052094B28
:103F700006F074F94FF0FF3206F0BAFF4FF04542F9
:103F8000054B05F0FBFEBDE8704005F009BE70BDB5
:103F9000B80100203108004085318A420648817806
:103FA00019B1406AB0F1804F01DA002070474FF03C
:103FB0007C5106F0B5BE0000B801002003488178AE
:103FC00009B1C0697047002070470000B8010020A7
:103FD0001CB50020CDE9000008226946A420FDF7A9
:103FE000B9FFDDE90010C94371EA000102D10020E8
:103FF000CDE900000E4CDDE90001C4E90E01C4E981
:104000001001F9F733F8F9F757FFD4E90E0150EA38
:10401000010208D0074A0023F4F7BAF9014606A0C6
:1040200000F002FC1CBD11A000F0FEFB1CBD000056
:10403000B801002000CA9A3B3E20B5E7C4DC3A2014
:10404000484C573830333220BECDD0F72028554168
:1040500052543520504432292C20C0FACAB7C2F637
:10406000B3E520256C752530396C75003E20B5E729
:10407000C4DC3A20484C573830333220BECDD0F71C
:104080002028554152543520504432290000000068
:1040900010B5074CA07840B1F7F7BAFD616B401A34
:1040A000B0F57A7F01D2012010BD002010BD0000C4
:1040B000B80100202DE9F84F00220221435C491C81
:1040C0001A44C9B2D2B21629F8D9C17D91427CD125
:1040D000817BC27B090441EA0221027C114374D036
:1040E000804C4FF0000861608178C278090441EA91
:1040F000022102791143A16041798279090441EAE0
:104100000221C2791143E160017A427A090441EA4D
:104110000221827A11432161C17A027B090441EABA
:104120000221427B11436161417C827C090441EAA6
:104130000221C27C1143A161017DB0F8150001F09C
:10414000800145BAA07800285DD06078814203D014
:10415000A06A401CA0626170F7F75AFD216B4FF016
:104160000109411A14392063822950D8E0780328C4
:1041700004D2401CC0B2E07003284AD3E06888B182
:1041800005F0D6FF06460F46A06805F0D1FF32467F
:104190003B4605F0F3FD4FF00052534B06F05EF83E
:1041A00005F0FEFC8346606990B105F0C1FF06464C
:1041B0000F46206905F0BCFF32463B4605F0DEFDA8
:1041C0004FF0FF3206F094FE00E022E005F0E8FC3C
:1041D0008246A069F8B105F0ABFF06460F4660685D
:1041E00005F0A6FF32463B4605F0C8FD4FF00052F1
:1041F0003D4B06F033F84FF0FF3206F079FE05F044
:10420000CFFC064608E06170C4F82880A4E784F873
:104210000390BDE8F88F0026E1695846009106F04A
:104220007FFD6FF00207394606F090FE009906F018
:1042300051FBE061216A50468B4606F071FD39461C
:1042400006F084FE594606F045FB2062616A30465E
:104250008A4606F065FD394606F078FE514606F0BE
:1042600039FB6062208DA27805EB004162B1E06A03
:10427000814201D3081A00E00846D4E90E532818F9
:1042800043EB0803C4E90E03E16232BB84F80290F9
:1042900016A0616800F0C8FA606805F049FF4FF0A9
:1042A0000052114B05F0DAFF4FF0FF3206F020FE0E
:1042B00002460B464FF04540154905F05FFD06F0FC
:1042C000A5FDD4E90E23121A8B4106D2C4E90E01D2
:1042D00000F05CF80FA000F0A7FAF7F799FC606314
:1042E00097E70000B8010020310800403E20B5E704
:1042F000C4DC3A20484C573830333220D4DACFDF90
:104300002C20B9A6C2CAB2CECAFD3D256C750000EC
:1043100085318A423E20B5E7C4DC3A20B5D7CAFDD4
:10432000D2D1B3F5CABCBBAFCEAA20312E303020DB
:104330006B576800F0B413490F25134A0B78012618
:104340006BB10024012B15D0D0545B1CD8B208707F
:1043500018280DD30C70F0BC1046FFF7ABBE5528E3
:1043600004D0AA2802D0B5EB101F01D110700E7036
:10437000F0BC70475A2801D00C70F0E75070022052
:104380000870F5E7B8010020D08900201CB50B4C5F
:10439000D4E90E10D4E910234A4043401A430CD00C
:1043A000CDE9001008226946A420FDF71DFF002872
:1043B00003D1D4E90E01C4E910011CBDB8010020ED
:1043C00070B5194E706800282CD005F0B1FE4FF082
:1043D0000052164B05F042FF4FF0FF3206F088FD09
:1043E00002460B464FF08060114905F0C7FC0446B9
:1043F0000D4600220F4B05F0F5FE01D20D4D0024B5
:104400002046294606F002FDB36B3C3696E83400A0
:104410001B1B62EB0502181A8A4103D3BDE87040EA
:10442000FFF7B4BF70BD0000B801002031080040A4
:104430006BF454420000F03FF0B5234885B0816929
:1044400041F00401816180694FF4805600F004005E
:1044500004901120CDE900601C4D032769460397A5
:104460002846F7F7C7FAEC140120CDE90040694669
:1044700003972846F7F7BEFA012221462846F7F7A8
:10448000C1FB012231462846F7F7BCFB31462846DE
:10449000F7F7ACFB002815D100260022214628465C
:1044A000F7F7B0FB0520FDF731FC01222146284635
:1044B000F7F7A8FB0520FDF729FC761C092EECDB9D
:1044C00000F0B2F805B0F0BD001002400008014055
:1044D0002DE9F0472E4D814600244FF40067224617
:1044E00039462846F7F78EFB1420FDF70FFC00260F
:1044F0004FF48058012239462846F7F783FB1420F1
:10450000FDF704FC6006040E41462846F7F76EFBF3
:1045100008B1641CE4B21420FDF7F8FB0022394610
:104520002846F7F76FFB1420FDF7F0FB761CF6B278
:10453000082EDFD3B9F1000F1AD0002246464146BB
:104540002846F7F75FFB012239462846F7F75AFB62
:104550000220FDF7DBFB002239462846F7F752FB25
:10456000012231462846F7F74DFB2046BDE8F0878B
:10457000012241462846F7F745FB012239462846E5
:10458000F7F740FB0220FDF7C1FB00223946E9E7BF
:10459000000801402DE9F041154E05464FF4006733
:1045A000002239463046F7F72DFB00244FF480589F
:1045B000EA0941463046F7F725FB6806050E02205A
:1045C000FDF7A4FB012239463046F7F71BFB02201A
:1045D000FDF79CFB002239463046F7F713FB641CBD
:1045E000E4B2082CE4D3BDE8F04100F037B8000095
:1045F0000008014070B501220A4D140321462846E7
:10460000F7F700FB0122D1022846F7F7FBFA042056
:10461000FDF77CFB21462846BDE870400022F7F7F5
:10462000F1BA00000008014070B50B4D4FF4805402
:10463000002221462846F7F7E5FA0122D102284652
:10464000F7F7E0FA0420FDF761FB21462846BDE8B4
:1046500070400122F7F7D6BA000801402DE9F04179
:104660000122154D1603002431462846F7F7CAFAF1
:104670000122D70239462846F7F7C4FA0BE0641C3A
:10468000E4B2FA2C04D9FFF7CFFF0120BDE8F08196
:104690000220FDF73BFB31462846F7F7A7FA002832
:1046A000EDD1002239462846F7F7ACFA1420FDF781
:1046B0002DFB0020EAE700000008014010B5044689
:1046C000B031C9B2002001F0A3FC102040EA14115F
:1046D000002001F09DFC04F00F01BDE81040002017
:1046E00001F096BC2DE9F04106460C4640F2FF75FC
:1046F000174635EA14502BD000221346304605F0F9
:1047000095FC25D03A463046214606F0F1FB064698
:104710000C4635EA145010D000221346304605F0FE
:1047200085FC15D10220F4F7FEFAFAF787FD0A4658
:10473000214662F31E01BDE8F0810220F4F7F3FA8E
:10474000FAF775FD0A46214662F31E01BDE8F081C5
:1047500030462146BDE8F081F0B585B01B48002504
:104760000295816941F010018161816901F01001B8
:104770000491816941F0040181618069144F00F066
:104780000400049001204603CDE90060022469463C
:1047900003943846F7F72EF900940E4C69462046EC
:1047A000F7F728F9002231463846F7F72BFA0122AD
:1047B00002212046F7F726FA074C2570F7F728FA6A
:1047C0006060F7F725FAA06005B0F0BD0010024068
:1047D0000010014000080140380100200FB405A17D
:1047E00010B503AB0120029AFAF78EFD10BC5DF8FC
:1047F00014FB000044454255470000000FB405A1DA
:1048000010B503AB0420029AFAF77EFD10BC5DF8E8
:1048100014FB00004552524F52000000014800783E
:1048200070470000B40000200FB405A110B503AB21
:104830000220029AFAF768FD10BC5DF814FB000034
:10484000494E464F0000000038B501248DF8004065
:1048500022466946A020FDF77DFB9DF80000052853
:1048600006D98DF8004001226946A020FDF7BCFC66
:1048700002499DF80000087038BD0000B400002017
:1048800010B5012004F02AFD0149486010BD000068
:10489000B4000020054908B508708DF80000012219
:1048A0006946A020FDF7A0FC08BD0000B400002070
:1048B0000FB405A110B503AB0320029AFAF724FD4B
:1048C00010BC5DF814FB00005741524E0000000080
:1048D00070B50546FFF78EFEA020FFF75BFE04468D
:1048E0002846FFF757FE0443FFF784FEA120FFF799
:1048F00051FE2043040007D0FFF796FE214608A092
:10490000FFF7D6FFFF2070BD0020FFF7E1FD044652
:10491000FFF78AFE0520F7F75BF8204670BD000020
:104920003E20454520B6C1B3F5CABCBBAFB4EDCE01
:10493000F3206572723D3078253032580000000057
:104940002DE9F04115460F460646FFF753FEA0201D
:10495000FFF720FE04463046FFF71CFE0443FFF736
:1049600049FEA120FFF716FE40EA040800246E1E4F
:1049700005E00120FFF7ACFD3855641CA4B2B44239
:10498000F7DB0020FFF7A4FD791901F8010CFFF710
:104990004BFE0520F7F71CF84046BDE8F08100000B
:1049A0002DE9F04100250E46074603241CE000BF18
:1049B000FFF720FEA020FFF7EDFD05463846FFF784
:1049C000E9FD05433046FFF7E5FD0543FFF72CFE03
:1049D0000A20F6F7FDFF55B12246394605A0FFF73C
:1049E00067FF0520F6F7F4FF641EE4B2E0D2284624
:1049F000BDE8F0813E20454520D0B4C8EBB4EDCEF3
:104A0000F3204025752C20D6D8CAD43D257500004A
:104A10002DE9F0470024174688468146032526E005
:104A2000FFF7E8FDA020FFF7B5FD06464846FFF773
:104A3000B1FD40EA0604002607E000BF18F80600B2
:104A4000FFF7A8FD0443761CF6B2BE4201D2002C4B
:104A5000F4D0FFF7E9FD0A20F6F7BAFF54B12A4671
:104A6000494606A0FFF724FF0520F6F7B1FF6D1EAB
:104A7000EDB2D5D22046BDE8F08700003E20454586
:104A800020D2B3D0B4C8EBB4EDCEF3204025752CC2
:104A900020D6D8CAD43D2575000000000549044839
:104AA0000860F6F709FAFBF759FEFBF753FFFEE73C
:104AB0000080000808ED00E02DE9F041314F1020A2
:104AC0003C463870042130A2384602F0C8FA04216E
:104AD0002154401C80B2C2212154401C80B20026C7
:104AE0002654401C80B23C212154401C81B207F561
:104AF0000072384602F0B3FA014607F506723846EE
:104B000002F0ADFA014607F50C72384602F0A7FA3A
:104B10000546001F80B280460146601CFDF7C4FBBD
:104B20000446032809D238194246391D401CF3F7C0
:104B3000B5FFC4F10300281A85B2154915A0FFF787
:104B400073FE29460F48FEF779F8194D2E700024A0
:104B50006420FCF7A8F800BF00F07EF80128FBD025
:104B6000287828B113A0FFF75FFE0020BDE8F08190
:104B7000641C322CECDB16A0FFF79AFE4FF0FF30DE
:104B8000F4E700006E6400204D5154540000000012
:104B90006E6600203E2057694669204D5154543AB4
:104BA00020434F4E4E454354206369643D257300B6
:104BB000A40000203E2057694669204D5154543AC4
:104BC00020434F4E4E41434B20B3C9B9A6000000CD
:104BD0003E2057694669204D5154543A20434F4E68
:104BE0004E41434B20B3ACCAB100000070B50D4636
:104BF0001646014617220D48F4F715F80B48002415
:104C00001722C47529461830F4F70DF80748172203
:104C100018303146C4751830F4F705F803483030C1
:104C2000C475034804704470847070BD6E660020C3
:104C3000A4000020064810B5C02101700021417079
:104C40000221FDF7FBFF03490120887010BD000021
:104C50006E640020A40000202DE9F84FDFF838A191
:104C60004C4DBAF80040DFF834B14FF0000954B1B0
:104C70004BA00090F3F763FE87B2BC421DD3002621
:104C8000A4EB07080AE08BF8009037E0A8193A4631
:104C90000099F3F704FE20B1761CB6B2B045F5DA00
:104CA0000BE0F54209D0BAF80000FCF7B7FF8BF82B
:104CB00000904FF0FF30BDE8F88F28780309581EA8
:104CC0000E2801D3012061E0002101263046A042D8
:104CD00014D22F5C07F07F0202FB061102463F064A
:104CE00004D5501CF601C0B20428F0D932B15618D0
:104CF000761CB6F5205FE5D2B44201D20020DAE797
:104D0000A8180124284A401C022B06D0032B21D0CE
:104D1000092B11D00D2B38D119E0022901D343788A
:104D20001BB1022903D3417802E014702DE0FF216A
:104D30001EA0FFF7BDFD28E0032904D3807880285A
:104D400001D0547021E022A0FFF7B2FD1DE082F8EF
:104D500002901AE0028852BA931C8B4215D88C1A22
:104D6000A41EB4F5C07F01D340F27F1481182246FF
:104D70001E48891CF3F74DFE1C491DA001F8049044
:104D8000FFF752FD194800F02DF9B0B2FCF746FFCD
:104D9000012090E7442E0020720000206C000020CB
:104DA000434C4F5345440000A40000203E20576967
:104DB0004669204D5154543A20434F4E4E41434B87
:104DC00020B1BBBEDCBEF82072633D25750000003B
:104DD0003E2057694669204D5154543A205355425C
:104DE00041434B20B1BBBEDCBEF80000EE620020A8
:104DF0003E2057694669204D51545420BDD3CAD531
:104E00003A20252E323030730000000070B50D4678
:104E10000646F3F794FD04462846F3F790FD211863
:104E2000C81D891CB0F5007F05D912A0FFF740FD11
:104E30004FF0FF3070BD184C30202070601CFDF723
:104E400033FA411C3246204602F009F9064628464C
:104E5000F3F775FD0246A0192946F3F7DAFD284657
:104E6000F3F76DFD304481B22046FDF7E7FE0020E8
:104E700070BD00003E2057694669204D5154543A98
:104E8000207075626C69736820B1A8CEC4B9FDB397
:104E9000A4202825752900006E6400202DE9F0412A
:104EA0001E4C06468220207001273046F3F747FD4E
:104EB000411D601CFDF7F8F9401C00252554401CDD
:104EC000411C27543246204602F0C9F82554401CA4
:104ED00084B2314612A0FFF7A7FC21460F48FDF728
:104EE000ADFE144E757000246420FBF7DCFE00BF9D
:104EF000FFF7B2FE0128FBD0707828B10EA0FFF7B3
:104F000093FC0020BDE8F081641C322CECDB11A086
:104F1000FFF7CEFC4FF0FF30F4E700006E64002096
:104F20003E2057694669204D5154543A205355420A
:104F300020257300A40000203E2057694669204DBB
:104F40005154543A2053554241434B20B3C9B9A65A
:104F5000000000003E2057694669204D5154543AE4
:104F60002053554241434B20B3ACCAB1000000006E
:104F700010B5074CE068002809D004F041FC022875
:104F800005D1C11EE068BDE8104004F0ADBB10BD06
:104F90007C00002010B5094CE06868B104F030FCDA
:104FA000022809D14FF4FA61E06804F09DFB012862
:104FB00002D04FF0FF3010BD002010BD7C0000205B
:104FC00010B5074CE068002808D004F019FC02284E
:104FD00004D1E068BDE8104004F0AABA10BD00009A
:104FE0007C0000202DE9F047C6B0054614211FA81B
:104FF000F3F7F2FD14221FA9284601F02BFD9DF8BE
:105000007C0028B16F491FA8F3F738FE002857D05D
:1050100013221FA96B48F3F706FE6BA12846F3F78E
:105020002CFC10B1284602F0BBF96BA12846F3F71F
:1050300024FC002841D06EA0FFF7F6FB202116A823
:10504000F3F7CAFD502102A8F3F7C6FD142140A8CA
:10505000F3F7C2FD0026ADF878604FF05108B14675
:105060006A4668A12846009601F098FD08B10098AC
:1050700086B21EAA64A1284601F0C0FC644CBDF8AB
:1050800078303246B4F8741062A0FFF7CDFB002EE2
:105090001BD0B4F87400B04217D3142240A928469C
:1050A00001F0D8FCB4F87410324666A0FFF7BCFBE0
:1050B0000A2240A970A0F8F701F946B0BDE8F087D0
:1050C0001FA973A0FFF7B0FBF7E751491D223C3140
:1050D00016A8F3F7A8FD76A102A8F3F70CFC14229A
:1050E00040A9284601F0B6FC642127A8F3F774FD17
:1050F000642327AA72A1284601F030FD002849D078
:1051000027A970A0FFF790FB27AF072272A13846AE
:10511000F3F734FC00B9FF1D2F213846F3F7A3FB4A
:1051200005463A213846F3F79EFB04000DF1580A74
:1051300021D00DB1AC421FD2E01B80460246394659
:105140005046F3F766FC0AF808904FF000086FF03D
:105150002F0105E008EB880201EB420200EB020898
:1051600014F8010FA0F13002092AF3D995B14F22AA
:10517000294602A80CE045B1EC1B224639465046B0
:10518000F3F747FC0AF80490F1E71D223946504630
:10519000F3F749FD02AB424616A951A0FFF744FBC5
:1051A000534840AB02AA407941460128BDF8780037
:1051B000CDE9006016A802D0FAF7C4FC7DE700F044
:1051C00087F97AE7AA560020696F742E70726F70A3
:1051D0002E73657400000000696F742E6F74612E69
:1051E000757067726164652E706F737400000000E3
:1051F0003E204F544120C9FDBCB6C3FCC1EEA3A163
:1052000000000000766572006372633136000000B2
:10521000BC0000203E204F544120B0E6B1BE3A20F1
:10522000B5B1C7B03D25752C20D0C2B0E6B1BE3DAA
:1052300025752C2063726331363D30782530345823
:10524000000000003E204F54413A20B0E6B1BECFEE
:10525000E0CDACBBF2B8FCB5CDA3ACCCF8B9FD2029
:1052600028B5B1C7B03D25752C20D0C2B0E6B1BE7F
:105270003D25752900000000696F742E6F74612E42
:1052800070726F67726573732E706F7374000000B5
:105290003E204D5154543A20D6D8B8B4CFFBCFA2BB
:1052A000CCF8B9FDA3AC69643D252E3136730000FE
:1052B0002F6669726D776172652E62696E000000FB
:1052C00075726C003E204F544120CFC2D4D8B5D85F
:1052D000D6B73A2025730000687474703A2F2F00F7
:1052E0003E204F54413A2025733A2564257300002F
:1052F0007C00002010B50EA0FFF7DAFAF8F7CAFD1F
:105300000020FDF70DFB1049002008704870C870A0
:1053100008710E4A10700E4A10704871F9F784F83F
:10532000FFF726FEFAF7C6F9BDE81040FFF748BEC2
:105330003E204E45543A20C7D0BBBB205769466932
:10534000202D3E20344700007C0000206D0000200E
:105350006E000020F8F768F8052003F06BFAF9E713
:10536000F0B58DB039A0FFF75FFA3D4D00202870F1
:105370006870FDF70DFAF8F773FDFDF7DBFA4FF0F3
:10538000FF37002846D14FF4FA64224635A136A0F3
:10539000FDF75EFC00283DD1621032A133A0FDF77D
:1053A00057FC22462FA133A0FDF752FC002831D133
:1053B0000024F7F7D7FE022803D10A20FDF7E0FB0F
:1053C00048B1FDF711FA38B1FDF768FC18B12CA00F
:1053D000FFF76EFA1EE00124314E06F13C00B6F8EC
:1053E0006410FCF7ADFFA8B906F12802A2F1140180
:1053F0003046FFF7FBFBFFF75FFB58B906F15003A0
:1054000028A2302101A80096F3F76AF801A8FFF757
:1054100045FD10B138460DB0F0BD214B23A230211F
:105420002648F3F75DF801202870F6F7F1FB686075
:1054300023A0FFF7F9F90CB1022000E00120F7F7F3
:10544000A1FE0120F8F78EF90020E4E73E2057691D
:1054500046693A20B3F5CABCBBAF2E2E2E00000021
:10546000980000204F4B000041540000415445304B
:105470000000000041542B43574D4F44453D31003F
:105480003E20576946693A20CBF9D3D020415020BD
:10549000C1ACBDD3B7BDCABDBEF9CAA7B0DC000060
:1054A000BC00002025732573000000002F696F7475
:1054B0002F646174612F75702F257300BE56002014
:1054C0003E20576946693A205265616479000000C0
:1054D0002DE9FC5F8046DDE90CBA002499461646AA
:1054E0000F462FA00194FFF79FF9FEF731F8002136
:1054F000012002F00FFC002249462EA0F7F7DEFE45
:105500004FF4FA70FBF7CFFB304D01202870304884
:10551000047001A80090534632463946404603F0D5
:105520008BFB0646FFF71CFF2C7040B129A0FFF74C
:10553000BFF98EB131A0FFF7BBF9BDE8FC9F4EB1BA
:105540000022494636A0F7F7B9FE4FF4FA60FBF7A0
:10555000AAFBEEE70122F4E736A0FFF765F93FA0CA
:10556000FFF762F947A0FFF75FF932A0FFF75CF998
:10557000524658460199F9F735F9082002F066FDC0
:105580006420FBF790FBBFF34F8F48480168484AFF
:1055900001F4E06111430160BFF34F8F00BFFDE7ED
:1055A0003E2057694669204F54413A20BFAACABCE1
:1055B00000000000696F742E6F74612E70726F6747
:1055C000726573732E706F73740000007E0000208C
:1055D000980000203E2057694669204F54413A20E8
:1055E0004D51545420D6D8C1ACCAA7B0DCA3ACBD31
:1055F000E1B9FBC9CFB1A8B6AACAA7003E20576936
:105600004669204F54413A20D2D1D6D0D6B9A3AC66
:10561000BBD6B8B4D5FDB3A3D4CBD0D00000000026
:10562000696F742E6F74612E726573756C742E7051
:105630006F7374002A2A2A2A2A2A2A2A2A2A2A2A1C
:105640002A2A2A2A2A2A2A2A2A2A2A2A2A2A2A2ABA
:105650002A2A2A2A2A2A2A2A2A2A00002A202057E5
:10566000694669204F544120CFC2D4D8CDEAB3C98E
:10567000A3A1202020202020202020202020202026
:10568000202A00002A2020D5FDD4DAD6D8C6F4BDC1
:10569000F8C8EB20426F6F744C6F616465722E2EF8
:1056A0002E20202020202020202A00000CED00E0C9
:1056B0000400FA0570B5264CA0780025002815D006
:1056C000A57024A0FFF7F4F82F4901200870257079
:1056D0000D2002F0BBFCFCF7F3FF10B12BA0FFF78D
:1056E000E7F86420F6F774F9F9F766FA20780028ED
:1056F0002CD000BFFFF7B0FA0128FBD0401C18D017
:10570000F6F786FA6168401A47F2305188421DD395
:105710002748007890B1E078401CC0B2E0700228C1
:105720000DD324A0FFF76AF85FF0050002F08EFCAD
:10573000D7E72CA0FFF762F80420F7E7E570F6F74B
:1057400067FA6060BDE87040FFF774BA70BD000092
:10575000980000203E20576946693A20CAD5B5BD59
:10576000BBD6B8B4B3F6B3A7C7EBC7F3A3ACD6B4F4
:10577000D0D02041542B524553544F524520B2A211
:10578000D6D8C6F4000000007E0000203E205769F5
:1057900046693A20524553544F524520CAA7B0DCBF
:1057A000A3ACC8D4C7BFD6C6D6D8C6F40000000084
:1057B000A60000203E20576946693A20D0C4CCF8A4
:1057C000B3ACCAB120363073A3A8B7FECEF1C6F78A
:1057D000CEDECFECD3A6A3A9A3ACCFB5CDB3B8B4DE
:1057E000CEBB00003E20576946693A20C1ACBDD30C
:1057F000B1BBB7FECEF1C6F7B9D8B1D5A3A8B1BB3E
:10580000C6BDCCA8CCDFCFC2CFDFA3A9A3ACCFB598
:10581000CDB3B8B4CEBB000010B50A4C2178002936
:105820000FD001460848FFF7F1FA002809D1607847
:10583000002806D101206070BDE8104003A0FEF7EB
:10584000F3BF10BD98000020BE5600203E205769CF
:1058500046693A20CAD7B4CEB7A2B2BCB3C9B9A67A
:105860000000000070B5174E002280213046F6F788
:10587000C9F90122D1031448F6F7C4F95FF0000416
:1058800004F1B000C1B2002000F0C2FB00210846C4
:1058900000F0BEFB1021002000F0BAFB0025002123
:1058A000012000F0B5FB6D1CEDB2802DF7D3641C18
:1058B000E4B2082CE4D33046BDE8704001228021D8
:1058C000F6F7A0B900100140000C01402DE9F043AB
:1058D00085B0002000900190029003902A488169D1
:1058E00041F008018161816901F008010491816939
:1058F00041F0100181618069012200F01000DFF8A1
:105900008C801403049021464046F6F77BF901226F
:10591000550229464046F6F775F90122160231462E
:105920004046F6F76FF9012280214046F6F76AF902
:105930000122DFF85C90D70339464846F6F762F952
:105940000120019002900220039069460094404695
:10595000F6F750F8694640460095F6F74BF8694669
:1059600040460096F6F746F880200090694640468B
:10597000F6F740F8694648460097F6F73BF8FEF719
:1059800075F805B0BDE8F08300100240001001403A
:10599000000C014070B58AB00446F6F739F942F2BE
:1059A0001071B0FBF1F00321B0FBF1F201FB12002A
:1059B0004600A048007800287ED04EF66020B4FB58
:1059C000F0F4F7F7C9FB01285BD09BA34FF4B46256
:1059D000B4FBF2F53C21B4FBF1F002FB154501FBF1
:1059E0001040B5FBF1F1B4FBF2F2CDE900210290D9
:1059F00092A2182104A8F2F773FD0021084600F0D6
:105A000051FA304600F03CFB04A800F0E3FAFEF740
:105A10003FFB002837D0FEF785FA04F02FFF05463C
:105A20000C46FEF7CBFA04F029FF03948DE823001F
:105A300087A2182104A8F2F753FD0021012000F0ED
:105A400031FA304600F01CFB04A800F0C3FAFEF760
:105A50007BFA04F013FF04460D46FEF79FFA04F0AC
:105A60000DFF8DE833007DA2182104A8F2F738FD60
:105A70000021022000F016FA304600F001FB04A8D5
:105A800013E07AA3A2E70021012000F00BFA3046D0
:105A900000F0F6FA77A000F09DFA0021022000F055
:105AA00001FA304600F0ECFA71A000F093FA754864
:105AB00090F86A1019B100E024E073A100E073A12E
:105AC00090F869200AB170A200E070A290F86830E6
:105AD0000BB16DA300E06DA30093CDE9012190F817
:105AE000670008B168A300E068A369A2182104A8B0
:105AF000F2F7F6FC0021032000F0D4F9304600F064
:105B0000BFFA42E0664805780021084600F0CAF96D
:105B1000304600F0B5FA63A000F05CFA072D36D0ED
:105B2000082D0CD0F7F718FB012843D05FA4072DF0
:105B300063D2DFE805F06257595B5D5F61000021C9
:105B4000012000F0AFF9304600F09AFA5AA000F0B8
:105B500041FA0021022000F0A5F9304600F090FA49
:105B600058A000BF00F036FA5A4C23685AA21821F8
:105B700004A8F2F7B5FC0021032000F093F93046A9
:105B800000F07EFA2068002827DD04A826E0002126
:105B9000012000F087F9304600F072FA51A000F0C1
:105BA00019FA0021022000F07DF9304600F068FA71
:105BB00050A0D7E70021012000F074F9304600F032
:105BC0005FFA50A000F006FA0021022000F06AF906
:105BD000304600F055FA4EA0C4E725A000F0FAF9CF
:105BE0000AB070BD4DA408E050A406E052A404E041
:105BF00055A402E058A400E05BA40021012000F0BD
:105C000051F9304600F03CFA5AA000F0E3F90021C7
:105C1000022000F047F9304600F032FA204600F04A
:105C2000D9F90021032000F03DF9304600F028FAB0
:105C3000D3E700007C0000203447000025732025B6
:105C40003032753A253032753A2530327500000011
:105C5000252E31665620252E32664100252E3166CE
:105C60005720252E32666B57680000005769466939
:105C700000000000BCC6C1BFD0BEC6ACC0EBCFDFC9
:105C800000000000BC000020BFAA0000B9D800003E
:105C9000BFAAB9D83A257325732573257300000070
:105CA00090000020B6CFCDF800000000B3F5CABCCC
:105CB000BBAFD6D000000000D6C7C4DCC5E4CDF829
:105CC00000000000C7EBB4F2BFAA415050B9E3B2E4
:105CD000A500000094000020CAA3D3E0202564732F
:105CE0000000000057694669B9CCB6A8C4A3CABD74
:105CF00000000000D5FDD4DACBD1CBF7C8C8B5E39E
:105D00000000000057694669C4A3CABD0000000036
:105D1000B3F5CABCBBAFD6D02E2E2E00C4A3BFE9AC
:105D2000B8B4CEBBB3C9B9A6000000004154D6B880
:105D3000C1EEB3C9B9A6000053494DBFA8BCECB22F
:105D4000E2B3C9B9A6000000B8BDD7C5CDF8C2E717
:105D5000B3C9B9A600000000C1ACBDD3B7FECEF1F7
:105D6000C6F7D6D000000000CEDE53494DBFA821B3
:105D700000000000D5FDD4DAB5C8B4FD3447C1AA8F
:105D8000CDF8000010B54FF4C870F5F721FEFFF70D
:105D90009DFD424C002280212046F5F733FF012271
:105DA000D1033F48F5F72EFFAE21002000F030F977
:105DB0002021002000F02CF91021002000F028F90B
:105DC000B021002000F024F9C821002000F020F9C3
:105DD0000021084600F01CF91021002000F018F9FD
:105DE0004021002000F014F98121002000F010F97A
:105DF000FF21002000F00CF9A121002000F008F99B
:105E0000A621002000F004F9A821002000F000F9EC
:105E10003F21002000F0FCF8A421002000F0F8F859
:105E2000D321002000F0F4F80021084600F0F0F83B
:105E3000D521002000F0ECF8F021002000F0E8F877
:105E4000D921002000F0E4F82221002000F0E0F841
:105E5000DA21002000F0DCF81221002000F0D8F850
:105E6000DB21002000F0D4F82021002000F0D0F841
:105E70008D21002000F0CCF81421002000F0C8F89B
:105E8000AF21002000F0C4F8012280212046F5F760
:105E9000B9FEBDE81040FFF7E5BC0000001001406E
:105EA000000C014042000248C90002704170704776
:105EB000000200202DE9F04F434C89B0814694F850
:105EC00000B094F801A0F2F73AFD617801EBC00050
:105ED0006070002070E000BFA0F1B001472909D830
:105EE00009EB08025278A12A04D35E20414301F253
:105EF000AD210BE0A0F1A10102291FD809EB080296
:105F00005278A12A1AD35E204143A139501840018A
:105F100020210091C2B2C0F3072101ABC0F30740BA
:105F200002F012F901AA51465846FBF7E1FF08F1C9
:105F3000020000F0FF080AF1100037E0A0F1200194
:105F40005E2936D8214901AB01EB001010210091E8
:105F5000C2B2C0F30721000C02F0F6F85C4601AFB4
:105F6000002280211A48F5F74DFE022621465046B0
:105F7000FEF7A4FB5FF0000517F8011B012000F0FD
:105F800047F86D1CEDB2082DF6D3641C761EE4B202
:105F900016F0FF06EAD1012280210D48F5F732FE06
:105FA00008F1010000F0FF080AF1080000F0FF0A04
:105FB00003E008F10100C0B2804619F8080000288B
:105FC0008AD109B0BDE8F08F0002002080CD030027
:105FD0000010014010B50146002409E0A12A05D3B4
:105FE0004A78A12A02D3891C103401E0491C0834E4
:105FF0000A78002AF2D1FFF75DFF03E003A0FFF764
:1060000059FF0834802CF9D310BD00002000000097
:106010002DE9F047194C0E4602464FF48079494667
:106020002046F5F7EFFD002280212046F5F7EAFD36
:106030000025A7144FF40078002239462046F5F7D2
:10604000E1FD06F0800241462046F5F7DBFD012226
:1060500039462046F5F7D6FD7006060E6D1C082D54
:10606000EADB012249462046F5F7CCFD2046BDE893
:10607000F04701228021F5F7C5BD00000010014066
:1060800002494A781044487070470000000200201E
:106090002DE9F0410A4C054620880026094F85422B
:1060A00001D3268008E020887919421B0548F2F7C1
:1060B000F5FC2088401B208020883E54BDE8F081FC
:1060C00072000020442E00202DE9F04107460E46C4
:1060D00090461046F2F733FC85B2AE420CD3002452
:1060E000761B07E038192A464146F2F7D8FB30B153
:1060F000641CA4B2A642F5DA0020BDE8F08138198C
:10610000FBE72DE9F04104460E4615461046F2F72E
:1061100016FC87B2BE4224D30023F61B1FE00020EA
:1061200014E01918625C295CA2F1410CBCF1190F52
:1061300001D82032D2B2A1F1410CBCF1190F01D823
:106140002031C9B28A4203D1401C80B2B842E8D3A0
:10615000B84202D1E018BDE8F0815B1C9BB29E42C0
:10616000DDDA0020F7E7000070B59EB00546032495
:10617000164E21E0A6F87450782214490020FCF74E
:1061800033F8B0B978216846F2F726FD78226946DF
:106190000020FBF7DFFEBDF874202946AA4205D196
:1061A0000BA0FEF741FB00201EB070BD0FA0FEF754
:1061B0007FFB1420F5F70CFC641EDBD2294615A0EA
:1061C000FEF776FB4FF0FF30EEE70000BC0000204A
:1061D0003E204F544120B0E6B1BED2D1B1A3B4E6C7
:1061E000B2A2D0A3D1E93A20257500003E204F5439
:1061F0004120B0E6B1BED0A3D1E9B2BBC6A5C5E48B
:106200003A20D0B4C8EB3D25752C20B6C1C8A13DBD
:10621000257500003E204F544120B0E6B1BEB1A329
:10622000B4E6CAA7B0DC3A2025750000F8B5F7F748
:10623000BFFF050071D0B9A1FBF7D2FCB94E30B158
:10624000307808B1B8A100E0BDA1C3A059E3C7A14F
:106250002846FBF7C5FC20B9C6A12846FBF7C0FCC1
:1062600098B16879312805D000243078844203D170
:10627000C2A050E30124F8E72046FDF799FB0CB1DA
:10628000C5A100E0C8A1CDA029E0D6A12846FBF712
:10629000A7FCD54E30B1307808B1D4A100E0D6A12A
:1062A000D8A02EE3DCA12846FBF79AFC20B9DCA19C
:1062B0002846FBF795FCC8B1E878312805D00024C2
:1062C0003078844203D1D8A025E30124F8E72046A2
:1062D000FDF716FE0CB1DBA100E0DCA1DDA0FEF7AE
:1062E000E7FA0B2001F0B2FEC820B8E0E3A128468F
:1062F000FBF776FC20B1E3A0FEF7DAFA0B20ABE067
:10630000EAA12846FBF76CFCEA4C48B1009434F84B
:10631000643FE84A218A3C3200E085E0E6A081E063
:10632000F0A12846FBF75CFC08B1012105E0EFA1D4
:106330002846FBF755FC10B1002101202BE0EDA110
:106340002846FBF74DFC08B1012105E0EBA12846EA
:10635000FBF746FC10B1002102201CE0E9A1284611
:10636000FBF73EFC08B1012105E0E8A12846FBF758
:1063700037FC10B1002103200DE0E6A12846FBF711
:106380002FFC08B1012105E0E4A12846FBF728FC19
:1063900028B100210420BDE8F84001F037BDE1A19B
:1063A0002846FBF71DFC60B10121084601F02EFDD7
:1063B0000121022001F02AFD0121032001F026FD28
:1063C000E0E7DAA12846FBF70BFC60B100210120D1
:1063D00001F01CFD0021022001F018FD0021032026
:1063E00001F014FDD5E7D3A12846FBF7F9FBE0B196
:1063F00094F86A0008B1D1A000E0D1A0009094F810
:10640000690008B1CDA300E0CDA394F8680008B1FD
:10641000CAA200E0CAA294F8670008B1C7A100E0D0
:10642000C7A1C8A0FEF700FAF8BDD1A12846FBF726
:10643000D7FB20B1CFA0FEF7F7F90C200CE0D7A1D5
:106440002846FBF7CDFBA8B1F6F786FE01280AD057
:10645000D5A0FEF72DFA0D2001F0F8FD6420F5F728
:10646000B7FAF8F7BBFBDDA0FEF722FAE5490120F9
:106470000870F8BDE4A12846FBF7B2FB30B1E4A0F8
:10648000FEF7D2F9BDE8F840FAF7E2BCE8A12846E9
:10649000FBF7A6FB20B10020FEF7FCF9E7A03AE2EB
:1064A000ECA12846FBF79CFB20B10120FEF7F2F996
:1064B000EBA030E2F0A12846FBF792FB20B10220CE
:1064C000FEF7E8F9EEA026E2F2A12846FBF788FBEA
:1064D00020B10320FEF7DEF9F0A01CE2F4A128466B
:1064E000FBF77EFB20B10420FEF7D4F9F3A012E203
:1064F000F8A12846FBF774FB20B10520FEF7CAF986
:10650000F7A008E2FCA12846FBF76AFB28B1FEF7DA
:1065100085F9FA4951F82010F2E1F6E15343414C74
:1065200045000000640100205343414C453120B335
:10653000C6D6D8CDB6C1CF28B4F8B3D32900000051
:106540005343414C453020CBC4C2B7BCCCB5E7C6A1
:10655000F728CEDEB3D329003E2042543A20B2FAC7
:10656000C6B7C4A3CABD2025730000005343414CE5
:10657000453000005343414C453100003E20425419
:106580003A20D2D1CAC7B8C3C4A3CABDA3ACCEDE19
:10659000D0E8C7D0BBBB0000B3C6D6D8CDB6C1CFFC
:1065A00028B4F8B3D3290000CBC4C2B7BCCCB5E73C
:1065B000C6F728CEDEB3D329000000003E204254A7
:1065C0003A20B2FAC6B7C4A3CABDD2D1C7D0B5BDAE
:1065D000202573A3ACD6D8C6F4C9FAD0A72E2E2E88
:1065E000000000004750530070000020BFAAC6F40E
:1065F0002847505331290000B9D8B1D52847505306
:10660000302900003E2042543A2047505320B6A87B
:10661000CEBB20257300000047505330000000001F
:1066200047505331000000003E2042543A20D2D15E
:10663000CAC7B8C3D7B4CCACA3ACCEDED0E8C7D001
:10664000BBBB0000BFAAC6F400000000B9D8B1D59A
:10665000000000003E2042543A2047505320B6A884
:10666000CEBBD2D1C7D0B5BD202573A3ACD6D8C67A
:10667000F4C9FAD0A72E2E2E000000005245534533
:10668000540000003E205553415254313A20CAD59F
:10669000B5BD20524553455420C3FCC1EEA3ACD533
:1066A000FDD4DAD6D8C6F42E2E2E0000494E464F21
:1066B00000000000BC0000203E20425420494E460D
:1066C0004F3A20B0E6B1BE3D25752C20B7FECEF185
:1066D000C6F73D25733A25642C20BFCDBBA7B6CBAA
:1066E0003D25730052314F4E0000000052314F469D
:1066F0004600000052324F4E0000000052324F461A
:106700004600000052334F4E0000000052334F4607
:106710004600000052344F4E0000000052344F46F5
:1067200046000000414C4C4F4E000000414C4C4F85
:10673000464600005354415455530000BFAA000080
:10674000B9D800003E204254205354415455533A86
:10675000205357313D25732C205357323D25732C40
:10676000205357333D25732C205357343D25730058
:106770004F5441003E204254204F54413A20D6D835
:10678000C6F4BDF8C8EB20426F6F744C6F6164654E
:106790007220BCECB2E9C9FDBCB600005245434FC3
:1067A00056455259000000003E20425420524543B5
:1067B0004F564552593A20344720C4A3CABDA3AC12
:1067C000B2BBB2D9D7F7205769466920C4A3BFE945
:1067D000A3ACBDF6D6D8C6F4000000003E2042545B
:1067E000205245434F564552593A20D2D1B0B2C5F6
:1067F000C5205769466920BBD6B8B4B3F6B3A7C95C
:10680000E8D6C3009A000020424C4553455400008E
:106810003E2042543A20C7BFD6C6D6D8D0C2C9E817
:10682000D6C3C0B6D1C0C3FBB3C62F55554944002B
:106830004C4F475452414345000000003E20425413
:106840003A20C8D5D6BEB5C8BCB62054524143453F
:10685000000000004C4F47444542554700000000EF
:106860003E2042543A20C8D5D6BEB5C8BCB6204456
:1068700045425547000000004C4F47494E464F00E7
:106880003E2042543A20C8D5D6BEB5C8BCB6204931
:106890004E464F004C4F475741524E003E20425407
:1068A0003A20C8D5D6BEB5C8BCB6205741524E0016
:1068B0004C4F474552524F52000000003E20425478
:1068C0003A20C8D5D6BEB5C8BCB6204552524F52A4
:1068D000000000004C4F47464154414C000000006E
:1068E0003E2042543A20C8D5D6BEB5C8BCB62046D4
:1068F0004154414C000000004C4F47007C010020F7
:106900000AA0BDE8F840FDF78FBF0EA12846FBF7AF
:1069100067F920B10D48BDE8F840FDF785BF29466D
:10692000BDE8F8400AA0FDF7C3BF00003E20425476
:106930003A20B5B1C7B0C8D5D6BEB5C8BCB62025BB
:106940007300000048454C5000000000F0B90108F9
:106950003E2042543A20CEB4D6AAC3FCC1EE202534
:1069600073000000F0B599B0174660236A4600F046
:106970006BF9002833D06846F1F7E1FF6C462546F5
:106980000DEB000622E0201D86420DD3042217A144
:106990002046F1F7F3FF38B9AC4203D014F8010CEC
:1069A000222801D001201DE0601D86420DD3052262
:1069B00010A12046F1F7E2FF38B9AC4203D014F839
:1069C000010C222801D000200CE0641CA642DAD879
:1069D0009DF80000302804D0312802D0002019B0E2
:1069E000F0BD303838600120F9E700007472756539
:1069F0000000000066616C736500000070B514460D
:106A000000F0EBF800221346002820D0017822295C
:106A100000D1401C0178A1F13005092D01D8E9B25F
:106A20000BE0A1F16105052D01D8573904E0A1F172
:106A30004105052D08D83739C9B241EA0211401C79
:106A40005B1C8AB2042BE5DB13B12280012070BDF0
:106A5000002070BD70B50D46144617A100F0BDF8BA
:106A6000002330B3002C24DD0178641E222913D1C9
:106A7000401C01E0E9545B1CA34214DAC15CA1F1A3
:106A80003002092AF6D9313A192AF3D92032192AC3
:106A9000F0D908E0E9545B1CA34204DAC15C302958
:106AA00001D33929F6D90020E854002B01DD01205B
:106AB00070BD002070BD00006964000030B591B069
:106AC0001546002440236A4600F0BEF800281BD07B
:106AD00020A1684600F081F810B9684600E0401C2B
:106AE00001782029FBD00929F9D00D29F7D00A29EE
:106AF000F5D02229F3D03A29F1D0CAB2303A6FF05A
:106B00002F010A2A09D3002011B030BD04EB840301
:106B100001EB43031A4494B2401C0278A2F1300303
:106B2000092BF3D9D3B24FF6FF722E2B0BD140783D
:106B3000A0F13003092B06D804EB840201EB4201DB
:106B4000084480B203E004EB840002EA400028809D
:106B50000120D9E776616C756500000070B51C46B0
:106B6000154600F03AF80021A8B10278222A12D185
:106B7000002C10DD401C641E01E06A54491C425C7C
:106B80001AB1222A01D0A142F7DB00206854002963
:106B900001DD012070BD002070BD000070B51446FD
:106BA00000F01BF8002120B10278302A01D3392AE5
:106BB00009D9002070BD00BF01EB810103EB410149
:106BC0001144401C01E06FF02F030278A2F1300560
:106BD000092DF1D90120216070BDF0B5054687B0BF
:106BE0000E460846F1F7ABFE041E23DDE01C182814
:106BF00020DC314622276E468DF800702246701C3C
:106C0000F1F707FF30190021477081700CE0281957
:106C1000801C00E0401C01782029FBD00929F9D014
:106C2000C9B23A2909D0AD1C69462846F1F725FEBC
:106C30000500ECD1002007B0F0BD10F8011F20299D
:106C4000FBD00929F9D0F6E770B51D461646FFF7C7
:106C5000C4FF00210C46002819D06D1E425C9AB179
:106C6000A94211DA7B2A04D07D2A04D02C2A07D02D
:106C700007E0641C05E03CB1641E02D1491C03E03E
:106C800014B17254491CE9E700207054012070BD12
:106C90002DE9F041184C0F46054626692068001D75
:106CA00001F0D8FC38B9206890F82C1001208840F9
:106CB000616981436161681C07D137B12168BDE812
:106CC000F0410E48091D01F035BD20683544B5423C
:106CD0004560216805D2A068BDE8F041091D01F0BA
:106CE00011BD6068091D01F00DFDE06A854200D20A
:106CF000E562BDE8F081000000000020E402002011
:106D00002DE9F041054601F021FD2C4CE068401CC6
:106D1000E06020682A4F10B1A06920B329E0256007
:106D2000E068012825D1002606EB860007EB8000ED
:106D300001F0DAFC761C052EF6D32148643001F010
:106D4000D3FC1F48783001F0CFFC1D488C3001F097
:106D5000CBFC1B48A03001F0C7FC194864306060D0
:106D60001430A06005E02068E96AC06A884200D853
:106D70002560A06A401CA062E96A0120626988401F
:106D80001043606101EB810007EB8000291D01F0D9
:106D9000D1FC01F0FBFCA06900280CD02068E96A56
:106DA000C06A884207D207494FF080500860BFF39D
:106DB0004F8FBFF36F8FBDE8F0810000000000200F
:106DC0004402002004ED00E02DE9F041856B1746F8
:106DD00004460026026C82B1C7B1E068F1F719FEE3
:106DE000E168206C091AE1602268914202D2616870
:106DF000081AE060022F16D017E02068A8B9606872
:106E000002F070FD0646002060600EE0A068F1F719
:106E100000FE216CA0680844A0606168884204D329
:106E20002068A06001E005B16D1E6D1CA5633046B1
:106E3000BDE8F08110484FF42051420706D0C01D34
:106E40000D4920F00700411AC1F520510B4A0023DB
:106E50000144C2E900030839103A21F0070111602A
:106E60004B600B600B1AC0E9001393604FF00040B9
:106E70005360D06070470000F802002054000020EA
:106E8000074C084D4FF080562068012804D92E6029
:106E9000BFF34F8FBFF36F8F01F0EFFBF4E70000FC
:106EA0004402002004ED00E02DE9F0470E46DDE944
:106EB00009841746824691009946089DA522206BB9
:106EC000F1F760FE6FF00301206B01EB87010844CE
:106ED00020F00707780707D0502080F31188BFF310
:106EE0004F8FBFF36F8FFEE72218315C82F83410AA
:106EF000315C11B1401C1028F6D3002684F84360A1
:106F0000052D00D30425E562C4E91156201D01F0CA
:106F1000F6FB04F1180001F0F2FB2461C5F1050055
:106F20006462A061E66484F850604A46514638467F
:106F300000F02AF92060B8F1000F01D0C8F8004035
:106F4000BDE8F08730B5114900E011460A68824279
:106F5000FBD34B685C18844203D1406818444860F6
:106F6000084643681C18944209D1084C103C246818
:106F7000A24209D052681A4442600A68126802604C
:106F8000814200D0086030BD0460F9E75400002061
:106F900010B5044601F0DAFBA06B28B15FF00004E5
:106FA00001F0F4FB204610BD0124F9E706484168D2
:106FB000096829B14168C968C9684968C1627047F0
:106FC0004FF0FF31FAE70000000000200848406859
:106FD000401C4FF0500080F3118804D0BFF34F8F56
:106FE000BFF36F8FFEE7BFF34F8FBFF36F8FFEE7E7
:106FF000380000202DE9F041044601F0A7FB94F988
:10700000455004F1240609E0606A48B1304602F0B8
:10701000FFFC08B101F03CFC6D1E6DB2002DF3DCED
:107020004FF0FF3684F8456001F0B0FB01F08EFBB5
:1070300094F9445004F1100709E0206948B138463A
:1070400002F0E6FC08B101F023FC6D1E6DB2002DCC
:10705000F3DC84F84460BDE8F04101F097BB2DE912
:10706000F04105460E4617461046F1F768FC84B21B
:10707000200AA855761CB0B222462C54401C86B279
:10708000A8193946F1F7C5FC301980B2BDE8F08186
:107090002DE9F0410546002701F0A0FC334E306891
:1070A00008B9FFF7C7FEF068054216D1ADB1083543
:1070B00068070ED005F00700C0F108000544680716
:1070C00007D0502080F31188BFF34F8FBFF36F8F2D
:1070D000FEE715B17068854202D902F0D3FC36E0B4
:1070E0002248103001460C6801E020460C466168D9
:1070F000A94202D221680029F7D131688C42ECD034
:1071000007682168016060680837411B10290ED9A3
:107110006019420707D0502080F31188BFF34F8FCA
:10712000BFF36F8FFEE741606560FFF70BFF61689B
:107130007068401A7060B268904200D2B060F06827
:1071400001430020C4E9000102F09CFC0FB901F0EA
:1071500097FA780707D0502080F31188BFF34F8F3C
:10716000BFF36F8FFEE73846BDE8F0814400002092
:107170000449086818B10868826C521C8264086867
:10718000704700000000002010B5031F4FF080740E
:107190001C601B1F21F001011960191F024B0B60BD
:1071A000143940380A6010BDCD6F010812282CD266
:1071B000DFE800F02B090B0D0F11131517191B1D1C
:1071C0001F212325292712A0704715A0704717A05B
:1071D00070471AA070471DA0704722A0704725A0D5
:1071E000704726A0704728A070472BA070472EA09C
:1071F000704731A0704733A0704737A070473CA05C
:10720000704740A0704742A0704746A070470000FA
:10721000C9CFB5E72FD2E2CDE2B5F4B5E700000063
:10722000B0B4BCFCB8B4CEBB00000000BFA8CBC05B
:10723000BFB4C3C5B9B7D2E7B3F60000B1BBC6BD92
:10724000CCA8CCDFCFC2CFDF00000000D0C4CCF888
:10725000B3ACCAB128B7FECEF1C6F7CEDECFECD3C1
:10726000A62900003447CEDECDF8C2E7B7FECEF146
:1072700000000000CEDE53494DBFA8004F5441C965
:10728000FDBCB6CDEAB3C9004F5441BDA1BFB5BCEA
:10729000ECB2E9B3ACCAB1003447B3F5CABCBBAF7A
:1072A000CAA7B0DC00000000B4AEBFDA52455345B7
:1072B00054C3FCC1EE000000B4AEBFDA4F5441C36A
:1072C000FCC1EE00B4AEBFDA5245434F56455259A9
:1072D000C3FCC1EE00000000CDE2B2BFB6CFB5E7FF
:1072E00028B7A8C0ADB5E7C8DDBCC7C2BC2900003F
:1072F0003447C4A3D7E9D2ECB3A3D7D4D6D8C6F4C5
:10730000000000004F5441CAA7B0DCD6D0D6B90067
:10731000C8EDBCFEB8B4CEBB28CEB4B1EABCC72918
:1073200000000000CEB4D6AA000000004FF4801286
:1073300002EB00302022F7F7DFBA024600200146B8
:10734000535C491C184480B20E29F9DB70470000D9
:1073500010B5044600680649884207D12046FFF769
:10736000ECFF218A884201D1012010BD002010BD10
:107370004C54535270B504460D460846FFF7DDFFE6
:1073800028824FF4801000EB043401122046F7F7F6
:10739000D4F820462946BDE870402022F7F7A2BB6A
:1073A0002DE9F0418AB08046142101A8F1F714FCC0
:1073B000414692A0FDF738FA142201A94046FFF792
:1073C00049FBA0B192A14046F1F757FA914E002532
:1073D000002843D08EA140460895F1F74EFAC078B8
:1073E0003038C4B2601E042803D38BA003E194A0FC
:1073F00001E173208DF81C0077208DF81D0004F149
:1074000030008DF81E008DF81F5008AA07A94046CD
:10741000FFF7A8FA88B1204600F0A2FB07463078B3
:1074200008B1012C0FD00898C1B2204600F072FCC0
:10743000089800280CD088A20BE0214687A0FDF711
:1074400037FA8CA2C2E08FA0FDF732FA9AA2BDE013
:10745000A0A22146A0A0FDF7E7F967E0A1A1404660
:10746000F1F70BFA00287BD008AAA1A140460895A5
:10747000FFF778FA88B30124204600F071FB074635
:107480003078002808982ED000284AD0FBF75EFDFF
:10749000002837D0ADF81C5007AA97A14046FFF747
:1074A0000DFBBDF81C00002831D0FBF709FF00BF21
:1074B000BDF81C0000282FD003F052FB904903F0C8
:1074C00071FA03F0DBF902460B468EA0FDF7ACF92A
:1074D000BDF81C00FBF774FF28E0FFE792A0FDF762
:1074E000E7F998A272E028B10121084600F012FCE9
:1074F00099A004E00021012000F00CFC9EA0FDF703
:1075000093F913E0A4A0FDF7D3F9ACA25EE0FBF77A
:1075100017FDADF81C00CBE7ADA0FDF7C9F9B6A289
:1075200054E0B8A0FDF780F9FCF712F80722BA4939
:107530006620FAF759FEB94D01206870F4F768FB30
:10754000A860AC70EF701421B548F1F723FB13224B
:1075500001A9B348F1F75DFA0AB0BDE8F081FFE791
:1075600065A14046FFF739FB41F28834B8B1307865
:1075700080B1ADF800506A465FA14046FFF79EFA21
:10758000BDF8000008B1A04206D9A6A0FDF790F909
:10759000AAA21BE0ADA01FE0FBF792FE22E0B4A17F
:1075A0004046FFF71AFB28B33078A0B1ADF8005081
:1075B0006A46AFA14046FFF781FABDF8000008B166
:1075C000A0420DD9ACA0FDF773F9B0A2002101A82B
:1075D000F6F734F9C0E7B1A0FDF76AF9B7A2F5E70D
:1075E000FBF7A0FEBBA2012101A8F6F727F900F0E6
:1075F000C9FBB1E7B8A0FDF75BF9ADE73E20BCCC15
:10760000B5E7C6F7C3FCC1EE3A20252E383073002B
:1076100022737700640100203E20BCCCB5E7C6F79A
:107620003A20737720B1E0BAC5CEDED0A7A3ACBDB7
:10763000F6D6A7B3D6207377317E73773400000077
:107640003E20BCCCB5E7C6F73A20696420BDE2CE47
:10765000F6CAA7B0DC000000BFAA00003E20BCCCE8
:10766000B5E7C6F73A207377256420D6B5CEDED0CD
:10767000A70000006261642073772076616C7565F5
:10768000000000003E20BCCCB5E7C6F73A20B3C6E8
:10769000D6D8CDB6CEB9C4A3CABDCFC2BAF6C2D46D
:1076A00020737731A3ACC7EBD3C3206665656469EB
:1076B0006E6720D6B8C1EE007377312064697361BC
:1076C000626C65642C207573652066656564696EFF
:1076D00067000000B9D800003E20535725642025DC
:1076E000730000002266656564696E672200000011
:1076F00066656564696E67006F6E63655774000048
:10770000000020413E20BCCCB5E7C6F73A20BFAA16
:10771000CABCCDB6CEB9A3AC6F6E636557743D25B8
:107720002E31664B470000003E20BCCCB5E7C6F7C3
:107730003A2066656564696E6720D6B5CEDED0A74F
:10774000000000006261642066656564696E672000
:1077500076616C75650000003E20BCCCB5E7C6F7CD
:107760003A20CAD6B6AFCDB6CEB9BFAAA3A8CEDE50
:10777000B3D3A3A9000000003E20BCCCB5E7C6F7F8
:107780003A20CAD6B6AFCDB6CEB9B9D8A3A8CEDE08
:10779000B3D3A3A9000000003E20BCCCB5E7C6F7D8
:1077A0003A20BEDCBEF8C6F4B6AFCDB6CEB9A3ACB7
:1077B000D6D8C1BFCEB4BECDD0F70000776569671B
:1077C0006874206E6F742072656164790000000037
:1077D0003E20BCCCB5E7C6F73A20CEDE206F6E6304
:1077E00065577420B5A5B4CECDB6CEB9C1BFA3AC94
:1077F000D2D1BAF6C2D400006E6F206F6E636557A7
:10780000740000003E20BCCCB5E7C6F73A20CDA3FB
:10781000D6B9CDB6CEB9000022010020A8000020C4
:10782000B66600203E20BCCCB5E7C6F73A206F6EA6
:107830006365577420CEDED0A7000000696E7661C4
:107840006C6964206F6E6365577400003E20BCCC89
:10785000B5E7C6F73A20BEDCBEF8C9E8D6C3206F4C
:107860006E63655774A3A8CEDEB3D3A3A90000004E
:107870007A65726F000000003E20BCCCB5E7C6F709
:107880003A207A65726F20CEDED0A700696E7661ED
:107890006C6964207A65726F000000003E20BCCCE9
:1078A000B5E7C6F73A20BEDCBEF8C9E8D6C3207AF1
:1078B00065726FA3A8CEDEB3D3A3A9006E6F207349
:1078C00063616C65206F6E207468697320646576EF
:1078D000696365004F4B00003E20BCCCB5E7C6F79E
:1078E0003A20CEB4D6AAD6B8C1EEA3A8CEDE207375
:1078F000772F66656564696E672F7A65726FA3A9D5
:107900000000000070B51E4CA578607800282FD0CC
:10791000607801282CD1F4F77BF9A168401A64281B
:1079200026D3284600F01CF9064600F00DF910B1E8
:10793000294614A00AE01C48284490F86600002854
:10794000E07816D038B9012E17D004E0FCF76CFFB0
:1079500016A2012105E0294615A0FCF7A9FF1DA2EA
:1079600000212548F5F76AFF00F00CFA002060704E
:1079700070BD0128EFD1002EEDD129461FA0E5E70B
:10798000A80000203E20BCCCB5E7C6F73A205357EC
:10799000256420B6AFD7F7D5FDB3A3A3A8CAD6B642
:1079A000AFC4A3CABDA3A900BC0000204F4B000078
:1079B0003E20BCCCB5E7C6F73A205357256420CE0D
:1079C000B4BDD3B8BAD4D8BBF2BCCCB5E7C6F7B611
:1079D000CFBFAA004C6F616420756E706F776572BF
:1079E0006564202F2072656C6179206661696C7511
:1079F0007265202100000000B66600203E20BCCC4D
:107A0000B5E7C6F73A205357256420B6AFD7F7D568
:107A1000FDB3A3002DE9F04786B03F4C0025029549
:107A2000A06940F00800A061A06900F0080004907F
:107A3000A06940F01000A061A069022700F01000CA
:107A4000CDE9037001268020CDE90006DFF8CCA047
:107A500069465046F3F7CEFF4FF4807869465046AA
:107A6000CDF80080F3F7C6FFDFF8B49069464846CA
:107A70000096F3F7BFFF0420009069464846F3F7ED
:107A8000B9FF40208DE8610069465046F3F7B2FF28
:107A90006015009069465046F3F7ACFF69464846CA
:107AA0000097F3F7A7FF0820009069464846F3F7D0
:107AB000A1FFA06940F00400A061A069CDF800809A
:107AC00000F004000490CDE9015769461548F3F72A
:107AD00091FF002280215046F4F794F812A0FCF7A1
:107AE000A3FE002241465046F4F78CF810A0FCF7A4
:107AF0009BFE002201214846F4F784F80EA0FCF713
:107B000093FE002204214846F4F77CF80CA0FCF711
:107B10008BFE06B0BDE8F08700100240000C01406B
:107B200000100140000801405357313AB9D8000015
:107B30005357323AB9D800005357333AB9D80000F6
:107B40005357343AB9D8000010B54FF48071034848
:107B5000F4F74CF8012800D0002010BD00080140C7
:107B600001460B48012908D0022908D009480329F9
:107B700008D0042908D000207047402105E04FF4C8
:107B8000007102E0022100E00821F4F72FB80000A4
:107B9000000C01400010014010B5F4F739F802491B
:107BA00048600120087010BDA800002070B52D4865
:107BB0002D4D2E4C007848B1002084F86700024615
:107BC00080212846F4F71EF829A00FE094F86700FA
:107BD00030B1012280212846F4F714F82CA005E0EA
:107BE000002280212846F4F70DF82DA0FCF71CFE9A
:107BF00094F868004FF4807128B101222846F4F708
:107C000001F82BA004E000222846F3F7FBFF2CA08C
:107C1000FCF70AFE94F869002D4D30B1012211469F
:107C20002846F3F7EFFF2BA005E0002201212846AC
:107C3000F3F7E8FF2BA0FCF7F7FD94F86A0030B1EA
:107C4000012204212846F3F7DDFF2AA005E00022E7
:107C500004212846F3F7D6FF2AA0BDE87040FCF7C0
:107C6000E3BD000064010020000C0140BC000020C6
:107C70005357313AB9D8A3A8B2BBBBD6B8B4A3AC5A
:107C8000CDB6CEB9B0B2C8ABB1A3BBA4A3A9000016
:107C90005357313ABFAAA3A8BBD6B8B4A3A90000D2
:107CA0005357313AB9D8A3A8BBD6B8B4A3A900009A
:107CB0005357323ABFAAA3A8BBD6B8B4A3A90000B1
:107CC0005357323AB9D8A3A8BBD6B8B4A3A9000079
:107CD000001001405357333ABFAAA3A8BBD6B8B48B
:107CE000A3A900005357333AB9D8A3A8BBD6B8B458
:107CF000A3A900005357343ABFAAA3A8BBD6B8B46F
:107D0000A3A900005357343AB9D8A3A8BBD6B8B436
:107D1000A3A90000421E042A2DD209B1012200E0CD
:107D20000022154B0128034483F86620134B09D029
:107D300002280DD0124B032812D004281BD1A9B160
:107D4000012214E009B1012200E0002280210FE0AD
:107D50004FF4807009B1012200E00022014607E0E3
:107D600009B1012200E00022012101E000220421EA
:107D70001846F3F747BF7047BC000020000C0140D5
:107D8000001001407FB5FBF7E1F802F0E9FE1D4E5F
:107D9000314602F007FE0446FBF7D2F802F0E0FE9F
:107DA000314602F0FFFD0546FBF7D6F802F0D8FE9B
:107DB000314602F0F7FD1449024691F86A0000B11D
:107DC000012003948DE8250091F8690008B1012392
:107DD00000E0002391F8680008B1012200E00022D1
:107DE00091F86700002802D04FF0010101E04FF048
:107DF000000102D04FF0010001E04FF00000F5F764
:107E000091FD7FBD00002041BC00002070B50446FC
:107E1000401E0D46042813D22046FFF77BFF0DB10C
:107E200008A200E008A2214608A0FCF7FDFC0722FA
:107E30000A496620FAF7D8F9BDE87040FFF7ACBEF2
:107E400070BD0000BFAA0000B9D800003E20425417
:107E50003A2053572564202573000000220100209A
:107E60002DE9F04300248DB0661EF9F741F9DFF8E3
:107E7000349109F10405D0B1A9F104000068D9F8E2
:107E80000060C10006D5286810B12868C4B20EE0B1
:107E900010240CE0810001D4410001D5032406E048
:107EA000410101D5022402E0000100D5012409A806
:107EB000FBF790FD07004FF000080BD4F8B26946BD
:107EC000FFF734FA9DF808000E2803D19DF8090049
:107ED000FF281ED031462046F8F7A4FEC5F80080E2
:107EE000C9F800802F48304908380160F9F7F8F8E0
:107EF0002C49083108602DA0FCF796FC0BA8FBF775
:107F000069FD05000FD530A0FCF78EFC0DB0BDE873
:107F1000F0838DF80980F8B26946FFF72BFA2EA09E
:107F2000FCF782FCDAE700240A26281B0A3090FBC3
:107F3000F6F106FB1100C0B202A9FFF7F7F902A89B
:107F4000FFF706FA00B30598401C21D005983C21A4
:107F5000B0FBF1F0B0FBF1F201FB12094FF4B46297
:107F6000B0FBF2F302FB1303B0FBF2F7B3FBF1F843
:107F70009DF81000FFF71AF902463B46611C1DA050
:107F8000CDE90089FCF750FC641C0A2CCDDBBDE771
:107F90009DF81000FFF70AF90246611C22A0FCF7C9
:107FA00043FCF1E708BF0020524853523E20C0FA7C
:107FB000CAB7D6D8C6F4BCC7C2BCA3A8D0C2A1FA5F
:107FC000BEC9A3A93A0000002020A3A8CEDEBCC7EA
:107FD000C2BCA3A9000000003E20C9CFB4CECEAAE7
:107FE000B6CFB5E7B9D8BBFAA3A8D2D1BCC7C2BC3B
:107FF000A3A9000020205B25645D20D6D8C6F4D458
:10800000ADD2F23A2025732020D4CBD0D0CAB1BC57
:10801000E43A202575CCEC25303275D0A1CAB125C3
:10802000303275B7D600000020205B25645D20D675
:10803000D8C6F4D4ADD2F23A2025732020D4CBD0C8
:10804000D0CAB1BCE43A20CEB4D6AA0010B50446DA
:10805000FCF79CF90448046003480C38F9F740F831
:108060000149091D086010BD0CBF0020F8B5F9F7E3
:108070003FF810B11148046801E04FF0FF343C2094
:10808000B4FBF0F2B4FBF0F100FB1245B1FBF0F2EF
:1080900000FB12134FF4B466B1FBF6F206FB1212AA
:1080A000B2FBF0F2B1FBF6F105480095FCF700FCDD
:1080B0002146BDE8F8400E20F8F7B4BD08BF002007
:1080C000C0BA0108054910B5086004480838F9F736
:1080D00007F802490831086010BD000008BF002001
:1080E0002DE9FF410122174D170300243946284688
:1080F000F3F788FD0020019002900390402000904B
:1081000069462846F3F776FC0026002239462846C1
:10811000F3F778FD6006040E40212846F3F766FD6C
:1081200008B144F00104012239462846F3F76AFDFC
:10813000761C082EE9DBFBF799FC04B02046BDE86D
:10814000F0810000001001402DE9F05FDFF8689039
:1081500092468B4607464FF400481D460022414692
:1081600048460A9EF3F74EFD144C0122802120461A
:10817000F3F748FD0022A1142046F3F743FD032046
:1081800000F01EF8384600F01BF8584600F018F8CA
:10819000504600F015F8002405E000BFFFF7A0FFEF
:1081A0002855641CE4B2B442F8D341464846BDE8C1
:1081B000F05F0122F3F726BD000C014000100140E2
:1081C0002DE9F0410E4E002405464FF40078B71417
:1081D00005F0800241463046F3F714FD6806050EAF
:1081E000002239463046F3F70DFD0122394630466C
:1081F000F3F708FD641C082CEADBBDE8F081000001
:108200000010014000B5254B21F0004287B09A4292
:1082100003DC0022134600922BE0214B9A4208D146
:1082200040B94FF00100F0F77EFDF6F7FAFF07B016
:1082300000BD03DBF6F7F2FF07B000BD02AAF6F7B8
:10824000DFFC10F003014FF001000DD0012914D024
:1082500002291AD00DF1080C9CE80F00F6F794FEE5
:1082600007B081F0004100BD0DF1080C00909CE8C2
:108270000F00F6F75DFF07B000BD0DF1080C9CE89C
:108280000F00F6F781FE07B000BD0DF1080C00905D
:108290009CE80F00F6F74CFFE2E70000FB21E93F06
:1082A0000000F07F2DE9F04106460F4602F016F976
:1082B00004000D4618BF0120284320F00040C0F103
:1082C0007F6000F1E040C00F0ED0301C18BF0120CD
:1082D000384320F00040C0F17F6000F1E040C00F63
:1082E00004BF0120F0F71FFD20462946BDE8F081BC
:1082F00010B5074CA068002809D001F081FA0228C7
:1083000005D1C11EA068BDE8104001F0EDB910BD57
:108310009401002010B5042000F0E0FF01498860BE
:1083200010BD00009401002010B5074CA068002883
:1083300008D001F065FA022804D1A068BDE8104019
:1083400001F0F6B810BD00009401002088B0F3F7EA
:108350005FFC8246F3F75CFC8346F3F759FC064664
:10836000F3F756FC8146F3F753FC00252C464FF4F7
:108370007A78544FCDF81800FDF758FF387808B1D7
:10838000012100E0002150480170F7F70BF8F3F7E6
:108390003FFCA0EB0B00322804D3F3F739FC8346F3
:1083A00000F09CF8F3F734FCA0EB0A0040450FD333
:1083B000F3F72EFC8246FCF703F82846FDF7EAFAAD
:1083C0004246002328462146EFF7E2FFFFF77AFEF8
:1083D000F3F71EFC821B551944F10004A0EB0901C0
:1083E0004EF660220646914219D33878B146B0B1B4
:1083F000002328462146EFF7CBFF3C22B0FBF2F1E9
:1084000002FB11034FF4B461B0FBF1FC01FB1C0C47
:10841000B0FBF1F1BCFBF2F22C48FCF705FA38781E
:10842000F0B3FBF735FED8B3F3F7F2FB0699401A29
:1084300042F2107188423CD3F3F7EAFB0690FBF757
:1084400083FD0790FBF7AAFD00902148807940B397
:1084500020490098884210DDF3F7DAFB1C49C9690E
:10846000401A47F23051884207D300BFF3F7D0FBE0
:108470001749C8610798F5F7EBF8009802F0FEF984
:10848000CDE90401FBF74EFD02F0F8F9CDE9020158
:10849000FBF794FD02F0F2F9CDE90001079801E045
:1084A00007E00AE002F0EAF902460B460A48FCF748
:1084B000BBF9142000F0BEF95EE705490120887180
:1084C000D4E700007C0000203801002014B001082F
:1084D000940100200000204139B001082DE9F05F2F
:1084E000FBF7C8FC01F024FE4FF06632474B01F069
:1084F000B5FE01F055FB464902F046FB02F0BEF91D
:108500004FF03332434B01F07DFB01F049FB02F0A9
:10851000B5F9414A414B02F0C7F80022404B01F047
:108520009DFEDFF804813F4A434601F027FC01F03D
:1085300037FB3E4E3E4F044610F1FF4F01D300245F
:1085400004E03C4884425EDCBC425CDA30780028BF
:1085500059D1DFF8C8B0DFF8C8A0DFF8C89000250F
:108560003220F3F735FAFBF785FC01F0E1FD4FF01F
:108570006632264B01F072FE01F012FB02F07EF92A
:1085800000222D4B01F06AFE4FF03332214B01F0F7
:1085900039FB01F005FB02F071F91F4A5B4602F05E
:1085A00083F80022534601F059FE4A46434601F043
:1085B000E5FB01F0F5FAB84225DA6D1C022DCFDBA0
:1085C0000020F5F7CFF800281DD10120307020469B
:1085D00002F0AAFA014619A0FCF726F9FBF7D6FE2D
:1085E000FFF744FD4FF4FA70F3F7F2F9BFF34F8F42
:1085F00016480168164A01F4E06111430160BFF3B7
:108600004F8F00BFFDE7BDE8F09F000066664A3F60
:10861000000030413333E33F9A9999999999254065
:1086200000005940C8CCCCCCCCCCFC3F340100205D
:10863000000020410000C842000026403E20B5E76F
:10864000C1BFB5CD3A202564252500000CED00E022
:108650000400FA05D0E9013201699A60D0E90123EA
:108660005A604A68824201D182684A6000220261EF
:108670000868401E086008687047F4F723BC0000D3
:1086800005A0FCF7BBF8502080F31188BFF34F8F93
:10869000BFF36F8FFEE700003E2052544F533A2045
:1086A0006D616C6C6F6320CAA7B0DCA3A8B6D1BAA9
:1086B000C4BEA1A3A900000005A0FCF79FF85020AC
:1086C00080F31188BFF34F8FBFF36F8FFEE7000079
:1086D0003E2052544F533A20C8CECEF1202573206D
:1086E000D5BBD2E7B3F6000000F108014FF0FF322E
:1086F000C0E90112C16001610021016070470021E1
:108700000161704730B50B685A1C02D000F10802B5
:1087100002E0026904E02246546825689D42FAD9C5
:1087200053684B6099608A60516008610168491C18
:10873000016030BD42684A6093688B6093685960FD
:10874000916008610168491C01607047502080F306
:108750001188BFF34F8FBFF36F8F0A494868401CE1
:10876000486001280CD10848006810F0FF0F07D0BE
:10877000502080F31188BFF34F8FBFF36F8FFEE758
:10878000704700003800002004ED00E00849486808
:1087900028B1401E486001D180F3118870475020F5
:1087A00080F31188BFF34F8FBFF36F8FFEE7000098
:1087B0003800002070B5002827D0144DA0F108041F
:1087C0006168E868014207D1502080F31188BFF347
:1087D0004F8FBFF36F8FFEE722683AB1502080F3CE
:1087E0001188BFF34F8FBFF36F8FFEE78143616046
:1087F00000F0F4F860686968084468602046FEF795
:10880000A1FBBDE8704001F03DB970BD44000020FF
:108810004FF0E02000210161816105494FF47A7237
:108820000968B1FBF2F1491E4161072101617047FE
:108830006800002010B5020014D00F48406B38B11A
:10884000502080F31188BFF34F8FBFF36F8FFEE787
:1088500000F0C4F800211046FEF71AFA01F012F9F0
:10886000002807D105494FF080500860BFF34F8FB3
:10887000BFF36F8F10BD00000000002004ED00E08A
:1088800002494A6A0260096941607047000000209D
:1088900001490120086270470000002010B50C4615
:1088A00050B1094909681831FFF72CFF2046BDE88F
:1088B00010400121FEF7ECB9502080F31188BFF37E
:1088C0004F8FBFF36F8FFEE70000002070B50400EC
:1088D0004BD0A26CA2B1606C884200D30146E06A22
:1088E000884242D0012A40D1204D2A6894420FD1BB
:1088F000502080F31188BFF34F8FBFF36F8FFEE7D7
:10890000502080F31188BFF34F8FBFF36F8FFEE7C6
:10891000E162A269002A02DBC1F10501A161144EE6
:1089200000EB8000616906EB800081421DD1201DB3
:10893000FFF790FE012150B9E06A00EB800256F883
:10894000222022B96A6901FA00F082436A61E06A72
:108950006A6981401143696100EB800006EB800089
:10896000211DBDE87040FFF7E5BE70BD000000208E
:10897000440200201CB515480024CDE900402346E0
:10898000802213A1144800F009FF012809D0401CDF
:108990001AD1502080F31188BFF34F8FBFF36F8F30
:1089A000FEE7502080F31188BFF34F8FBFF36F8F26
:1089B00006484FF0FF313038C16201218161046106
:1089C000BDE81C4000F036BC1CBD0000300000209B
:1089D00049444C4500000000816E01080248416B8B
:1089E000491C4163704700000000002010B51F4C77
:1089F000606B10B10120206210BD00202062206851
:108A00004FF0A531006B02688A4208D142688A4261
:108A100005D182688A4202D1C068884204D02168A8
:108A200020683431FFF748FE60691149B0FA80F0E0
:108A3000C0F11F0000EB800051F820206AB101EB6B
:108A4000800000F10802416849684160914201D10B
:108A500049684160C868206010BD502080F31188CB
:108A6000BFF34F8FBFF36F8FFEE7000000000020C1
:108A7000440200202DE9F04F14461D468BB00646F7
:108A80000F465A4A5A4B01F0ADFB14D3594A5A4B80
:108A90003046394601F0E0FC0DD3584A584B204689
:108AA000294601F09FFB06D3564A574B20462946DC
:108AB00001F0D2FC08D21498C0E900671598C0E90B
:108AC00000450BB0BDE8F08F0022504B20462946F0
:108AD00001F0EAFD8046894600224D4B304639467A
:108AE00001F0E2FD8B46824642464B46FAF7CEFF46
:108AF000CDE9040142464B4650465946FBF7C2F8C1
:108B0000CDE900010022434B2046294601F036F909
:108B1000414A424B01F0A2FBCDE90601FFF772FB8F
:108B200081468A463E4A3F4B01F098FB4A465346EF
:108B300001F094FB00223C4B01F0C4FC82468B46C2
:108B4000FFF7B0FB8146884652465B4601F086FB44
:108B500002460B463548364901F010F92E4A2F4B94
:108B600001F07CFB82468B46DDE904010022294BA3
:108B700001F074FB52465B4601F000F98B4604900D
:108B8000DDE90601F9F766F8824607914A46434651
:108B90004FF08040274901F0F1F85246079B01F061
:108BA0005DFB1D4A1D4B01F059FB80468946DDE9FE
:108BB00000010022174B01F051FB42464B4601F0E9
:108BC000DDF8804689465B4620462946049A01F036
:108BD00019F8159A4B46C2E900014246304639461B
:108BE00001F010F8149AC2E900016AE7C74B37890F
:108BF00041005240143FC6DCB53A614061545227EF
:108C0000A089EA3FC442AD69DEE94B4000804140A3
:108C100000405A4000806640182D4454FB21094012
:108C20000BEF80AF8F6A7B3F0000F03FC155E32D13
:108C3000102B5841C15458412DE9FF4F0024BDB0BD
:108C4000601E8946A2464FF6FF7B3C90F9F7ECFC8C
:108C50001FFA89F13D98F9F773FB18B1A9A0FBF74A
:108C600027FE4CE140F6FF30DFF8B88203E05045C4
:108C700001D3AAF101003D9ACDE90240CDE90029D6
:108C8000A94AE02104A83F9BEFF72AFCF9F76AFF05
:108C900004A8EFF754FE81B204A8F9F7CFFFF2F76A
:108CA000B7FF054643F69826474620E03220F7F7FF
:108CB000FAFF39889DA2B8469E48FDF705FA60B1D3
:108CC0009C49461A361D17D005229BA19948EFF7FB
:108CD00055FEB0B121469AA010E0B8F800109FA24E
:108CE0009448FDF7F1F910B121469EA006E0F2F795
:108CF0008FFF401BB042D9D32146A2A0FBF7D8FD7D
:108D0000FDE0A7A210218B48FDF7DEF918B1BAF1FA
:108D1000000F09D036E00021782E00D37826854850
:108D200081550146A0A0E9E7B1B2ADA28148FDF7A7
:108D3000E8F960B12F21EFF796FD40B1401CEFF745
:108D400085FD5FEA000A02D0BAF5603F02D95146BC
:108D5000A7A0D3E7AEA0FBF767FDB7A0FBF764FDC4
:108D60005146BFA0FBF760FDA9A0FBF75DFDC6A0C3
:108D7000FBF75AFD4FF480200146F5F7DEFBC9A052
:108D8000FBF752FD0025B1B2CCA26A48FDF7B9F954
:108D900038B10F30EFF75AFD050002D0B5F5406F3E
:108DA00005D922462946C9A0FBF782FDA7E0B0B24B
:108DB000FDF76EF90026F2F72BFF00903BE0B8F8C4
:108DC00000004746A0B1F2F723FF00903F88A81BA0
:108DD00081B2B94200D287B2C4483A4630445549BC
:108DE000EFF717FEF01986B23846FDF751F922E089
:108DF000F2F70EFF0099401A44F62061884217D915
:108E00002B4632462146BAA0FBF752FDB8F80010B7
:108E1000C1480068CDE90001C04890F83A20406B95
:108E200000684168BE480368BEA0FBF741FD66E0EC
:108E30001420F7F738FFAE42C1D304F580202A464C
:108E4000AA490646F5F74EFE2A46A8493046F5F7E8
:108E500009FE10B10026A54F0BE02146C0A0FBF78C
:108E6000CDFC4CE0B95D5846F8F742FF761C8346CE
:108E7000B6B2AE42F6D32C4464206043B0FBFAF1A4
:108E8000642900DD64210A2091FBF0F33C9A92FBF7
:108E9000F0F083420ADD53462246BCA03C91FBF72A
:108EA000C3FC4FF40051BE48F2F7A5FE54450BD366
:108EB0005946BCA0409AFBF7B7FC409858B140997E
:108EC0008B4508D0C1A018E004F6FF30BAF1000FBE
:108ED0003FF4CCAECBE651464FF48020F5F7CCFA08
:108EE00050B14A99C3A0C1F800A05146FBF79CFCC1
:108EF000002041B0BDE8F08FC7A0FBF77FFC4FF02A
:108F0000FF30F6E73E2057694669204F54413A202A
:108F1000C1ACBDD3B9CCBCFEB7FECEF1C6F7CAA773
:108F2000B0DC000072000020C8B801080D0A0D0A6C
:108F300000000000442E0020485454502F00000030
:108F40003E2057694669204F54413A20CFECD3A6C2
:108F5000D2ECB3A32040257500000000434C4F53D2
:108F6000454400003E2057694669204F54413A204D
:108F7000B7FECEF1C6F7B9D8B1D5C1ACBDD320404C
:108F8000257500003E2057694669204F54413A201C
:108F9000CFECD3A6CDB7B3ACCAB120402575000045
:108FA00020323036000000003E2057694669204FCD
:108FB00054413A20B7C72032303620CFECD3A6A395
:108FC000A8B7FECEF1C6F7B2BBD6A7B3D620526182
:108FD0006E67653FA3A93A20252E36307300000046
:108FE000636F6E74656E742D72616E67653A000012
:108FF0003E2057694669204F54413A20B9CCBCFE07
:10900000D7DCB4F3D0A1D2ECB3A3202575000000C7
:109010002A2A2A2A2A2A2A2A2A2A2A2A2A2A2A2AB0
:109020002A2A2A2A2A2A2A2A2A2A2A2A2A2A2A2AA0
:109030002A2A2A2A2A2A00002A202057694669203B
:109040004F544120C9FDBCB6BFAACABC2020202075
:10905000202020202020202020202020202A000046
:109060002A2020B9CCBCFEB4F3D0A13A202575202B
:10907000D7D6BDDA2020202020202020202020202C
:1090800020202020202A00003E20D5FDD4DAB2C1C5
:10909000B3FD2057323551363420D0C2B2DBCEBBBF
:1090A0002E2E2E003E2057323551363420D0C2B2FB
:1090B000DBCEBBB2C1B3FDCDEAB3C900636F6E7442
:1090C000656E742D6C656E6774683A003E20576952
:1090D0004669204F54413A20BFE9B3A4B6C8D2EC48
:1090E000B3A320257520402575000000EE56002012
:1090F0003E2057694669204F54413A20CAFDBEDDE3
:10910000BDD3CAD5B3ACCAB12040257520D2D1CACF
:10911000D52025752F25750054010020BC8800201E
:10912000500100203E204F544120D5EFB6CF3A20C9
:10913000434E4454523D25752052785374617465F2
:109140003D257520727863706C743D2575206F72B3
:10915000653D25752070656E64696E673D257500F7
:109160003E2057694669204F54413A2057323551C5
:10917000363420BBD8B6C1D0A3D1E9CAA7B0DC2011
:109180006F66667365743D25750000003E205B25A3
:10919000336425255D2025752F25754200000000CC
:1091A000001001403E20573235513634204352439F
:1091B00031363D3078253034582028B7FECEF1C600
:1091C000F73D307825303458290000003E2057699B
:1091D0004669204F54413A20435243313620D0A3B0
:1091E000D1E9B2BBC6A5C5E4A3A1D6D0D6B9CFC23A
:1091F000D4D800003E2057694669204F54413A2098
:10920000CFC2D4D8CDEAB3C9A3AC25754220D0A330
:10921000D1E9CDA8B9FD00003E2057694669204F2D
:1092200054413A20B9CCBCFECDB7D0A3D1E9CEDEB3
:10923000D0A700001CB5264908780190FF200870CF
:1092400008788DF800009DF800009DF8002000F0DF
:10925000F000904207D0502080F31188BFF34F8F69
:10926000BFF36F8FFEE79DF800001A4B00F050002F
:1092700018700720986005E09DF8002052008DF8D6
:109280000020401E9DF800201206F5D498600328A7
:1092900007D0502080F31188BFF34F8FBFF36F8F3B
:1092A000FEE74FF440709860019808700A48016822
:1092B00041F470010160016841F070410160FFF705
:1092C000A7FA00205860EFF709F800201CBD000045
:1092D00000E400E03800002020ED00E010B5024678
:1092E0000021012000F00CF8040007D000214160AB
:1092F00001600B460A46C16000F06AF8204610BDC6
:1093000070B50E46050013D0D6B105FB06F0483007
:10931000FDF7BEFE040009D004F1480120468EB1DD
:109320000160C0E90F56012100F00EF8204670BD23
:10933000502080F31188BFF34F8FBFF36F8FFEE78C
:109340000020E4E70060ECE770B50D46040025D08E
:10935000FFF7FCF9D4E90F20216802FB00116160DE
:109360000021A1632168A1600A46D4E90F01401ED3
:1093700000FB0121E16021464FF0FF3001F8440F6E
:10938000487004F110008DB1FFF7AEF904F124002C
:10939000FFF7AAF9FFF7FAF9012070BD502080F31A
:1093A0001188BFF34F8FBFF36F8FFEE7216900294C
:1093B000F0D000F02DFB0028ECD004494FF0805095
:1093C0000860BFF34F8FBFF36F8FE3E704ED00E05A
:1093D0002DE9FF4782B01D468A464FF00008040081
:1093E00003D0BAF1000F08D011E0502080F31188AB
:1093F000BFF34F8FBFF36F8FFEE7206C38B1502063
:1094000080F31188BFF34F8FBFF36F8FFEE7022DFC
:109410000AD1E06B012807D0502080F31188BFF3F8
:109420004F8FBFF36F8FFEE700F0EAF93F4F4FF029
:1094300000094FF0805648B9049838B1502080F3A5
:109440001188BFF34F8FBFF36F8FFEE7FFF77EF9F1
:10945000A06BE16B884207D3022D05D00498D0B1F0
:10946000B8F1000F1AD01EE02A4651462046FDF7FB
:10947000ABFC616A19B104F1240000F0C9FA20B113
:109480003E60BFF34F8FBFF36F8FFFF77FF901206F
:1094900006B0BDE8F087FFF779F922E06846FFF7EC
:1094A000EFF94FF00108FFF771F9FFF797FAFFF7AF
:1094B0004DF994F94400401C01D184F8449094F98A
:1094C0004500401C01D184F84590FFF75FF904A9DD
:1094D000684600F029F930B12046FDF78BFD00F019
:1094E000D1FA0020D4E7FFF731F9A06BE16B884295
:1094F00013D1FFF74BF904F110000499FFF7CEF9EF
:109500002046FDF777FD00F0BDFA00289ED13E60B1
:10951000BFF34F8FBFF36F8F98E7FFF737F9204600
:10952000FDF768FD00F0AEFA90E7000004ED00E002
:1095300010B5040009D000F05DF96168884214D1CB
:10954000E068401EE06008D00DE0502080F31188F4
:10955000BFF34F8FBFF36F8FFEE700231A46194604
:109560002046FFF735FF012010BD002010BD000090
:109570002DE9F343002683B00400354609D0206C62
:1095800078B1502080F31188BFF34F8FBFF36F8FF6
:10959000FEE7502080F31188BFF34F8FBFF36F8F2A
:1095A000FEE700F02DF9DFF83C814FF000094FF0A5
:1095B000805748B9049838B1502080F31188BFF320
:1095C0004F8FBFF36F8FFEE7FFF7C0F8A06BC8B1F6
:1095D000401EA063206810B9FDF7CAFD60602069D5
:1095E00050B104F1100000F013FA28B1C8F800706F
:1095F000BFF34F8FBFF36F8FFFF7C8F8012005B09F
:10960000BDE8F083049808B166B10FE03DB1502089
:1096100080F31188BFF34F8FBFF36F8FFEE7FFF723
:10962000B5F85DE06846FFF72BF90126FFF7AEF8C5
:10963000FFF7D4F9FFF78AF894F94400401C01D1F0
:1096400084F8449094F94500401C01D184F8459079
:10965000FFF79CF804A9684600F066F80028204649
:1096600012D0FDF7C7FC00F00DFA2046FDF790FC84
:109670000028A9D09DB3FFF769F8606A50B3206B4A
:109680000068C0F1050126E0FDF782FCE0B120682A
:1096900038B9FFF75BF8606800F070F90546FFF72E
:1096A00075F804F124000499FFF7F8F82046FDF757
:1096B000A1FC00F0E7F9002886D1C8F80070BFF3DC
:1096C0004F8FBFF36F8F7FE72046FDF793FC00F0CD
:1096D000D9F979E700216068FFF7F8F89FE7FFE71D
:1096E00000208CE704ED00E070B50D46040009D0C1
:1096F00000F080F8616888420CD1E068401CE060AE
:10970000012070BD502080F31188BFF34F8FBFF34D
:109710006F8FFEE729462046FFF72AFF0028F0D08A
:10972000E168491CE16070BD2DE9F0410C4605007F
:1097300011D0C4B1FFF70AF8174B1A696E68206898
:10974000911B471C17D02F685B6A9F4219D0964225
:1097500017D8012410E0502080F31188BFF34F8FF9
:10976000BFF36F8FFEE7502080F31188BFF34F8F58
:10977000BFF36F8FFEE70024FFF708F82046BDE82F
:10978000F081884205D9401A20602846FFF778F812
:10979000F1E700202060DCE7000000202DE9FF5FFA
:1097A0008346DDE90E87994616468A469000FDF706
:1097B0006FFC05001AD05420FDF76AFC040012D09B
:1097C00025630021CDE90241CDE900874B463246B1
:1097D00051465846FDF768FB2046FDF791FA0120F7
:1097E00004B0BDE8F09F2846FEF7E4FF4FF0FF30DD
:1097F000F6E7000001480068704700000000002004
:109800000548816919B1406B18B1002070470120EB
:109810007047022070470000000000202DE9F04151
:109820002E4C0027606B40B1E069401CE061206A6B
:1098300000B101273846BDE8F0812669761C266113
:1098400013D16068006838B1502080F31188BFF3ED
:109850004F8FBFF36F8FFEE76068A1686160A06003
:10986000606A401C6062FDF7A1FBE06ADFF870806F
:10987000864209D36068006880B16068C068C568C6
:10988000686886420DD2E0622068C06A00EB800101
:1098900058F821000128CAD90127C8E74FF0FF3046
:1098A000F1E7281DFEF7D6FEA86A18B105F11800E9
:1098B000FEF7D0FEE86A01216269814011436161CF
:1098C00000EB800108EB8100291DFEF733FFE86AF9
:1098D0002168C96A8842CDD30127CBE70000002068
:1098E0004402002070B504004FF0000140D0214D2B
:1098F0002868844207D0502080F31188BFF34F8F2F
:10990000BFF36F8FFEE7A06C38B1401EA064636C9C
:10991000E26A9A422CD040B12AE0502080F31188AC
:10992000BFF34F8FBFF36F8FFEE7201DFEF792FE50
:10993000114A012150B9E06A00EB800352F823304C
:1099400023B96B6901FA00F083436B61606CE062DC
:10995000C0F10500A061E06A6B698140194369614B
:1099600000EB800002EB8000211DFEF7E3FE0121E9
:10997000084670BD000000204402002070B50400BD
:109980004FF0000038D0204DE16A2A68D26A914237
:1099900033D2A069002804DB2868C06AC0F1050042
:1099A000A0611A4E01EB8101606906EB81018842DA
:1099B0001ED1201DFEF74EFE012150B9E06A00EBDA
:1099C000800256F8222022B96A6901FA00F0824327
:1099D0006A612868C06AE0626A698140114369610E
:1099E00000EB800006EB8000211DFEF7A3FE02E0E5
:1099F0002868C06AE062012070BD616C2A68D26A82
:109A00009142F8D370BD0000000000204402002005
:109A10002DE9F041C068C468ACB104F118000746F4
:109A2000FEF718FE154D686B0126A0B139461448A3
:109A3000FEF780FEE06A2968C96A88421CD90120C5
:109A40002E62BDE8F081502080F31188BFF34F8F64
:109A5000BFF36F8FFEE7201DFEF7FCFDE16A6A6928
:109A600006FA01F01043686101EB810004498C396A
:109A700001EB8000211DDBE70020E2E70000002071
:109A8000D00200202DE9F0472C4D00242746686BBA
:109A900038B1FEF75BFE686B401E6863686B40B1CF
:109AA00046E0502080F31188BFF34F8FBFF36F8FD4
:109AB000FEE7E968224E0120D1B3A6F18C09804669
:109AC0003068E8B1F068C46804F11800FEF7C2FD20
:109AD000201DFEF7BFFDE06A6A6908FA00F1114334
:109AE000696100EB800109EB8100211DFEF722FE78
:109AF000E06A2968C96A8842E2D3C5F82080DFE7B6
:109B00000CB1FDF753FAEC6944B14646FFF786FE07
:109B100000B12E62641EF9D10020E861286A38B1D4
:109B20000849012738070860BFF34F8FBFF36F8FD5
:109B3000FEF72CFE3846BDE8F0870000000000204C
:109B4000D002002004ED00E010B500290AD008780A
:109B5000002807D005487844EFF790F8002801D096
:109B6000002010BD0248784410BD0000D61F000040
:109B7000CE1F000010B500290AD00878002807D0B1
:109B800005487844EFF77AF8002801D0002010BD8E
:109B90000248784410BD0000BA200000B220000046
:109BA00021F00042A2F16052B2F5801F01F00043A3
:109BB00028BFD2F17F6C0BD95FEA001C43EAC202D6
:109BC00042EB507018BF704728BF20F0010070476B
:109BD000B2F5801FBCBF184670474FEA410C1CF518
:109BE000001F02D2084601F096B870B500F0E0FB05
:109BF00000000089FFF7F6BF4FF00040A0F580009D
